:020000040001F9
:100000003868022099020100E9CE0100258801002C
:1000100027CD010031380100D94F02000000000057
:10002000000000000000000000000000E12E0200BF
:10003000B9560100000000004D0E0200B137020069
:100040001598010025980100359801004598010098
:100050005598010065980100759801008598010088
:1000600095980100A5980100B5980100C598010078
:10007000D5980100E5980100F59801000599010067
:100080001599010025990100359901004599010054
:100090005599010065990100759901008599010044
:1000A00095990100A5990100B5990100C599010034
:1000B000D5990100E5990100F5990100059A010023
:1000C000159A0100299A01003D9A0100519A0100F8
:1000D000659A0100799A01008D9A0100A19A0100A8
:1000E000B59A0100C99A0100DD9A0100F19A010058
:1000F000059B0100199B01002D9B0100419B010004
:10010000559B0100699B01007D9B0100919B0100B3
:10011000A59B0100B99B0100CD9B0100E19B010063
:10012000F59B0100099C01001D9C0100319C010010
:10013000459C0100599C01006D9C0100819C0100BF
:10014000959C0100A99C0100BD9C0100D19C01006F
:10015000E59C0100F99C01000D9D0100219D01001D
:10016000359D0100499D01005D9D0100719D0100CB
:10017000859D0100999D0100AD9D0100C19D01007B
:10018000D59D0100E99D0100FD9D0100119E01002A
:10019000259E0100399E01004D9E0100619E0100D7
:1001A000759E0100899E01009D9E0100B19E010087
:1001B000C59E0100D99E0100ED9E0100019F010036
:1001C000159F0100299F01003D9F0100519F0100E3
:1001D000659F0100799F01008D9F0100A19F010093
:1001E000B59F0100C99F0100DD9F0100F19F010043
:1001F00005A0010019A001002DA0010041A00100EF
:1002000055A0010069A001007DA0010091A001009E
:10021000A5A00100B9A00100CDA00100E1A001004E
:10022000F5A0010009A101001DA1010031A10100FB
:1002300045A1010059A101006DA1010081A10100AA
:10024000DB020100DB020100DB020100DB02010036
:10025000DB020100DB020100DB020100DB02010026
:10026000DB020100DB020100DB020100DB02010016
:10027000DB020100DB020100DB020100DB02010006
:10028000DFF810D000F004FC0048004765A1020030
:10029000AFF300803868022010484FF0770101600A
:1002A0000F484FF0770101600E484FF4885101600C
:1002B0000A484FF07601016009484FF0760101606D
:1002C0000948804709480047FEE7FEE7FEE7FEE7EA
:1002D000FEE7FEE7FEE7FEE7FEE7FEE7040805406F
:1002E0000C08054000080540713802008102010039
:1002F0002DE9F05F0546002092469B46884606465B
:10030000814640241BE0284641464746224600F0ED
:1003100089FA53465A46C01A914110D311461846DD
:10032000224600F016F82D1A67EB01084F462246C8
:100330000120002100F00DF817EB00094E41201EAE
:10034000A4F10104DFDC484631462A464346BDE8B5
:10035000F09F202A04DB203A00FA02F100207047C7
:100360009140C2F1200320FA03F3194390407047F3
:10037000202A06DBCB17203A41FA02F043EAE07369
:1003800006E041FA02F3D040C2F120029140084356
:100390001946704740EA01039B0703D009E008C9EA
:1003A000121F08C0042AFAD203E011F8013B00F83A
:1003B000013B521EF9D27047D2B201E000F8012B86
:1003C000491EFBD270470022F6E710B513460A46D5
:1003D00004461946FFF7F0FF204610BD2DE9FE4FF9
:1003E000804681EA0300C00F0C46009021F00041D6
:1003F00023F00045B8EB0200A94105D24046214652
:1004000090461C460B46024623F00040104347D05E
:10041000270DC7F30A00C3F30A510290401A019056
:1004200040286BDAC3F3130040F4801B0098924617
:1004300020B10023D2EB030A63EB0B0B0198594662
:10044000C0F140025046FFF784FF06460D46504675
:100450005946019AFFF78CFF10EB08006141002418
:1004600087EA115284EAE7731A4340D0009A62B3D4
:10047000019A012A4FEA075215DC001B61EB0201C9
:100480004FF0004202EA0752CDE90042001C41F55C
:10049000801132462B4600F01BFA03B0BDE8F08F06
:1004A00040462146F9E7001B61EB0201001C41F5C3
:1004B000801300185B412018A2F5001747EB0301D9
:1004C00040EAD570B6196D4111E06D084FEA360665
:1004D00045EAC0754FEA0752001B61EB0201001CA0
:1004E00041F5801149084FEA300000195141324668
:1004F0002B4603B0BDE8F04F00F0DBB900980122B5
:1005000040000023D0EB020263EBE0730098214629
:100510004FEAE074B8EB000061EB0401E9E783F017
:1005200000435BE781F0004158E72DE9FE4F81EA87
:10053000030404F0004421F0004100944FF0000B4C
:1005400023F0004350EA01045ED052EA03045BD07A
:10055000C3F30A54C1F30A552C44A4F2F3340194B2
:10056000A0FB0254C1F3130141F48011C3F3130340
:1005700043F4801301FB024400FB034E840A970AF4
:1005800044EA815447EA8357A4FB076802958D0A21
:1005900005FB07854FEA932C04FB0C542705029DAD
:1005A0004FEA065847EA1637B5EB08056EEB070C1D
:1005B000870E920E47EA811742EA8312A7FB0201D7
:1005C000B6EB0B0164EB00042B0D43EA0C335E1811
:1005D00044EB1C50DA465146E7FB0201C5F3130415
:1005E0004FEA0B3343EA14534FEA0432019C43EAC7
:1005F0000603A4F10C040294009CCDE900B400F0C1
:1006000067F903B0BDE8F08F00200146F9E72DE956
:10061000F04D81EA030404F0004B21F0004514463C
:100620004FF0000A23F0004150EA050220D054EABE
:1006300001021DD0C5F30A570246C5F31303C1F3E7
:100640001300C1F30A5640F4801543F48013A7EB5E
:100650000608101BD64608F2FD3873EB050002D3DE
:1006600008F1010801E092185B41B8F1000F03DACC
:1006700000200146BDE8F08D00204FF480110646B1
:1006800084460EE0171B73EB050705D3121B63EBC3
:10069000050306434CEA010C49084FEA3000921862
:1006A0005B4150EA0107EDD152EA030012D082EA21
:1006B000040083EA0501084305D0101BAB4106D2B4
:1006C0000122002306E000224FF0004302E06FF019
:1006D000010253101AEB06004CEB085110EB0A0014
:1006E00041EB0B01BDE8F04D00F0E3B80EB540F270
:1006F000334102910021CDE900110A460B4600F07A
:10070000E7F803B000BDC1F30A5210B5C1F31301FD
:1007100040F2FF3341F480119A4201DA002010BD0B
:1007200040F233439A42A2F2334203DC524200F0D9
:1007300079F810BD904010BD00F0004230F000404C
:100740000AD0C10D01F56071C0F3160042EA0151F3
:10075000C20840071143704700200146704700005F
:1007600030B5041E71F1000404DB4FF00044404238
:1007700064EB0101141E73F1000405DB1C464FF00D
:100780000043524263EB04038B4208BF824230BDF8
:1007900030B5041E71F1000404DB4FF00044404208
:1007A00064EB0101141E73F1000405DB1C464FF0DD
:1007B0000043524263EB0403994208BF904230BDAC
:1007C00001F0004330B421F0004150EA010206D0AC
:1007D0000A0DA2F56072C1F31301002A02DC30BCDD
:1007E00000207047440F44EAC104C100E01830BC47
:1007F00000EBC25000F026B830B50B460146002091
:100800002022012409E021FA02F59D4205D303FAD2
:1008100002F5491B04FA02F52844151EA2F1010253
:10082000F1DC30BD202A04DB203A21FA02F000215D
:10083000704721FA02F3D040C2F1200291400843F0
:10084000194670470029A8BF7047401C490008BFDF
:1008500020F00100704710B4B0FA80FC00FA0CF0F0
:1008600050EA010404BF10BC704749B1CCF1200428
:1008700021FA04F411FA0CF118BF012121430843B5
:10088000A3EB0C01CB1D4FEA00614FEA102042BFE1
:10089000002010BC704700EBC35010440029A4BFD7
:1008A00010BC7047401C490008BF20F0010010BC7C
:1008B000704710B5141E73F1000408DA401C41F1B2
:1008C000000192185B411A4301D120F0010010BDD4
:1008D0002DE9F04D92469B4611B1B1FA81F202E04A
:1008E000B0FA80F220329046FFF733FD04460F46FF
:1008F00040EA0A0041EA0B0153465A46084313D026
:10090000114653EA010019D0C8F140025046FFF7E2
:1009100089FF05460E46504659464246FFF719FDE7
:10092000084305D0012004E020463946BDE8F08D9B
:100930000020054346EAE0762C4337430A986305D6
:10094000E40AA0EB08000022FD0A44EA47540A30FA
:1009500002D500200146E9E7010510196941DDE9EA
:10096000084500196941BDE8F04DA2E770B521F0D6
:10097000004303430CD0C1F30A550024D5EB040512
:1009800064EB0403D617AD1AB34102DB0020014625
:1009900070BD201841EB025170BD2DE9F04D0023D0
:1009A0001A461B1A8A4103DB00200146BDE8F08D80
:1009B000C1F30A52C1F3130141F480154FF0000B4B
:1009C000D10702D100186D41521E0027044640F2A3
:1009D000FF11384601EB620A3E468046024600207F
:1009E0004FF48011FFF71EFFC2197141BB1846EB8F
:1009F0000100B4EB030C75EB000C04D3E41A65EBB7
:100A0000000517460E46241908F101006D41804685
:100A10003428E3DDF91946EB0600091BA84103D28F
:100A20004FF0FF32134601E0002213461BEB070094
:100A300046EB0A51BDE8F04DFFF73BBF0EB5C10FC5
:100A400080EAE0700844CA07002140F233438DE891
:100A50000E000A460B46FFF73BFF03B000BDC1F393
:100A60000A52C1F3130140F2FF3341F480119A425C
:100A700002DA00200146704740F233439A42A2F264
:100A8000334202DC5242FFF7CDBEFFF762BC0000EA
:100A9000064C074D06E0E06840F0010394E80700CB
:100AA00098471034AC42F6D3FFF7EEFBE0A5030005
:100AB00010A6030070B58C1810F8015B15F0070341
:100AC00001D110F8013B2A1106D110F8012B03E0E7
:100AD00010F8016B01F8016B5B1EF9D12B0705D4EF
:100AE0000023521E0DD401F8013BFAE710F8013B38
:100AF000CB1A921C03E013F8015B01F8015B521E54
:100B0000F9D5A142D8D3002070BD48F25B0CC1F6E4
:100B1000FF7C604748F2390CC1F6FF7C604748F221
:100B2000010CC1F6FF7C604748F2A51CC1F6FF7CB2
:100B30006047000070B504460D460420002C43D0E9
:100B4000002D41D0297901293ED8204EB44207D04A
:100B50001F48844204D040F25A211EA004F05EFDDA
:100B6000B44214D12868C0F31000297939B1218A20
:100B700001432182618A41EA104161820FE0A1892B
:100B80000143A181E18941EA1041E18107E0288820
:100B9000C0F30800297931B1218A01432182002163
:100BA000002220340EE0A1890143A181F7E7C307A9
:100BB00005D01346AE68521CD2B2F35C63544008B1
:100BC000491CC9B20028F2D170BD000000000440E9
:100BD000000404402E2E5C2E2E5C2E2E5C2E2E5CED
:100BE0002E2E5C6472697665725C7372635C6863F6
:100BF0003332663436305F6164632E630000000078
:100C000070B504460D460420002C1ED00F4EB44291
:100C100007D00F48844204D040F221310DA004F0E7
:100C2000FDFCB44202D1C5F3100001E0C5F3080099
:100C30004FEA1041A28A42EA0002A28203D1E08A6E
:100C400040EA0100E0824FF0000070BD0000044067
:100C5000000404402E2E5C2E2E5C2E2E5C2E2E5C6C
:100C60002E2E5C6472697665725C7372635C686375
:100C70003332663436305F6164632E6300000000F7
:100C800070B504460D46002C10D00948844207D0A8
:100C90000848844204D040F2F24107A004F0BEFCB0
:100CA00014F8460F0121A9408843207070BD000050
:100CB00000000440000404402E2E5C2E2E5C2E2EDC
:100CC0005C2E2E5C2E2E5C6472697665725C73728B
:100CD000635C68633332663436305F6164632E630D
:100CE0000000000010B500F0D3FB00F07FFB00F027
:100CF00053FCBDE8104004F0E3BC000070B50446AE
:100D00000D460420002C18D00C48844207D00C4813
:100D1000844204D040F2FE210AA004F07FFC3DB1E1
:100D2000681E062804D940F2FF2106A004F076FCD4
:100D3000608865F30A206080002070BD00000440D8
:100D4000000404402E2E5C2E2E5C2E2E5C2E2E5C7B
:100D50002E2E5C6472697665725C7372635C686384
:100D60003332663436305F6164632E630000000006
:100D700070B504460D46002C07D0601E0D2804D91E
:100D800040F22A410AA004F049FC012D05D025B10A
:100D900040F22B4106A004F041FC1048018864F3A6
:100DA00003010180818965F30001818170BD00002C
:100DB0002E2E5C2E2E5C2E2E5C2E2E5C2E2E5C6437
:100DC00072697665725C7372635C68633332663431
:100DD00036305F6164632E6300000000C20004408F
:100DE00010B502220021064804F046F9054C2046C1
:100DF00000F07CFA2046BDE810400021FFF740BF1C
:100E0000003005400000044070B504460D46042043
:100E1000002C1AD00D4EB44207D00D48844204D0A5
:100E200040F2A7210BA004F0F9FB280CA189A943EB
:100E3000A181218AA9432182B44205D1E18981435C
:100E4000E181618A81436182002070BD000004401D
:100E5000000404402E2E5C2E2E5C2E2E5C2E2E5C6A
:100E60002E2E5C6472697665725C7372635C686373
:100E70003332663436305F6164632E6300000000F5
:100E80002DE9F0470546884617461C46042005F123
:100E90005006002D2AD0002F28D0002C26D0DFF8B5
:100EA00050904D4507D01348854204D040F2AB51D5
:100EB00011A004F0B3FB4D4502D1C8F3100001E0CE
:100EC000C8F30800002100230CE0C20707D036F861
:100ED000112027F813205B1CDBB2641EE4B240082B
:100EE000491CC9B208B1002CEFD10020BDE8F08741
:100EF00000000440000404402E2E5C2E2E5C2E2E9A
:100F00005C2E2E5C2E2E5C6472697665725C737248
:100F1000635C68633332663436305F6164632E63CA
:100F20000000000070B504460E46002509488442C2
:100F300007D00948844204D040F2D64107A004F00B
:100F40006DFB94F846000121B140084200D0012514
:100F5000284670BD00000440000404402E2E5C2E84
:100F60002E5C2E2E5C2E2E5C2E2E5C6472697665B5
:100F7000725C7372635C68633332663436305F610F
:100F800064632E630000000070B504460D46042023
:100F9000002C56D0002D54D02A48844206D02A482E
:100FA000844203D0F82129A004F038FB28780228D5
:100FB00006D0012804D018B1F92124A004F02EFB9A
:100FC000687828B1012803D0FA2120A004F026FB7C
:100FD000A878012804D018B1FB211CA004F01EFB46
:100FE000E87848B1012807D0022805D0032803D0AB
:100FF000FC2116A004F012FB287928B1012803D0A7
:10100000FD2112A004F00AFB002020702A786188DC
:1010100062F3051161806A78618862F3C7116180AB
:10102000AA78618862F386116180EA78618862F348
:10103000010161802A79A18862F38201A18084F88C
:10104000470070BD00000440000404402E2E5C2EBA
:101050002E5C2E2E5C2E2E5C2E2E5C6472697665C4
:10106000725C7372635C68633332663436305F611E
:1010700064632E630000000010B50446002C06D007
:10108000012C04D040F23C4109A004F0C7FA1348F7
:10109000012C05D030F8C01F21F00F01018010BDD8
:1010A00030F8C01F21F00F010E31018010BD00008B
:1010B0002E2E5C2E2E5C2E2E5C2E2E5C2E2E5C6434
:1010C00072697665725C7372635C6863333266342E
:1010D00036305F6164632E6300000000000004404E
:1010E00010B50446002C17D0012C15D0022C13D0BB
:1010F000042C11D0082C0FD0102C0DD0202C0BD08C
:10110000402C09D0802C07D0B4F5807F04D040F269
:10111000574103A004F082FA0C48048010BD00007F
:101120002E2E5C2E2E5C2E2E5C2E2E5C2E2E5C64C3
:1011300072697665725C7372635C686333326634BD
:1011400036305F6164632E6300000000CC00044011
:101150003EB5434C204600F09BF800212046FFF7A7
:10116000E1FE0028F9D006236A4640F23B112046F2
:10117000FFF786FE00212046FFF782FDBDF80A003A
:101180009FED381A00EE100A384CF8EE400A81EE56
:10119000200ADFED350A20EE200A84ED000ABDF8B2
:1011A000060001EE100AF8EE411A81EEA01A21EEB7
:1011B000001A84ED031ABDF8080001EE100AF8EEDB
:1011C000411A81EEA01A21EE000A84ED020ABDF850
:1011D000000000EE100AB8EE400A84ED040ABDF8E3
:1011E000020000EE100AB8EE400A84ED050ABDF8D0
:1011F000040000EE100AB8EE400A70EEC00A00EEDD
:10120000100AB8EE401A80EE810A10EE100AFFF7BD
:1012100093FA41EC100B14F077F99FED151B51EC8C
:10122000100B53EC112BFFF780F99FED131B53ECC0
:10123000112BFFF7D3F841EC100B53EC102B9FED63
:10124000100B51EC100BFFF7E2F99FED0F1B53EC65
:10125000112BFFF764F9FFF7B3FA60603EBD0000A1
:1012600000040440BE9F8A3F00F07F458083FF1F3B
:101270000000006066A272400000000000F4AA4076
:101280000000000013642F410000006066127140EE
:1012900010B504460420002C0DD00748844207D026
:1012A0000648844204D040F2944105A004F0B6F907
:1012B00001202070002010BD000004400004044004
:1012C0002E2E5C2E2E5C2E2E5C2E2E5C2E2E5C6422
:1012D00072697665725C7372635C6863333266341C
:1012E00036305F6164632E630000000038B5044649
:1012F000042100250095002C19D00E48844207D007
:101300000D48844204D040F2B1410CA004F086F9AB
:10131000002142F2107207E025700098401C0090F6
:10132000904201D9092102E020780128F4D0084632
:1013300038BD000000000440000404402E2E5C2E46
:101340002E5C2E2E5C2E2E5C2E2E5C6472697665D1
:10135000725C7372635C68633332663436305F612B
:1013600064632E630000000070B504460E46154607
:101370000420002C1AD0012E18D80F48844207D020
:101380000E48844204D04FF4F3710DA004F046F9E6
:1013900035B1012D04D040F2E71109A004F03EF967
:1013A0002EB1608965F3CF306081002070BD608907
:1013B00065F3C7106081F8E70000044000040440B2
:1013C0002E2E5C2E2E5C2E2E5C2E2E5C2E2E5C6421
:1013D00072697665725C7372635C6863333266341B
:1013E00036305F6164632E630000000030B587B063
:1013F00022A00068039022A003C8CDE901010020CB
:101400000590042104918DF8140003A806901E4C49
:101410000222204600F05EF804A92046FFF78AFB6E
:1014200001210020FFF7A4FC0420FFF759FE012052
:10143000FFF722FE40F23B14049401A80690134DDE
:1014400002222146284600F045F804A92846FFF765
:1014500071FB01212846FFF751FC21462846FFF782
:10146000CFFB012108020FF075FC102002F05CFE9A
:1014700001200FF0A9FC07B030BD000011000000F2
:10148000FFFFFF64646400000000044000040440A7
:101490001CB50024009401948DF800408DF80140A3
:1014A00001208DF80300012108460FF053FC694626
:1014B0000648FFF769FD0094012102200FF04AFC65
:1014C00069460348FFF760FD1CBD000000000440B2
:1014D000000404402DE9F0411746002500260B4A80
:1014E000904201D18CB20CE0CCB2042609E0E007B6
:1014F00004D0A819C0B2394600F00AF864086D1C7F
:10150000EDB2002CF3D1BDE8F081000000000440F2
:101510007CB504460D4600200121012200230093E2
:1015200001938DF800508DF80430102C2DD2DFE897
:1015300004F02D080A0C0E10121416181B1D20237F
:101540002629022122E0042120E008211EE01021AA
:101550001CE020211AE0402118E0802116E0012043
:1015600014E00120022111E002200FE002200221FC
:101570000CE00220042109E00220082106E00220FC
:10158000102103E00220202100E00022002A02D0E6
:101590006A460EF013FF7CBD70B5012148040FF0C0
:1015A00025FB0C4C002211462046FFF7DDFE0A4DBC
:1015B000002211462846FFF7D7FE002201212046CF
:1015C000FFF7D2FE2846BDE8704000220121FFF758
:1015D000CBBE000000000440000404402DE9F04FA1
:1015E0002DED048B83B0FE490A780020FD4EDFF814
:1015F000F893FE4FDFF8F883062A06D00A78042A0B
:101600000ED00A78052A0DD00DE03880A8F8000029
:1016100001223280F74A108089F80000087002E049
:10162000087000E00870502548F610440A2246234E
:1016300000211046CDE9004500F05CFD1422462350
:1016400000211046CDE9004500F054FD1E2246233E
:1016500000211046CDE9004500F04CFD282246232C
:1016600000211046CDE9004500F044FD322246231A
:1016700000211046CDE9004500F03CFD3C22462308
:1016800000211046CDE9004500F034FD46231A46FE
:1016900000211846CDE9004500F02CFD50224623DC
:1016A00000211046CDE9004500F024FD5A224623D2
:1016B00000211046CDE9004500F01CFD64224623C0
:1016C00000211046CDE9004500F014FD6E224623AE
:1016D00000211046CDE9004500F00CFD782246239C
:1016E00000211046CDE9004500F004FD822246238A
:1016F00000211046CDE9004500F0FCFC8C22462379
:1017000000211046CDE9004500F0F4FC9622462366
:1017100000211046CDE9004500F0ECFC0A239F2291
:1017200019460020CDE9004500F0E4FC14239F2277
:1017300019460020CDE9004500F0DCFC1E239F2265
:1017400019460020CDE9004500F0D4FC28239F2253
:1017500019460020CDE9004500F0CCFC32239F2241
:1017600019460020CDE9004500F0C4FC3C239F222F
:1017700019460020CDE9004500F0BCFC4FF0FF0AFF
:10178000CDE9004A002146230122084600F0B2FCC0
:10179000CDE9004A002101239F22084600F0AAFC5F
:1017A000CDE9004A46239F2200219E2000F0A2FCA2
:1017B000CDE9004A46239F224521002000F09AFCF3
:1017C0000C2001F0F1FC8C48008801F0F3FC46216C
:1017D000002001F0E3FC8949894C91ED000A10EEEC
:1017E000100AA04205DA022091ED000A01F01EFC69
:1017F00004E0012091ED000A01F018FC81A001F045
:1018000065F94621242001F0C9FC7F4991ED000AC9
:1018100010EE100AA04205DA022091ED000A01F054
:1018200005FC04E0012091ED000A01F0FFFB77A028
:1018300001F04CF94621482001F0B0FC744991EDCB
:10184000000A10EE100AA04205DA022091ED000A0B
:1018500001F0ECFB11E091ED000A6E4A10EE100A67
:10186000904205DA012091ED000A01F0DFFB04E06F
:10187000002091ED000A01F0D9FB67A001F026F9E4
:101880004621762001F08AFC30880321400001F0D7
:101890003FFC62A001F01AF90024DFF884B1DFED0B
:1018A000618A9FED618A614D9FED619A614ED9E039
:1018B000401E844238D13BF81400FF2300EE100A8A
:1018C00038882A88B8EE400A60EE280A00EE100A2E
:1018D000B8EE401A80EE810A38EE400ABCEEC00A2B
:1018E00010EE100AC1B2204600F0E4FB5248FF237C
:1018F000328830F8140000EE100AB8F80000B8EE94
:10190000400A60EE090A00EE100AB8EE401A80EEB6
:10191000810A38EE400ABCEEC00A10EE100AC1B2CD
:10192000204600F0C7FB9BE004F1010922463BF88A
:10193000190000EE100A3888B8EE400A60EE280A56
:1019400000EE100AB8EE401A80EE810A38EE400A26
:10195000BCEEC00A10EE101A8BB23BF8141000EE69
:10196000101AB8EE400A60EE280A00EE100AB8EE2F
:10197000401A80EE810A38EE400ABCEEC00A10EE32
:10198000100AC1B22888CDE9000A204600F0B2FB57
:101990002949DFED2A0A31F8190031F8141000EE58
:1019A000100AB8F80000B8EE400A60EE200A00EE17
:1019B000100AB8EE401A80EE810A38EE400ABCEEFA
:1019C000C00A10EE102A00EE101A93B2B8EE400AC8
:1019D00060EE090A00EE100AB8EE401A30E000008E
:1019E0006083FF1F048DFF1FFB8CFF1FFE8CFF1FFA
:1019F000008DFF1F028DFF1FAE83FF1F3483FF1F6B
:101A000000002041560000003C83FF1F4100000001
:101A10004083FF1F0000C84257000000532F64009E
:101A2000F45E02200000704200008C42A883FF1F79
:101A300000000C42AA83FF1F3460022000002042F5
:101A400080EE810A224638EE400ABCEEC00A10EE53
:101A5000100AC1B23088CDE9000A204600F04AFBE6
:101A6000641CE4B2244800788442FFF421AF288843
:101A700001F0A0FB388842F21074A04204D2002189
:101A80007F2001F08BFB03E00021782001F086FB32
:101A900038889FED1A8A00EE100A0220F8EE400AFC
:101AA00080EE880A01F0C2FAAFF2A80001F00EF849
:101AB000308801F07FFBB8F80000A04204D2142166
:101AC0007F2001F06BFB03E01421782001F066FB1E
:101AD000B8F8000000EE100A0220F8EE400A80EE8E
:101AE000880A01F0A3FAAFF2DC0003B0BDEC048B6E
:101AF000BDE8F04F00F0EABFFB8CFF1F00007A4406
:101B00001CB50021009101918DF8001001228DF883
:101B100001208DF802108DF803208DF804000221B9
:101B20008DF805108DF80600684602F043F91CBDDB
:101B30002DE9F04107468846164600240021384624
:101B400012F0DEFA05460121384612F0D9FA012ECC
:101B500006D04146384612F0D3FA012806D006E0F6
:101B6000012D01D0012802D1012400E00124012C23
:101B70000BD10020064942F21072096801E000BF53
:101B8000401CB1FBF2F38342F9D8BDE8F0810000BC
:101B9000B482FF1F2DE9FC4100F0FCF8102001F099
:101BA00003FB6748008801F005FB0021084601F0AF
:101BB000F5FA64A000F0D8FB0024DFF89881644EA9
:101BC0001927A8F56575308801F0F4FA07EB0410C1
:101BD000C1B2002001F0E2FA687B844212D10221F6
:101BE000002000F06FF90C2001F0DEFA5A4800885E
:101BF00001F0E0FA59A000F069FF6FF00101002048
:101C000000F060F9102001F0CFFA08EB84100068B2
:101C100000F0AAFB24B1012C63D0022C70D168E043
:101C2000A87B08286CD2DFE800F00F1A25303B466D
:101C300051044BA000F098FB0021022000F042F973
:101C400048A000F091FB5BE049A000F08DFB002173
:101C5000022000F037F947A000F086FB50E046A0D4
:101C600000F082FB0021022000F02CF941A000F0DE
:101C70007BFB45E041A000F077FB0021022000F053
:101C800021F93FA000F070FB3AE03FA000F06CFBB0
:101C90000021022000F016F939A000F065FB2FE0CA
:101CA0003AA000F061FB0021022000F00BF934A003
:101CB00000F05AFB24E036A000F056FB0021022081
:101CC00000F000F92EA000F04FFB19E02AA000F070
:101CD0004BFB0021022000F0F5F829A000F044FBA6
:101CE0000EE01FA000F040FB0021E87B01F010FA9D
:101CF00006E01BA000F038FB0021287C01F008FA68
:101D0000641CE4B2032CFFF45EAFFF243088CDE9FD
:101D100000049E224F230021104600F0EBF930888A
:101D2000CDE90004687B9F22C0EBC00101EB4013AA
:101D30005B1C00219D2000F0DDF9BDE8FC81000066
:101D4000AC83FF1FB1B3B9E2C9E8D6C300000000FD
:101D5000AA83FF1F4487FF1FA883FF1F3E000000C8
:101D60003A000000B1A3B3D6BFAAC6F40000000039
:101D70003A313500C3EB00003A3330003A3100000D
:101D8000B7D6D6D3000000003A3200003A35000042
:101D90003A3130002DE9F041464D2F78464C00266F
:101DA000042FA17B227C637BE07B12D02F780A2F4B
:101DB0000FD02F78052F27D02F780B2F24D095F810
:101DC00000C03E4FBCF1060F37D0287809285BD001
:101DD00064E023B1012B07D0022B5FD10CE007296F
:101DE0005CD2491CA17359E0642801D2401CE07305
:101DF000E07B09F001F851E0824201D2521C2274CA
:101E0000207C08F0F9FF49E023B1012B06D0022B1A
:101E100044D10BE0B9B3491EA1733FE0012801D9B9
:101E2000401EE073E07B08F0E7FF37E00AB1521E86
:101E30002274207C08F0E0FF30E094F800C0BCF190
:101E4000000F01D15B1C6373637B032B26D1BCF1B4
:101E5000000F23D102236373F9703871824200D9D5
:101E60002074207C787105F0C7FF387908F0C4FF32
:101E700013480168226B891AB1F5487F0ED90121F8
:101E800021700068206309E013B15B1E637304E0F6
:101E9000387908F0B1FF112060702E70287806287C
:101EA00005D02878052802D02878042800D12E7083
:101EB000BDE8F0816083FF1FB083FF1F74610220C3
:101EC0007C83FF1F034A937818449070D0780844AD
:101ED000D07070479C83FF1F024A9070D0780844EE
:101EE000D07070479C83FF1F2DE9FF4F85B0DDE95F
:101EF00012783844C6B2C81900F0FF09784202EBE4
:101F0000400101F0FF0CCDF81CC003EB4001CAB248
:101F100000243D46032101EB4001DDF81CC009EB24
:101F2000020A06EB0C0B48E0A9EB0502394B02EB69
:101F300082024FEA082003EB8212A6EB040E00EBAC
:101F40001820049222F81E00A9EB040202EB820280
:101F500003EB821C721BCDE9022C2CF812000AF054
:101F6000FF0202EB050C0CEB8C0C03EB8C1C2CF829
:101F70001E00224402EB820203EB821E029A2EF81C
:101F800012000BF0FF0213192CF813002A442EF84C
:101F90001200DDF810C02CF81300DDF80CC02CF88E
:101FA0001200641C002903DA01EB8401891D04E09E
:101FB000601B01EB80010A316D1EAC42B4DDFF24D1
:101FC000F01BCDE9008482B25346C0B2494600F00E
:101FD00091F80798F119CDE900840A185346D0B258
:101FE000494600F087F8A9EB0700CDE9008483B2E9
:101FF000C1B25A46304600F07DF8CDE900840AEBC4
:1020000007035A46D9B2304600F074F809B0BDE86B
:10201000F08F00004CD501202DE9FE4F0025002651
:10202000171AA3EB010881468A46681E002F03DDBC
:102030004FF00101019107E003D14FF00001019140
:1020400002E00190C7F10007B8F1000F03DD4FF087
:102050000100009007E003D14FF00000009002E083
:102060000090C8F10008474501DD3C4600E04446C9
:102070004FF0000B601C029017E00AF0FF0109F01E
:10208000FF00FF230C9A00F015F83D444644A5429A
:1020900002DD2D1B01988144A64202DD361B00980B
:1020A00082440BF1010B1FFA8BFB02988345E4DDA0
:1020B000BDE8FE8F30B504461046A02C16D8502936
:1020C00014D801EB81020A4901EB821535F814207E
:1020D0001AB1110A01EB02218AB20146184614F026
:1020E00057FF010201EB102025F8140030BD00005D
:1020F0004CD501202DE9F04F8046DDF824B016467E
:102100001F46B8F1A00F32D2502930D2A02E2ED2C5
:10211000502F2CD2B04503D9404606F0FF080646A2
:10212000B94202D90846F9B207460D46DFF844A085
:102130001BE0444615E005EB85000AEB801939F8F1
:1021400014201AB1100A00EB022082B259460A98F4
:1021500014F01EFF010201EB102029F81400641C8A
:10216000E4B2B442E7D96D1CEDB2BD42E1D9BDE89D
:10217000F08F00004CD501202DE9FF4F8CB0DDE938
:102180001986404400F0FF0901EB0800C0B20D9031
:10219000C8F1000002EB4001CAB20E9203EB40010D
:1021A000C9B200244546032202EB40070E9A09EB10
:1021B000020003900D98084402907DE030020D99D2
:1021C0005B4A491B0B9101EB810102EB8111A9EBE9
:1021D000040A00EB16200A9121F81A000D99A9EBC8
:1021E000050B091B099101EB810102EB811108919B
:1021F00021F81B000299CBB25919079101EB81011B
:1022000002EB811E2EF81A001919069101EB8101CB
:1022100002EB811121F81B00039AD2B202EB040CED
:10222000CDF814C02EF81C002A4421F812000A9997
:1022300021F81C000899049221F81200FF20CDE932
:1022400000600B991FFA8CF28BB2C9B20AF0FF0042
:10225000FFF750FFFF20CDE900600999049A8BB287
:1022600092B2C9B20BF0FF00FFF744FFFF20CDE9A7
:1022700000600799DDF814C08BB21FFA8CF2C9B266
:102280000AF0FF00FFF736FFFF20CDE90060069956
:10229000049A8BB292B2C9B20BF0FF00FFF72AFF8B
:1022A000641C002F03DA07EB8407BF1D04E0601BEA
:1022B00007EB80070A376D1EAC427FF77FAFFF2424
:1022C000CDE90064A9EB0805AAB2E8B2029B0D991A
:1022D000FFF710FF0E9809EB0801CDE900640A181A
:1022E000D0B2029B0D99FFF705FF0D98CDE9006470
:1022F000A0EB080083B2C1B24846039AFFF7FAFE8A
:102300000298CDE9006400EB0803D9B24846039A6D
:10231000FFF7F0FEDDE90230CDE9006400EB0802D2
:102320006D1CE8B20D99FFF7E5FE10B0BDE8F08F27
:102330004CD5012010B50021020A02EB0020094C07
:1023400082B2002001EB810304EB831323F81020F9
:10235000401C80B2A028F9D3491C89B25029F0D37F
:1023600010BD00004CD501202DE9F84F0746002490
:10237000DFF808841DE27E297ED99B23787800EB64
:10238000012081B20020FE4A13E032F830608E4214
:102390000DD802EBC00676888E4208D332F8303072
:1023A00002EBC000C91A8088084485B203E0401CD3
:1023B00080B29842E9D3BF1CF248F34A30F83500A6
:1023C0009178C0F1A0038B4202DA4FF0A00A02E03C
:1023D000084400F0FF0A92F80390B9F1400F02D9C7
:1023E000502000903BE009F11000C0B2009036E0B0
:1023F000E54886781EE009EB890008EB801B3BF876
:1024000016201AB1100A00EB022082B2DD48DF4923
:1024100000EBC50021444068405CDB49C98814F0EA
:10242000B7FD010201EB10202BF81600641CA4B2CA
:10243000761CF6B25645DED3BAF1A00F0BD1D148C7
:1024400030F83500B4FBF0F100FB1141C9B211B115
:102450002044401A84B209F1010909F0FF090098EB
:102460008145C5D30024C748C74910F835008A788C
:10247000104488709DE1FFE7C34A5078102807D0C8
:102480001C287DD00C287CD10A260020C04B14E1EA
:1024900012260020BF4B14E033F830C061450ED344
:1024A00003EBC00CBCF802C0614508D833F83050CB
:1024B00003EBC000491B8088084485B203E0401C40
:1024C00080B2B042E8D37F1CB248903030F835106B
:1024D0009078C1F1A003834202DA4FF0A00A02E033
:1024E000084400F0FF0A92F80390B9F1420F02D9B4
:1024F000502000903DE009F10E00C0B2009038E09D
:10250000A14886781FE009EB890008EB801B3BF8A7
:1025100016201AB1100A00EB022082B29D489E4993
:10252000903000EBC50021444068405C9649C98862
:1025300014F02EFD010201EB10202BF81600641C94
:10254000A4B2761CF6B25645DDD3BAF1A00F0CD179
:102550009048903030F83500B4FBF0F100FB1141A9
:10256000C9B211B12044401A84B209F1010909F03D
:10257000FF0900988145C3D300248648903001E0CC
:1025800007E01AE110F835107F4882781144817015
:102590000FE104260020814B14E033F830C0614580
:1025A0000ED303EBC00CBCF802C0614508D833F869
:1025B000305003EBC000491B8088084485B203E01B
:1025C000401C80B2B042E8D37F1C74489178203020
:1025D00030F83500C0F1A0038B4202DA4FF0A00AB8
:1025E00002E0084400F0FF0A92F80390B9F1370FB7
:1025F00002D9502000903EE009F11900C0B20090CD
:1026000039E06148867820E009EB890008EB801BFF
:102610003BF816201AB1100A00EB022082B25F4884
:102620005E49203000EBC500903140682144405C99
:102630005549C98814F0ACFC010201EB10202BF8BD
:102640001600641CA4B2761CF6B25645DCD3BAF16F
:10265000A00F0CD15148203030F83500B4FBF0F118
:1026600000FB1141C9B211B12044401A84B209F1F2
:10267000010909F0FF0900988145C2D300244748A9
:10268000203010F83510404882781144817090E075
:1026900033F830C061450ED303EBC00CBCF802C068
:1026A000614508D833F8305003EBC000491B8088DF
:1026B000084485B203E0401C80B2B042E8D37F1CDE
:1026C00033489178503030F83500C0F1A0038B4288
:1026D00002DA4FF0A00A02E0084400F0FF0A92F884
:1026E0000390B9F1450F02D9502000903DE009F167
:1026F0000B00C0B2009038E0234886781FE009EB59
:10270000890008EB801B3BF816201AB1100A00EB79
:10271000022082B21E482249503000EBC5002144FD
:102720004068405C1849C98814F032FC010201EB92
:1027300010202BF81600641CA4B2761CF6B2564585
:10274000DDD3BAF1A00F0CD11148503030F835006C
:10275000B4FBF0F100FB1141C9B211B12044401AA1
:1027600084B209F1010909F0FF0900988145C3D33A
:1027700000240748503010F8350013E04CD50120F4
:1027800034E402000CE902009C83FF1F04EE020007
:10279000545B030028BE0200E0C002002CA9020026
:1027A000EC5D030006498A781044C0B288709F2807
:1027B00003D8397800297FF4DEADBDE8F88F00003A
:1027C0009C83FF1F0EB509293BD2DFE801F0050B02
:1027D00011171D23292F350002461CA1684612F04F
:1027E000DDFD2EE002461AA1684612F0D7FD28E072
:1027F000024619A1684612F0D1FD22E0024618A156
:10280000684612F0CBFD1CE0024617A1684612F0A4
:10281000C5FD16E0024616A1684612F0BFFD10E0A5
:10282000024615A1684612F0B9FD0AE0024614A15D
:10283000684612F0B3FD04E0024613A1684612F0A8
:10284000ADFD684600F042F90EBD000025580000BD
:1028500025303158000000002530325800000000BB
:1028600025303358000000002530345800000000A7
:102870002530355800000000253036580000000093
:10288000253037580000000025303858000000007F
:102890002DE9FF4F07468846002403E138787E285B
:1028A0007ED99B2317F8011C01EB002080B2002287
:1028B0007F4913E031F8326086420DD801EBC20641
:1028C0007688864208D331F8323001EBC201C01A53
:1028D0008988084485B203E0521C92B29A42E9D337
:1028E000BF1E7448744A30F835109078C1F1A003C7
:1028F000834202DA4FF0A00A02E0084400F0FF0A27
:1029000092F80390B9F1400F02D94FF0500B3AE022
:1029100009F1100000F0FF0B35E0674A9678654832
:10292000664900EBC500039009EB890001EB8010BC
:10293000029013E00398416861482044085C5E49B6
:102940000A89C98814F024FB010201EB10200299C6
:1029500021F81600641CA4B2761CF6B25645E9D3E1
:10296000BAF1A00F0BD1534830F83500B4FBF0F1A9
:1029700000FB1141C9B211B12044401A84B209F1DF
:10298000010909F0FF09D945C7D3002449484A493C
:1029900010F835008A7810448870A8F1020800E029
:1029A00002E008F0FF087DE012230022454913E011
:1029B00031F83260B0420DD301EBC2067688B042E6
:1029C00008D831F8323001EBC201C01A89880844B6
:1029D00085B203E0521C92B29A42E9D37F1E394875
:1029E000354A903030F835009178C0F1A0038B4221
:1029F00002DA4FF0A00A02E0084400F0FF0A92F861
:102A00000390B9F1420F02D94FF0500B3BE009F1AE
:102A10000E0000F0FF0B36E0274A9678274909EBB5
:102A2000890001EB801001902648903000EBC50032
:102A3000009013E00098416823482044085C1E4938
:102A40000A89C98814F0A4FA010201EB1021019847
:102A500020F81610641CA4B2761CF6B25645E9D3D1
:102A6000BAF1A00F0BD1134830F83500B4FBF0F1E8
:102A700000FB1141C9B211B12044401A84B209F1DE
:102A8000010909F0FF09D945C6D300240D4890304B
:102A900010F835100848827811448170A8F10108B7
:102AA00008F0FF08B8F1000F7FF4F8AEBDE8FF8F23
:102AB00034E402000CE902009C83FF1F4CD5012086
:102AC00004EE020028BE0200E0C002002DE9F84F2B
:102AD00006460024FE4A9078D178A02872D8502962
:102AE00070D8DFF8F08392E2F94A507810280FD0BE
:102AF0001C2868D00C2867D0422863D19B237E29EC
:102B00007ED9707800EB012081B20020F24F04E200
:102B100012237E291FD9707800EB012081B200209A
:102B2000EE4F14E037F830C08C450ED807EBC00CE0
:102B3000BCF802C08C4508D337F8303007EBC00032
:102B4000C91A8088084485B203E0401C80B29842CC
:102B5000E8D3B61C1AE00020E04F14E037F830C08C
:102B600061450ED307EBC00CBCF802C0614508D824
:102B700037F8303007EBC000C91A8088084485B2A6
:102B800003E0401C80B29842E8D3761CD348917889
:102B9000903030F83500C0F1A0038B4202DA4FF0DC
:102BA000A00A02E0084400F0FF0A92F80390B9F18D
:102BB000420F02D95020009040E009F10E00C0B24F
:102BC00000903BE027E246E0E4E0C148877820E05F
:102BD00009EB890008EB801B3BF817201AB1100A9B
:102BE00000EB022082B2BD48BD49903000EBC50029
:102BF00021444068405CB649C98814F0C9F900E036
:102C00008FE1010201EB10202BF81700641C7F1CE0
:102C1000FFB25745DCD3BAF1A00F0BD1AF489030CB
:102C200030F8350094FBF0F100FB1141C9B209B155
:102C30002044441A09F1010909F0FF09009881456F
:102C4000C3D30024A548A249903010F835008A78F3
:102C500010448870DBE104237E291FD9707800EBD3
:102C6000012081B200209F4F14E037F830C08C451E
:102C70000ED807EBC00CBCF802C08C4508D337F85F
:102C8000303007EBC000C91A8088084485B203E0E1
:102C9000401C80B29842E8D3B61C1AE00020914F45
:102CA00014E037F830C061450ED307EBC00CBCF818
:102CB00002C0614508D837F8303007EBC000C91AA8
:102CC0008088084485B203E0401C80B29842E8D373
:102CD000761C84489178203030F83500C0F1A0038C
:102CE0008B4202DA4FF0A00A02E0084400F0FF0A2B
:102CF00092F80390B9F1370F02D9502000903CE0D0
:102D000009F11900C0B2009037E0714887781FE0E0
:102D100009EB890008EB801B3BF817201AB1100A59
:102D200000EB022082B26F486E49203000EBC500F4
:102D3000903140682144405C6549C98814F028F905
:102D4000010201EB10202BF81700641C7F1CFFB25E
:102D50005745DDD3BAF1A00F0BD16248203030F8CF
:102D6000350094FBF0F100FB1141C9B209B12044D8
:102D7000441A09F1010909F0FF0900988145C4D3FB
:102D8000002458485249203010F835008A78104401
:102D900088703CE10A237E291FD9707800EB01205E
:102DA00081B20020504F14E037F830C08C450ED867
:102DB00007EBC00CBCF802C08C4508D337F83030A4
:102DC00007EBC000C91A8088084485B203E0401CA4
:102DD00080B29842E8D3B61C1AE00020424F14E0BB
:102DE00037F830C061450ED307EBC00CBCF802C009
:102DF000614508D837F8303007EBC000C91A808821
:102E0000084485B203E0401C80B29842E8D3761CA7
:102E100035489178503030F83500C0F1A0038B422E
:102E200002DA4FF0A00A02E0084400F0FF0A92F82C
:102E30000390B9F1450F02D9502000903BE009F111
:102E40000B00C0B2009036E0214887781EE009EB05
:102E5000890008EB801B3BF817201AB1100A00EB21
:102E6000022082B220482149503000EBC5002144A5
:102E70004068405C1649C98814F08AF8010201EBE9
:102E800010202BF81700641C7F1CFFB25745DED3BF
:102E9000BAF1A00F0BD11448503030F8350094FB34
:102EA000F0F100FB1141C9B209B12044441A09F103
:102EB000010909F0FF0900988145C5D300240A489B
:102EC000503010F8351002488278114481709EE02D
:102ED0009C83FF1F4CD5012034E4020028BE020071
:102EE000E0C002002CA90200545B0300EC5D03006B
:102EF00037F830C08C450ED807EBC00CBCF802C0C8
:102F00008C4508D337F8303007EBC000C91A8088E9
:102F1000084485B203E0401C80B29842E8D3B61C56
:102F20001AE000203D4F14E037F830C061450ED361
:102F300007EBC00CBCF802C0614508D837F8303048
:102F400007EBC000C91A8088084485B203E0401C22
:102F500080B29842E8D3761C3148917830F8350039
:102F6000C0F1A0038B4202DA4FF0A00A02E008444D
:102F700000F0FF0A92F80390B9F1400F02D95020F7
:102F8000009039E009F11000C0B2009034E025480B
:102F900087781DE009EB890008EB801B3BF81720C0
:102FA0001AB1100A00EB022082B21D481E4900EB44
:102FB000C50021444068405C1A49C98813F0E8FF05
:102FC000010201EB10202BF81700641C7F1CFFB2DC
:102FD0005745DFD3BAF1A00F0AD1114830F83500B8
:102FE00094FBF0F100FB1141C9B209B12044441A2D
:102FF00009F1010909F0FF0900988145C7D30024B0
:10300000074810F8351007488278114481703178EC
:1030100000297FF469ADBDE8F88F000034E40200B8
:103020000CE902009C83FF1F04EE02000EB5062887
:1030300051D2DFE800F003101D2A374410EE100AC9
:10304000FDF77AFB41EC100B25A153EC102B6846E1
:1030500012F0A4F93FE010EE100AFDF76DFB41EC11
:10306000100B21A153EC102B684612F097F932E0B7
:1030700010EE100AFDF760FB41EC100B1CA153ECA5
:10308000102B684612F08AF925E010EE100AFDF7C1
:1030900053FB41EC100B18A153EC102B684612F0B7
:1030A0007DF918E010EE100AFDF746FB41EC100B1D
:1030B00013A153EC102B684612F070F90BE010EEE0
:1030C000100AFDF739FB41EC100B0FA153EC102B4C
:1030D000684612F063F96846FFF7F8FC0EBD000081
:1030E000252E306600000000252E3166000000000D
:1030F000252E326600000000252E336600000000F9
:10310000252E346600000000252E356600000000E4
:103110000EB5062927D2DFE801F003090F151B21A0
:10312000024613A1684612F039F91CE0024611A1CB
:10313000684612F033F916E0024610A1684612F014
:103140002DF910E002460FA1684612F027F90AE0B7
:1031500002460EA1684612F021F904E002460DA1D4
:10316000684612F01BF96846FFF7B0FC0EBD000080
:1031700025640000253031640000000025303264F1
:103180000000000025303364000000002530346466
:10319000000000002530356400000000014A9070F6
:1031A000D17070479C83FF1F014948707047000031
:1031B0009C83FF1F0149C880704700009C83FF1F4C
:1031C0002DE9FF4F89B0064688461746002453E292
:1031D0001798102812D017981C2874D017980C280C
:1031E00072D01798422870D19B227E2B6ED97878A6
:1031F00000EB032081B20020F84BC6E112227E2BA7
:103200001FD9787800EB032081B20020F44B14E042
:1032100033F830C08C450ED803EBC00CBCF802C0AC
:103220008C4508D333F8302003EBC000891A80881E
:10323000084485B203E0401C80B29042E8D3BF1C32
:103240001AE00020E64914E031F830C063450ED39F
:1032500001EBC00CBCF802C0634508D831F830203F
:1032600001EBC0009A1A8088104485B203E0401C2C
:1032700080B29042E8D37F1CD948903030F83500B6
:10328000C0F1A001B14202DA4FF0A00B02E03044DD
:1032900000F0FF0BB8F1420F02D95020009003E07C
:1032A00008F10E00C0B20090C2462AE0B146CC48F8
:1032B000CC49903000EBC50008900AEB8A0001EB86
:1032C0008010079017E027E0B1E0D9E161E10898AC
:1032D0000C9A4168C4482044085C169913F058FEC3
:1032E000010201EB1020079921F81900641C09F173
:1032F000010909F0FF09D945E9D30AF1010A0AF0E9
:10330000FF0A00988245D1D30024B548903010F8C8
:1033100035003044C6B2AFE104227E2B1FD9787845
:1033200000EB032081B20020B04B14E033F830C032
:103330008C450ED803EBC00CBCF802C08C4508D3FA
:1033400033F8302003EBC000891A8088084485B226
:1033500003E0401C80B29042E8D3BF1C1AE000207A
:10336000A24914E031F830C063450ED301EBC00C24
:10337000BCF802C0634508D831F8302001EBC0002A
:103380009A1A8088104485B203E0401C80B29042B3
:10339000E8D37F1C9548203030F83500C0F1A001FB
:1033A000B14202DA4FF0A00B02E0304400F0FF0B14
:1033B000B8F1370F02D95020009003E008F119004E
:1033C000C0B20090C24627E0B14688488549203007
:1033D00000EBC50006900AEB8A0001EB8010059017
:1033E00014E006980C9A4168804890302044085CAC
:1033F000169913F0CDFD010201EB1020059921F87B
:103400001900641C09F1010909F0FF09D945E8D345
:103410000AF1010A0AF0FF0A00988245D4D3002479
:103420007248203010F835003044C6B224E10A2238
:103430007E2B1FD9787800EB032081B200206C4BE3
:1034400014E033F830C08C450ED803EBC00CBCF848
:1034500002C08C4508D333F8302003EBC000891A32
:103460008088084485B203E0401C80B29042E8D3D3
:10347000BF1C1AE000205E4914E031F830C06345FB
:103480000ED301EBC00CBCF802C0634508D831F87C
:10349000302001EBC0009A1A8088104485B203E006
:1034A000401C80B29042E8D37F1C5148503030F825
:1034B0003500C0F1A001B14202DA4FF0A00B02E0EA
:1034C000304400F0FF0BB8F1450F02D950200090B6
:1034D00003E008F10B00C0B20090C24635E0B146EF
:1034E00043484049503000EBC50004900AEB8A0085
:1034F00001EB8010039013E004980C9A41683D485A
:103500002044085C169913F043FD010201EB1020E2
:10351000039921F81900641C09F1010909F0FF0958
:10352000D945E9D3BBF1A00F0BD13148503030F869
:10353000350094FBF0F100FB1141C9B209B1204400
:10354000441A0AF1010A0AF0FF0A00988245C6D31C
:1035500000242748503010F835003044C6B28BE0C4
:1035600033F830C08C450ED803EBC00CBCF802C059
:103570008C4508D333F8302003EBC000891A8088CB
:10358000084485B203E0401C80B29042E8D3BF1CDF
:103590001AE00020114914E031F830C063450ED321
:1035A00001EBC00CBCF802C0634508D831F83020EC
:1035B00001EBC0009A1A8088104485B203E0401CD9
:1035C00080B29042E8D37F1C0B4830F83500C0F140
:1035D000A001B14212DA4FF0A00B12E034E4020075
:1035E00028BE02004CD50120E0C002002CA9020038
:1035F000545B0300EC5D03000CE90200304400F072
:10360000FF0BB8F1400F02D95020009003E008F101
:103610001000C0B20090C24625E0B1461A490AEB3C
:103620008A0001EB80100290184800EBC500019061
:1036300013E001980C9A416815482044085C1699DB
:1036400013F0A6FC010201EB1020029921F81900E9
:10365000641C09F1010909F0FF09D945E9D30AF110
:10366000010A0AF0FF0A00988245D6D300240748D1
:1036700010F835003044C6B23B78002B7FF4A8AD7B
:103680000DB0BDE8F08F00004CD501200CE9020020
:1036900004EE02002DE9F04186B00646DDE90C4556
:1036A0000F469846062A51D2DFE802F003101D2A81
:1036B000374410EE100AFDF73FF841EC100B29A13A
:1036C00053EC102B03A811F069FE3FE010EE100A36
:1036D000FDF732F841EC100B24A153EC102B03A89A
:1036E00011F05CFE32E010EE100AFDF725F841EC17
:1036F000100B20A153EC102B03A811F04FFE25E076
:1037000010EE100AFDF718F841EC100B1BA153EC5A
:10371000102B03A811F042FE18E010EE100AFDF77E
:103720000BF841EC100B17A153EC102B03A811F070
:1037300035FE0BE010EE100AFCF7FEFF41EC100B1B
:1037400012A153EC102B03A811F028FE434603AA44
:1037500039463046CDE90045FFF732FD06B0BDE8F9
:10376000F0810000252E306600000000252E316615
:1037700000000000252E326600000000252E336672
:1037800000000000252E346600000000252E35665E
:10379000000000002DE9F04186B00646DDE90C8509
:1037A0000E9C0F46062B21D2DFE803F003080D1212
:1037B000171C14A103A811F0F1FD17E012A103A832
:1037C00011F0ECFD12E012A103A811F0E7FD0DE0ED
:1037D00011A103A811F0E2FD08E011A103A811F066
:1037E000DDFD03E010A103A811F0D8FDCDE90054E0
:1037F000434603AA39463046FFF7E2FC06B0BDE86F
:10380000F0810000256400002530316400000000D4
:1038100025303264000000002530336400000000D1
:1038200025303464000000002530356400000000BD
:1038300010B5AFF3008010BD10B50446002C0CD0BD
:10384000012C0AD0022C08D0032C06D0042C04D062
:103850004FF4C86111A001F0E1FE1B4854B1012CE6
:103860000DD0022C10D0032C13D090F84100C0F3DF
:10387000000010BD90F83C00C0F3000010BD90F8AF
:103880003C00C0F3C00010BD90F83C00C0F34010F5
:1038900010BD90F83C00C0F3801010BD2E2E5C2EA1
:1038A0002E5C2E2E5C2E2E5C2E2E5C64726976654C
:1038B000725C7372635C68633332663436305F63A4
:1038C0006C6B2E630000000000400540F8B5054613
:1038D000002000900024284EB6F8FE034AF2015161
:1038E0000843A6F8FE03002D06D0012D04D040F2B7
:1038F000252122A001F092FE4DB196F8360020F06D
:10390000010086F8360009244FF4805525E096F82A
:10391000260040070ED0D6F8000100060ED596F816
:103920002A00C00708D096F8360040F0010086F85B
:10393000360015E0012413E0012411E096F836006A
:1039400040F0010086F836000AE00020FFF774FF1F
:1039500001280FD00098401C00900098A842F4D392
:10396000B6F8FE0320F0010040F42540A6F8FE035F
:103970002046F8BD0024F3E7004005402E2E5C2EC3
:103980002E5C2E2E5C2E2E5C2E2E5C64726976656B
:10399000725C7372635C68633332663436305F63C3
:1039A0006C6B2E6300000000F8B505460020009007
:1039B0000024002D06D0012D04D040F236311EA087
:1039C00001F02CFE274EB6F8FE034AF201510843DF
:1039D000A6F8FE034DB196F82A0020F0010086F803
:1039E0002A0009244FF4805516E096F8260000F0CE
:1039F0000700052806D096F82A0040F0010086F856
:103A00002A000CE001240AE00220FFF715FF01283C
:103A10000FD00098401C00900098A842F4D3B6F84C
:103A2000FE0320F0010040F42540A6F8FE032046E6
:103A3000F8BD0024F3E700002E2E5C2E2E5C2E2E07
:103A40005C2E2E5C2E2E5C6472697665725C7372DD
:103A5000635C68633332663436305F636C6B2E634D
:103A6000000000000040054010B50446002C5BD06B
:103A70002068801E0E2804D940F205312BA001F0E9
:103A8000CDFD6068401E0F2804D940F2063127A002
:103A900001F0C4FDA068801E0E2804D940F2073151
:103AA00022A001F0BBFDE0681438B0F5E67F04D930
:103AB0004FF442711DA001F0B1FD2069401E17288E
:103AC00004D940F2093119A001F0A8FD2248B0F84C
:103AD000FE124AF201521143A0F8FE122178026848
:103AE000491E61F31F72026021790268491E61F369
:103AF0001B620260217A0268491E61F3175202605C
:103B0000A1890268491E61F310220260217C0268CB
:103B1000491E61F304020260B0F8FE1221F00101B7
:103B200041F42541A0F8FE1210BD00002E2E5C2E9F
:103B30002E5C2E2E5C2E2E5C2E2E5C6472697665B9
:103B4000725C7372635C68633332663436305F6311
:103B50006C6B2E63000000000041054010B5044668
:103B6000002C08D0A4F10800052804D940F24351E4
:103B70000BA001F053FD1549B1F8FE034AF20252C1
:103B80001043A1F8FE03088A64F303000882B1F829
:103B9000FE0320F0020040F42540A1F8FE0310BD12
:103BA0002E2E5C2E2E5C2E2E5C2E2E5C2E2E5C6419
:103BB00072697665725C7372635C68633332663413
:103BC00036305F636C6B2E630000000000400540E0
:103BD00010B50446002C06D0012C04D040F2E5219B
:103BE0000BA001F01BFD1549B1F8FE024AF201528B
:103BF0001043A1F8FE02086864F3C7100860B1F82A
:103C0000FE0220F0010040F42540A1F8FE0210BDA4
:103C10002E2E5C2E2E5C2E2E5C2E2E5C2E2E5C64A8
:103C200072697665725C7372635C686333326634A2
:103C300036305F636C6B2E6300000000004105406E
:103C400070B586B00446002605962E4D286804906F
:103C500068680390A8680290E8680190002C07D07B
:103C6000601E042804D940F2DD3127A001F0D6FC03
:103C700030482861304991F826004A1500F00700C5
:103C8000052801D0052C0BD12C482860C012686093
:103C9000A860E8600598401C059005989042F9D30B
:103CA0002631B1F8D8034AF201531843A1F8D803DA
:103CB000087864F302000870B1F8D80320F001001E
:103CC00040F42540A1F8D80305960598401C0590BE
:103CD00005989042F9D30498286003986860029888
:103CE000A8600198E8601348401E28610596059871
:103CF000401C059005989042F9D306B0BDE870408D
:103D00000FF060BD008004402E2E5C2E2E5C2E2E07
:103D10005C2E2E5C2E2E5C6472697665725C73720A
:103D2000635C68633332663436305F636C6B2E637A
:103D3000000000000100A5A500400540EEFAFFFFCD
:103D400010B50446A01E022807D9801F052804D9F3
:103D500040F227510BA001F061FC1549B1F8DA03DC
:103D60004AF201521043A1F8DA03087864F307100D
:103D70000870B1F8DA0320F0010040F42540A1F802
:103D8000DA0310BD2E2E5C2E2E5C2E2E5C2E2E5CA9
:103D90002E2E5C6472697665725C7372635C686314
:103DA0003332663436305F636C6B2E630000000084
:103DB00024400540F0B585B0044600260496434DE6
:103DC0002868039068680290A8680190E8680090ED
:103DD0003F482861002C76D02178E27891421BD8A8
:103DE0006379994218D8A079814215D8A178914277
:103DF00012D8994210D821790A1A032A11D0022A1E
:103E00000FD0012A0DD081420BD0401A012808D0D2
:103E1000022806D0032804D040F23C412DA001F036
:103E2000FDFB374991F826004A1500F007000528E8
:103E30000BD134482860C0126860A860E86004981C
:103E4000401C049004989042F9D3B1F8FE034AF262
:103E500001531843A1F8FE03A078E378677940EA9C
:103E6000031023791B0243EA07331843A37940EA7E
:103E70000340637840EA0353207843EA006343EA4F
:103E800000700862B1F8FE0320F0010040F4254004
:103E9000A1F8FE0304960498401C049004989042F4
:103EA000F9D303982860029868600198A860009888
:103EB000E8600748401E286104960498401C04905E
:103EC00004989042F9D305B0F0BD00000080044092
:103ED0000100A5A52E2E5C2E2E5C2E2E5C2E2E5CB7
:103EE0002E2E5C6472697665725C7372635C6863C3
:103EF0003332663436305F636C6B2E630000000033
:103F000000400540EEFAFFFF38B50446002C06D00D
:103F1000012C04D040F29F3122A001F07FFB2C49FC
:103F2000B1F8FE034AF201521043A1F8FE03012C3E
:103F300004D091F82E0040F0010003E091F82E002B
:103F400020F0010081F82E00B1F8FE0320F00100FE
:103F500040F42540A1F8FE0300204FF480550CB139
:103F6000009017E0009007E00098401C0090009837
:103F7000A84201D9092038BD0320FFF75DFC0028C5
:103F8000F2D10CE00098401C00900098A84201D9A2
:103F9000092038BD0320FFF74FFC0128F2D1002093
:103FA00038BD00002E2E5C2E2E5C2E2E5C2E2E5C3C
:103FB0002E2E5C6472697665725C7372635C6863F2
:103FC0003332663436305F636C6B2E630000000062
:103FD0000040054070B50446002C7CD02068801E4F
:103FE0000E2804D940F26F313EA001F017FB606843
:103FF000801E0E2804D94FF45C713AA001F00EFB2C
:10400000A068801E0E2804D940F2713135A001F05D
:1040100005FBE0681438B0F5E67F04D940F2723150
:1040200030A001F0FBFA2069801E162804D940F266
:1040300073312CA001F0F2FA354DD5F800010006DD
:1040400001D4344801E0344800682169B0FBF1F044
:10405000E6684643314908443149884204D940F270
:104060007A3120A001F0DAFA2E482E493044494234
:10407000884204D940F27B311AA001F0CFFA05F54D
:104080008275B5F8FA024AF201510843A5F8FA021E
:1040900020782968401E60F31F7129602079296803
:1040A000401E60F31B612960207A2968401E60F37E
:1040B00017512960A0892968401E60F310212960EA
:1040C000207C2968401E60F304012960B5F8FA02DB
:1040D00020F0010000E003E040F42540A5F8FA02DA
:1040E00070BD00002E2E5C2E2E5C2E2E5C2E2E5CC3
:1040F0002E2E5C6472697665725C7372635C6863B1
:104100003332663436305F636C6B2E630000000020
:104110000040054000127A00B082FF1FC0BDF0FFD2
:10412000C0F35E0100E4B1F10421012803D00228AC
:1041300001D0102805D104494FF4AA420A80088012
:1041400000210846704700000CA10440F8B526483D
:104150000090002003F0DCFE00F0070120FA01F2DD
:10416000884010442149884203D921490844440821
:1041700003E01F494942084444001E4F01261E4DDA
:104180003868A04202D1EE760120F8BD287F48B100
:104190006E772E2003F02AFE3860A04202D1EE7620
:1041A0000120F8BD1549009808441449009A0939BE
:1041B000114411E0027872B10278082302E052083B
:1041C0005B1EDBB2D407FAD00099401AC01C03EB87
:1041D000C000A87602E0401E8842EBD2A87E08B15B
:1041E0000120F8BD0020F8BD53AE004333DDD353AA
:1041F00034DDD3D35491FF1FB083FF1FC65DFFBFD3
:1042000070B5002500F0D2F81020FEF7CDFF4D4824
:104210000088FEF7CFFF00210846FEF7BFFF4AA047
:10422000FEF754FC00210420FDF74CFE49A0FEF7E8
:104230004DFC494C2088FEF7BDFF10210020FEF701
:10424000ADFF46A0FEF742FC46A0FEF73FFC002073
:1042500003F05EFE0821FEF7B5FA20210020FEF7EC
:104260009DFF41A0FEF780F840210020FEF796FF59
:104270002088FEF79FFF404CA07E38B13FA0FEF79C
:1042800073F80021A07EFEF743FF05E03EA0FEF795
:104290006BF83FA0FEF71AFC40480088FEF78AFF43
:1042A000A07F3F4C082835D2DFE800F034040B1221
:1042B0001920272E20680121000F03F049FE054632
:1042C00028E020680221000E03F042FE054621E0AE
:1042D00020680321000D03F03BFE05461AE020682C
:1042E0000421000C03F034FE054613E0206805218C
:1042F000000B03F02DFE05460CE020680621000AA5
:1043000003F026FE054605E020680721000903F0BA
:104310001FFE054623A003F081FE2844C0B23221CF
:10432000FEF73CFF20A0FEF7D1FB30210020FEF776
:1043300035FF1CA0FEF7CAFB2068BDE870400821CD
:10434000FEF740BAAC83FF1F69444B4D657465723C
:104350000000000030324300AA83FF1F532F4E3A63
:104360000000000030780000C7EBCAE4C8EBD7A219
:10437000B2E1C2EB3A000000B083FF1F52656D61ED
:10438000696E5573653A00005151C8BA3A00000091
:10439000373838303133313230000000A883FF1F06
:1043A0005491FF1F3E3078005F000000F8B571485F
:1043B0000090714F3A78714C714D00262068A97FAA
:1043C000042A14D03A780A2A11D03A78052A53D010
:1043D0003A780B2A50D03878062870D03A78284698
:1043E000092A807E6CD039780C296AD0B6E0634AFD
:1043F0001268D24308290AD2DFE801F0040A121A2F
:10440000222A3239110F02D000F180502060A5E03D
:104410006FEA1061090702D000F1807020609DE012
:104420006FEA1051090702D000F58010206095E076
:104430006FEA1041090702D000F5803020608DE05E
:104440006FEA1031090702D000F58050206085E046
:104450006FEA1021090702D000F5807020607DE02E
:104460006FEA1011090779D01030206076E011074B
:1044700074D0401C206071E008296FD2DFE801F0A1
:10448000040A111822293036010F67D0A0F180509C
:10449000206063E0010E090760D0A0F18070206009
:1044A0005CE0010D090759D0A0F58010206055E0AF
:1044B000010C090752D0A0F5803020604EE01AE0D0
:1044C00041E049E0010B090748D0A0F58050206089
:1044D00044E0010A090741D0A0F5807020603DE06A
:1044E000010909073AD01038206037E0010735D0BC
:1044F000401E206032E0287808B9491CA977A87FBF
:1045000008282BD1AE77FFF721FEE87E78B16E70D8
:104510002E766E762E20216803F0C2FC03F06CFC30
:10452000184A00982168104403F0C0FC16E01648B1
:1045300001682A6B891AB1F5487F0FD902212970C9
:10454000006828630AE011B1491EA97702E008B1AA
:10455000112068703E7001E000B16E703878062856
:1045600005D03878052802D03878042800D13E706C
:10457000F8BD000053AE00436083FF1F5491FF1F3E
:10458000B083FF1FB55DFFBF7C83FF1F2DE9FC419A
:1045900000F086F81020FEF707FE3B4EF08DFEF788
:1045A00009FE00210846FEF7F9FD38A0FDF7DCFE04
:1045B000B08DFEF7FFFD10210020FEF7EFFD002477
:1045C00006F27457B08DFEF7F5FD601C0546000736
:1045D000010E0020FEF7E2FDF07D844211D10221A0
:1045E0000020FDF76FFC0C20FEF7DEFD708DFEF75E
:1045F000E1FD2AA0FEF76AFA6FF001010020FDF745
:1046000061FC1020FEF7D0FD04EB041057F82000E9
:10461000FDF7AAFEECB2042CD4D3FF24708DCDE9B3
:1046200000042023842210216420FDF763FDB08D57
:10463000CDE900043523842225216420FDF75AFDAD
:10464000F08DCDE900044A2384223A216420FDF74D
:1046500051FDB08DCDE900049E224F23002110466C
:10466000FDF748FDB08DCDE90004F07D9F2200EB01
:10467000800101EBC000012101EB400300219D20DE
:10468000FDF738FDBDE8FC81B083FF1FD6F7CCE213
:10469000D1D5C9ABC9E8D6C3000000003E00000078
:1046A00070B53D4E31783D4C00250429E07D03D0A6
:1046B0003178052908D00EE0032802D2401CE075AD
:1046C00000E0E575357006E010B1401EE07501E0D0
:1046D0000320E0753570E07D50B14FF6DC514FF6A8
:1046E000F37201280ED0022812D003281FD117E040
:1046F0004FF64D30608540F27960A0854DF69A30D6
:10470000E08514E06185A2854AF67D70E0850EE0C3
:104710004FF638706085A1854EF27350E08506E053
:10472000628546F2F370A0854AF6DC60E085307859
:10473000062807D03078092803D1657511206070EC
:10474000357070BD2078D0B9618D282003F094FBBE
:10475000A18D2A2003F090FBE18D2C2003F08CFB2F
:104760000F49E07D81F8320003F046FB0D49608D72
:1047700008800D48A18D01800C49E08D08800C480F
:104780000168226B891AB1F5487F03D90121217094
:1047900000682063357070BD6083FF1FB083FF1F0A
:1047A00074610220A883FF1FAA83FF1FAC83FF1F31
:1047B0007C83FF1F70B500F0ABF81020FEF7F4FC0F
:1047C0003D480088FEF7F6FC00210846FEF7E6FCAF
:1047D0003AA0FDF7C9FD3C4D2888FEF7EBFC1021FF
:1047E0000020FEF7DBFC39A0FDF7BEFD3A4C0520AA
:1047F00094ED150AFEF71AFC20210020FEF7CEFCEE
:1048000036A0FDF7B1FD3849052091ED000AFEF70D
:104810000DFCA07D354C6FF0020628B301284AD16B
:1048200030210020FEF7BAFC31A0FDF79DFD208865
:10483000FEF7C0FC0C20FEF7B7FC40210020FEF77D
:10484000ADFC03210020FDF73DFB2CA0FEF73EF957
:1048500031460020FDF736FB1020FEF7A5FCBDE831
:10486000704027A0FDF780BD2088FEF7A3FC302113
:104870000020FEF793FC0C20FEF796FC032100209D
:10488000FDF720FB1DA0FEF721F931460020FDF7C2
:1048900019FB1020FEF788FC15A0FDF765FD2888A0
:1048A000FEF788FC40210020FEF778FCBDE8704050
:1048B00013A0FDF759BD70BDAC83FF1FB5E7C1F76D
:1048C000D0A3D7BC00000000AA83FF1FD0C2D0A392
:1048D000D7BCB2CECAFD3A00B083FF1FBEC9D0A379
:1048E000D7BCB2CECAFD3A004C83FF1FA883FF1F7E
:1048F000B1A3B4E6D0C2B2CECAFD00003E000000B3
:10490000BBD6B8B4C4ACC8CFB2CECAFD000000005C
:104910002DE9F041204E3178204C00250127A07D63
:1049200004290ED0317805290FD03178062911D00D
:104930003078092803D16575192060703570BDE89D
:10494000F08100B9A7753570F9E708B1401EA07570
:104950003570F4E7217841B998B1192003F036FA9F
:104960001D2003F093FA03F047FA0D480168226B0B
:10497000891AB1F5487F02D9277000682063357025
:10498000DDE7084894ED150A80ED000A90ED000A75
:104990001D2003F07BFAE6E76083FF1FB083FF1F53
:1049A0007C83FF1F4C83FF1F7CB500F0DBF81020D9
:1049B000FEF7FAFB4F480088FEF7FCFB0021084693
:1049C000FEF7ECFB4CA0FDF7CFFC4E4D2888FEF720
:1049D000F1FB4D48007830B14FF4007100200BF02E
:1049E0008BFC002833D018210020FEF7D7FB288845
:1049F000FEF7E0FB45A0FDF7B7FC28210020FEF7FD
:104A0000CDFB47A0FDF7B0FC484E042096ED140AFC
:104A1000FEF70CFB46A0FEF759F838210020FEF700
:104A2000BDFB44A0FDF7A0FC4549042091ED000A20
:104A3000FEF7FCFA3EA0FEF749F8717D4148FF24DD
:104A400005293ED2DFE801F00C16202A3400282187
:104A50000020FEF7A3FBBDE87C403BA0FDF784BC33
:104A60000088CDE900043723392236213120FDF7B3
:104A700041FB26E00088CDE9000437234722362198
:104A80003F20FDF737FB1CE00088CDE90004372309
:104A9000502236214820FDF72DFB12E00088CDE999
:104AA00000043723592236215120FDF723FB08E06B
:104AB0000088CDE900043723622236215A20FDF711
:104AC00019FB2888CDE900049E224F2300211046BF
:104AD000FDF710FB2888CDE90004707D9F2200EBD4
:104AE000400101EB0013DB1C00219D20FDF702FBC0
:104AF0007CBD0000AC83FF1FB5E7C1F7D0A3D7BCD6
:104B000000000000AA83FF1F3083FF1FC7EBC9E826
:104B1000D6C3B1EAD7BCB5E7C1F7D6B53A000000B5
:104B2000B1EAD7BCB5E7C1F73A000000B083FF1F78
:104B300041000000B5B1C7B0B5E7C1F73A000000C9
:104B40003883FF1FA883FF1FC7EBCAB9D3C3B9AB14
:104B5000CDB7CAE4C8EBBBF2CDE2BDD3484944D0DF
:104B6000A3D7BC0070B52DED028B5C4D2978B7EE54
:104B7000008A9FED5B2ADFED5B0ADFED5B1A9FED9C
:104B80005B1A5B4C0026042994ED140A607D0CD05E
:104B900029780A2909D0297805292ED029780B29C6
:104BA0002BD02878062850D059E005281CD2DFE801
:104BB00000F003080D12170030EE080A84ED140A05
:104BC00012E030EE020A84ED140A0DE030EE200A05
:104BD00084ED140A08E030EE210A84ED140A03E0A3
:104BE00030EE010A84ED140A4249206D884268DDE6
:104BF000B1EE040A84ED140A63E005281CD2DFE854
:104C000000F003080D12170030EE480A84ED140A74
:104C100012E030EE420A84ED140A0DE030EE600A34
:104C200084ED140A08E030EE610A84ED140A03E012
:104C300030EE410A84ED140A206DB0F17C5F40DA59
:104C4000B6EE000A84ED140A3BE02B48007850B120
:104C50004FF4007100200BF04FFB012803D028789F
:104C6000092826D02DE0607D401CC0B26075052863
:104C700027D166752148224A90ED000A10EE101ADD
:104C8000914211DDD4ED140A90ED001A80EE810AF4
:104C900084ED150A10EE100A514208441949884261
:104CA00004D384ED158A01E084ED158A1A20607022
:104CB00007E0607D10B1401E607501E0112060705A
:104CC0002E702878062805D02878052802D0287864
:104CD000042800D12E70BDEC028B70BD6083FF1FD5
:104CE000CDCCCC3D0AD7233C6F12833A17B7D138CD
:104CF000B083FF1F0000A0403083FF1F3883FF1FD9
:104D00009A99993E6766A60170B506460D46144607
:104D10005F48864207D05F48864204D040F2D17196
:104D20005DA000F07BFC55B1012D08D0022D06D00E
:104D3000032D04D040F2D27157A000F06FFC207810
:104D400040B1012806D0022804D040F2D37152A00D
:104D500000F064FC607840B1012806D0022804D03D
:104D600040F2D4714CA000F059FCA07830B1012879
:104D700004D040F2D57148A000F050FCE07830B18A
:104D8000012804D040F2D67143A000F047FC2079FE
:104D900030B1012804D040F2D7713FA000F03EFCB2
:104DA000607930B1012804D04FF4FB613AA000F0E3
:104DB00035FCA07940B1012806D0022804D040F289
:104DC000D97135A000F02AFCE07930B1012804D077
:104DD00040F2DA7130A000F021FC207A30B10128D5
:104DE00004D040F2DB712CA000F018FC607A30B1E6
:104DF000012804D040F2DC7127A000F00FFC06EB84
:104E00008510C16D227821F003011143C165C16D88
:104E1000627821F00C0141EA8201C165C16DA2787E
:104E200021F0100141EA0211C165C16DE27821F063
:104E3000200141EA4211C165C16D227921F0400192
:104E400041EA8211C165C16D627921F0800141EAB8
:104E5000C211C165C16DA27921F4407141EA0221FC
:104E6000C165C16DE27921F4806141EA8221C165A9
:104E7000C16D227A21F4006141EAC221C165C16D90
:104E8000627A21F4805141EA0231C16570BD0000AF
:104E900000300540003405402E2E5C2E2E5C2E2E58
:104EA0005C2E2E5C2E2E5C6472697665725C737269
:104EB000635C68633332663436305F646D61632EE1
:104EC000630000002DE9F04704460D461746002612
:104ED0005B48844207D05B48844204D040F287217B
:104EE00059A000F09BFB55B1012D08D0022D06D032
:104EF000032D04D04FF4227153A000F08FFB37B183
:104F0000012F04D040F289214FA000F087FB5949BE
:104F1000087810B10120BDE8F08701230B70E0692B
:104F2000AB409843002290B3E0694FF00A0CC007F1
:104F30004FF4A04817D0B5B1A06C000CD4F868901D
:104F4000BCEB194F0FD3D4F86890B0EB194F07D8CA
:104F500009E0761CB6B2464502D90A700920DAE7A4
:104F6000E069C007F5D1E06980071BD5012D19D094
:104F7000D4F88800000CD4F8A860BCEB164F11D30D
:104F8000D4F8A860B0EB164F0CD9002007E03AE047
:104F9000401C80B2404502D90A700920BBE7E6698F
:104FA000B607F5D4E06940071AD5022D18D00020C5
:104FB000D4F8C860360CD4F8E890BCEB194F0FD386
:104FC000D4F8E890B6EB194F07D809E0401C80B23E
:104FD000404502D90A7009209DE7E6697607F5D4B5
:104FE000E06900071AD5032D18D00020D4F8085125
:104FF0002D0CD4F82861BCEB164F0FD3D4F82861E0
:10500000B5EB164F07D809E0401C80B2404502D9E5
:105010000A7009207FE7E5692D07F5D43FB1012F1C
:105020000AD1E06903F00F031843E06104E0E0698E
:105030000F259D432840E0610A7000206BE70000C7
:1050400000300540003405402E2E5C2E2E5C2E2EA6
:105050005C2E2E5C2E2E5C6472697665725C7372B7
:10506000635C68633332663436305F646D61632E2F
:10507000630000006C91FF1F2DE9F04105460C46CE
:10508000164600272548854207D02548854204D08A
:1050900040F24E2123A000F0C1FA54B1012C08D0F7
:1050A000022C06D0032C04D040F24F211DA000F0AA
:1050B000B5FA56B1012E08D0022E06D0032E04D028
:1050C0004FF4147117A000F0A9FA3CB1012C05D0DF
:1050D000022C03D0032C01D004270CE00120A040B7
:1050E00066B110340121A140012E0BD0022E0DD04B
:1050F000032E0FD004273846BDE8F08169690143CB
:105100006961F8E7686908436861F4E7A9690143E0
:10511000A961F0E7A8690843A861ECE70030054001
:10512000003405402E2E5C2E2E5C2E2E5C2E2E5C26
:105130002E2E5C6472697665725C7372635C686360
:105140003332663436305F646D61632E6300000075
:1051500070B504460D460C48844207D00B48844283
:1051600004D04FF4C1710AA000F058FA35B1012DF6
:1051700004D040F2831106A000F050FA206865F3D5
:105180000000206070BD0000003005400034054084
:105190002E2E5C2E2E5C2E2E5C2E2E5C2E2E5C6413
:1051A00072697665725C7372635C6863333266340D
:1051B00036305F646D61632E6300000070B5064693
:1051C0000D4614463A48864207D03A48864204D0F3
:1051D00040F6120138A000F021FA55B1012D08D097
:1051E000022D06D0032D04D040F6130132A000F0AA
:1051F00015FA2088800A04D040F614012EA000F091
:105200000DFAA089800A04D040F616012AA000F009
:1052100005FAE089800A04D040F6170126A000F0C4
:10522000FDF901213046FFF793FF06EB8513D86D9A
:1052300020F48050D86560681864A0685864986C41
:1052400021886FF30900084398646188986C61F3C2
:105250001F409864D86CA1896FF309000843D86493
:10526000D86C20490840E18940EA0140D864186DB3
:1052700061696FF3130008431865218B186D61F3A2
:105280001F501865586DE1696FF3130008435865A6
:10529000218C586D61F31F5058652069986504F1A1
:1052A000240229463046BDE87040FFF72DBD0000BE
:1052B00000300540003405402E2E5C2E2E5C2E2E34
:1052C0005C2E2E5C2E2E5C6472697665725C737245
:1052D000635C68633332663436305F646D61632EBD
:1052E00063000000FFFF00FC2DE9F04180460D4601
:1052F0001646002400271548804507D014488045ED
:1053000004D040F2354113A000F088F955B1012DC9
:1053100008D0022D06D0032D04D040F236410DA056
:1053200000F07CF908EB85114E644FF4805006E0E4
:10533000641CA4B2844201D9092700E04E644A6E7D
:10534000B242F5D13846BDE8F0810000003005409A
:10535000003405402E2E5C2E2E5C2E2E5C2E2E5CF4
:105360002E2E5C6472697665725C7372635C68632E
:105370003332663436305F646D61632E6300000043
:105380002DE9F04180460D461646002400271548B9
:10539000804507D01448804504D040F2F33113A073
:1053A00000F03CF955B1012D08D0022D06D0032D97
:1053B00004D04FF47D710DA000F030F908EB851199
:1053C0000E644FF4805006E0641CA4B2844201D9FC
:1053D000092700E00E640A6EB242F5D13846BDE8F6
:1053E000F081000000300540003405402E2E5C2E78
:1053F0002E5C2E2E5C2E2E5C2E2E5C6472697665E1
:10540000725C7372635C68633332663436305F6437
:105410006D61632E630000002DE9F04180460D466A
:105420001646002400271848804507D017488045B5
:1054300004D040F2BB4116A000F0F0F855B1012DA8
:1054400008D0022D06D0032D04D040F2BC4110A09C
:1054500000F0E4F808EB8511886C66F31F4088645F
:105460004FF4805009E0641CA4B2844201D909279A
:1054700003E08A6C66F31F428A648A6EB6EB124FB1
:10548000F1D13846BDE8F0810030054000340540D8
:105490002E2E5C2E2E5C2E2E5C2E2E5C2E2E5C6410
:1054A00072697665725C7372635C6863333266340A
:1054B00036305F646D61632E630000002DE9F041BA
:1054C0000446884615460C4E0C4FB44206D0BC42EA
:1054D00004D040F247710AA000F0A0F81349B4428A
:1054E00001EB880003D1C0F81458BDE8F081BC423C
:1054F000FBD1C0F82458F8E70030054000340540DF
:105500002E2E5C2E2E5C2E2E5C2E2E5C2E2E5C649F
:1055100072697665725C7372635C68633332663499
:1055200036305F646D61632E63000000000001404F
:1055300010B54FF4007101200BF018F81021BDE8F0
:10554000104001200BF012B810B54FF4007101208B
:105550000BF040F81021BDE8104001200BF006B818
:1055600010B54FF4007101200BF034F81021BDE8A4
:10557000104001200BF02EB810B54FF480710120BF
:105580000AF0F4FF0821BDE8104001200AF0EEBF48
:1055900010B54FF4807101200BF01CF80821BDE814
:1055A000104001200AF0E2BF10B54FF480710120D5
:1055B0000BF010F80821BDE8104001200BF00AB8EC
:1055C0001CB50020009001908DF800006A464FF451
:1055D000807101200AF0F2FE6A46082101200AF0DB
:1055E000EDFE4FF400746A46214601200AF0E6FE03
:1055F0006A46102101200AF0E1FE6A462146002099
:105600000AF0DCFE6A46210100200AF0D7FE6A4655
:10561000610100200AF0D2FE1CBD000010B50A4650
:10562000014602A00FF0AAFEFEE7000057726F6E5F
:105630006720706172616D65746572732076616C4C
:1056400075653A2066696C65202573206F6E206C45
:10565000696E652025640D0A0000000008B5084940
:1056600042F210720968B1FBF2F304E00093009972
:105670004A1E0092FBD2401E411CF7D108BD00001B
:10568000B482FF1F08B50A490A4A096891420BD93A
:10569000B1FBF2F304E0009300994A1E0092FBD2A2
:1056A000401E411CF7D108BD401E411CFCD108BD65
:1056B000B482FF1F8096980010B5AFF3008010BD34
:1056C00030B58FB0302103A8FAF77DFE0024019495
:1056D0000294012188030BF089FA012148040BF0A0
:1056E00085FA0125ADF80C50A802ADF80E0033483C
:1056F0000490334805900794ADF824400894ADF821
:105700002C400A948DF830408DF831508DF834409B
:105710008DF835408DF836508DF837408DF839507A
:10572000284C03AA00212046FFF748FD4FF4E07201
:1057300000212046FFF7C2FE01212046FFF708FDA9
:10574000012200212046FFF7BDFB0520ADF8060031
:105750001D4802902020ADF8040001A812F0A0FC22
:10576000BDF90600F021002804DB00F1E02080F8FC
:10577000001405E000F00F0000F1E02080F8141D97
:10578000BDF90600002809DB00F01F0105FA01F150
:105790004009800000F1E020C0F88012BDF9060049
:1057A000002808DB00F01F018D404009800000F157
:1057B000E020C0F800510FB030BD0000540004409C
:1057C0004CCD012000300540E10D010010B504462C
:1057D000002C05D0012C03D0BB2107A0FFF71EFF32
:1057E0001049012C03D0086840F0010002E008686D
:1057F00020F00100086010BD2E2E5C2E2E5C2E2E97
:105800005C2E2E5C2E2E5C6472697665725C7372FF
:10581000635C68633332663436305F65666D2E6371
:10582000000000000404014010B50446012C11D012
:10583000022C0FD0042C0DD0082C0BD0102C09D02A
:10584000202C07D0B4F5807F04D040F2951105A03C
:10585000FFF7E4FE0E480068204201D0012010BD91
:10586000002010BD2E2E5C2E2E5C2E2E5C2E2E5C6B
:105870002E2E5C6472697665725C7372635C686319
:105880003332663436305F65666D2E63000000008B
:105890001004014004480168012903D143F210219A
:1058A0000160016070470000000401400FB5064927
:1058B000009106490A6801924A6802928968039138
:1058C00001A90EC90EC00FBD3FCA024050040140DD
:1058D00010B50446002C21D0012C1FD0022C1DD065
:1058E000032C1BD0042C19D0052C17D0062C15D056
:1058F000072C13D0082C11D0092C0FD00A2C0DD056
:105900000B2C0BD00C2C09D00D2C07D00E2C05D055
:105910000F2C03D0DC2104A0FFF780FE0D480168A6
:1059200064F30711016010BD2E2E5C2E2E5C2E2E0E
:105930005C2E2E5C2E2E5C6472697665725C7372CE
:10594000635C68633332663436305F65666D2E6340
:1059500000000000080401402DE9F04705460F460D
:1059600000260024244885420BD223483830854243
:1059700007D92248854204D940F21B2120A0FFF715
:105980004DFE3F20FBF7C1F8DFF8A090D9F80000EA
:10599000C0F30048D9F8000020F48030C9F80000B6
:1059A0000120FBF7B7F809F10402106820F070003D
:1059B000103010602F609114101D04E0641CA4B21C
:1059C0008C4200D909260368DB05F7D5BF4200D019
:1059D00001261020FBF799F8106820F07000106085
:1059E0000020FBF797F8D9F8000068F31040C9F8D9
:1059F00000003046BDE8F087C00F0003DFFF07005E
:105A00002E2E5C2E2E5C2E2E5C2E2E5C2E2E5C649A
:105A100072697665725C7372635C68633332663494
:105A200036305F65666D2E6300000000080401409B
:105A3000034840F22311016043F2102101607047D6
:105A40000004014010B504462178002921D0012925
:105A50001FD002291DD003291BD0042919D00529E4
:105A600017D0062915D0072913D0082911D00929E4
:105A70000FD00A290DD00B290BD00C2909D00D29E4
:105A800007D00E2905D00F2903D06D210BA0FFF7F9
:105A9000C5FD2078164901EB80016278086862F341
:105AA000C7100860A278086862F305100860E27801
:105AB000086862F301000860002010BD2E2E5C2EE5
:105AC0002E5C2E2E5C2E2E5C2E2E5C64726976650A
:105AD000725C7372635C68633332663436305F6560
:105AE00078696E745F6E6D695F7377692E6300000D
:105AF0001010054003498A6D012383401A438A65CB
:105B0000002070470010054070B50F210B2002F0F7
:105B1000A3F80421022002F09FF84FF40051022064
:105B20000AF0EAFB0125164C01280BD00220FFF7F2
:105B300095FD402000F091F9C0F3401100F0030002
:105B400019B106E02570012070BD10B1257001204B
:105B500070BD0821022002F07FF80220FFF77EFDD1
:105B6000402000F07AF9C0F3401100F0030000B1CA
:105B700009B1002070BD02202070012070BD00001E
:105B80002083FF1F70B50F210B2002F065F807215D
:105B9000022002F061F84FF4005102200AF0ACFB41
:105BA0000125164C01280BD00220FFF757FD40209D
:105BB00000F053F9C0F3401100F0030019B106E002
:105BC0002570012070BD10B12570012070BD0B2122
:105BD000022002F041F80220FFF740FD402000F0D3
:105BE0003CF9C0F3401100F0030000B109B10020FE
:105BF00070BD02202070012070BD00002083FF1FB7
:105C000010B503210C2002F027F80421022002F035
:105C100023F80D49002008704870C87008712821C9
:105C20000A48FAF7D0FB38210948FAF7CCFB4FF4C1
:105C300086710848FAF7C7FB07480178092901D19E
:105C40000821017010BD00002083FF1F24CD01201A
:105C500044B7FF1FE4B8FF1FB183FF1F10B500F06A
:105C600089F84FF4804102200AF046FB18B1BDE8E4
:105C7000104000F00BB800F03BF802480068024901
:105C8000C86110BD7C83FF1F44B7FF1F10B5FFF72D
:105C90003BFF002826D0FF210E2001F0DDFF01216F
:105CA0000F2001F0D9FFE7210A2001F0D5FF0021E4
:105CB000062001F0D1FF0C480078012802D002280C
:105CC00005D008E00421022001F0C6FF03E008210E
:105CD000022001F0C1FF0121072001F0BDFF0349AF
:105CE0000220887310BD00002083FF1F44B7FF1FF0
:105CF00010B5FFF747FF00282DD0FF210E2001F03F
:105D0000ABFFE7210A2001F0A7FF0021062001F0E8
:105D1000A3FF11480078012802D0022809D010E022
:105D20000521022001F098FF2121032001F094FFBA
:105D300007E00A21022001F08FFF2221032001F059
:105D40008BFF0121072001F087FF0449032088739E
:105D500003491420087010BD2083FF1F44B7FF1FA4
:105D6000B183FF1F10B500F08DF8BDE810400C2086
:105D7000FFF7C0BE70B586B0002405940394049468
:105D8000019402940C268DF8146001258DF81550AD
:105D90008DF816508DF8174005A8FFF753FE0194B3
:105DA00002948DF804408DF806508DF8085001AA31
:105DB000290301200AF002FBADF80C600420ADF8C5
:105DC0000E001948049003A812F06AF9BDF90E00FC
:105DD000002809DB00F01F0105FA01F140098000ED
:105DE00000F1E020C0F88012BDF90E00F02100287B
:105DF00004DB00F1E02080F8001405E000F00F0063
:105E000000F1E02080F8141DBDF90E00002808DB29
:105E100000F01F018D404009800000F1E020C0F833
:105E2000005106B070BD0000655D010038B5054643
:105E30000C46002C10D043200090222003F088F95B
:105E400018B90121684603F0F9F803F09FF92246DA
:105E50002946222003F06AF838BD01B582B022201D
:105E600003F076F918B9012102A803F0E7F803F06E
:105E70008DF9012201A9222003F058F89DF80400B1
:105E80000EBD00002DE9FC47944D6889944E00EB4F
:105E9000C00006EB80000121FFF7C8FFA6F138091A
:105EA0004FF002080127FAE06889022100EBC000E8
:105EB00006EB8000801CFFF7B9FF688900EBC0008B
:105EC00016F82000DF2838D84FF4005102200AF0DD
:105ED00013FA012872D16878012818D0688900EB7C
:105EE000C00006EB80004088C0F38110A8702878BD
:105EF000012802D0022805D008E00121032001F08A
:105F0000ABFE03E00221032001F0A6FE6F7068895A
:105F100000EBC00006EB8000408800F01F00012865
:105F20004CD0688900EBC00006EB80004088C0F3CD
:105F30004220288100F072F940E0687802283DD0C4
:105F4000688900EBC00006EB80004088C0F3811038
:105F5000A87099F80E00012802D002282CD02DE05C
:105F6000688900EBC00006EB80004088C0F3422047
:105F7000288100F01BF9688900EBC00006EB800067
:105F800080F820702878012802D0022809D010E07B
:105F9000A878052101EB4010C1B2032001F05CFE9E
:105FA00007E0A878062101EB4010C1B2032001F000
:105FB00053FE85F8018001E085F80180688900EBD7
:105FC000C00006EB80004088C0F30230698901EB15
:105FD000C10106EB81014988C90B3BD0012839D9A1
:105FE000401E84B26889022100EBC00006EB8000ED
:105FF00000EB8400001DFFF719FF688900EBC0006B
:1060000006EB800000EB8400406810F4F04F12D0E3
:1060100002216846FFF70AFFA006010E688900EB1F
:10602000C00006EB8000001DFFF700FF042168465A
:10603000FFF7FCFE1CE0A006010E688900EBC00023
:1060400006EB8000001DFFF7F1FE06216846FFF712
:10605000EDFE0DE08006010E688900EBC00006EB46
:106060008000001DFFF7E2FE04216846FFF7DEFE18
:10607000688900EBC00006EB800080F82170688919
:10608000401C688168890A2801D1002068816889DC
:10609000012100EBC00006EB8000FFF7C7FE688916
:1060A00000EBC00016F82000C028BFF4FDAE3F2072
:1060B000FFF7D3FEC0070CD0688940B16889401E45
:1060C00000EBC00006EB800080F8207001E086F84D
:1060D0006471BDE8FC474220FFF7BFBE2083FF1F6D
:1060E0007CB7FF1F3EB5044600212B4A6B46505C2F
:1060F0005854491C0A29FADB9DF8060000F0F1000B
:106100008DF806002549A4B11B208DF802008DF8FA
:1061100003009DF8050040F0400001220B7942EA9F
:1061200043028DF80620897840EA81108DF8050039
:106130000BE0CA7840EA42008DF806009DF80500A1
:10614000897840EA81108DF805000A21684601F03F
:106150006DFDECB109F0C6FF114B124AE02418881E
:1061600000EB400102F821409DF805409DF80650E3
:1061700002EB810104EB05244C8042F20F7188424E
:1061800001D2401C188008480168491C01603EBDCE
:1061900009F09CFFE0E70000CAA802002083FF1F6F
:1061A0007083FF1FF0B9FF1F7883FF1F0EB500201B
:1061B00015496A460B5C1354401CC0B20A28F9D337
:1061C0009DF8070000F0F10010499DF806208B783B
:1061D00042EA83128DF80620098940EA41008DF8D1
:1061E00007000A21684601F021FD0948094A0121FA
:1061F000008800EB400002EB80000172064908684D
:10620000401C08600EBD0000C0A502002083FF1FD7
:106210007083FF1FF0B9FF1F7883FF1F0EB50020AA
:1062200011496A460B5C1354401CC0B20A28F9D3CA
:106230009DF8070000F0F1000C49098940EA41008F
:106240008DF807000A21684601F0F0FC0848094A69
:106250000121008800EB400002EB8000017206483B
:106260000168491C01600EBDB6A502002083FF1F16
:106270007083FF1FF0B9FF1F7883FF1F3EB500201A
:1062800021496A460B5C1354401C0A28FADB9DF82E
:10629000060000F0F1001D49CA7840EA42008DF87E
:1062A00006009DF80500897840EA8110C0B28DF89B
:1062B00005001749C97D012903D140F020008DF860
:1062C00005000A21684601F0B1FC09F0FFFE114A01
:1062D000114BE024108800EB400103F821409DF8A9
:1062E00005409DF8065003EB810104EB05244C802A
:1062F00042F20F71884201D2401C108007480168A9
:10630000491C01603EBD00005EA702002083FF1F04
:1063100024CD01207083FF1FF0B9FF1F7883FF1F7A
:106320007FB50020244A6946135C0B54401C0E289C
:10633000FADB9DF8060000F0F1002049CA7840EA37
:1063400042008DF806009DF80500897840EA81102A
:106350008DF805001A4800681A4948620E216846FF
:1063600001F064FC09F0B2FE174A184BE0241088D3
:1063700000EB400103F821409DF805409DF80650D0
:1063800003EB810104EB05244C809DF807309DF858
:106390000A409DF8085003EB04639DF8094024046B
:1063A00004EB052423444B6042F20F71884201D272
:1063B000401C10807FBD000002A902002083FF1F47
:1063C0007C83FF1F44B7FF1F7083FF1FF0B9FF1FBF
:1063D0007FB50020244A6946135C0B54401C0E28EC
:1063E000FADB9DF8060000F0F1002049CA7840EA87
:1063F00042008DF806009DF80500897840EA81107A
:106400008DF805000E21684601F010FC09F05EFED3
:10641000174B184AE024188800EB400102F821408D
:106420009DF805409DF8065002EB810104EB052420
:106430004C809DF807209DF80A409DF8085002EB1B
:1064400004629DF80940240404EB052422444A60B8
:1064500042F20F71884201D2401C18800648016840
:10646000491C01607FBD0000D4A802002083FF1FEB
:106470007083FF1FF0B9FF1F7883FF1F2DE9F041E4
:1064800088B0FE4C694694F821200B2A5ED2DFE8E2
:1064900002F05D060E172029323B444C55000020C7
:1064A000F74B1D5C0D54401C0E28FADB4EE000201B
:1064B000F34B8C331D5C0D54401C0E28FADB45E079
:1064C0000020EF4B9A331D5C0D54401C0E28FADB64
:1064D0003CE00020EA4BA8331D5C0D54401C0E2804
:1064E000FADB33E00020E64BB6331D5C0D54401C54
:1064F0001E28FADB2AE00020E14BD4331D5C0D544A
:10650000401C1E28FADB21E00020DD4BF2331D5C2D
:106510000D54401C1228FADB18E00020D94B1D5CFA
:106520000D54401C1228FADB10E00020D54B12332A
:106530001D5C0D54401C1E28FADB07E00020D14BE7
:1065400030331D5C0D54401C1228FADB9DF8060008
:1065500000F0F100CC49CB7840EA43008DF806000A
:106560009DF80500897840EA81108DF805000B2A16
:1065700038D2DFE802F037060B10151A1F24292E37
:1065800033000E21684601F051FB2BE00E216846D6
:1065900001F04CFB26E00E21684601F047FB21E0AC
:1065A0000E21684601F042FB1CE01E21684601F006
:1065B0003DFB17E01E21684601F038FB12E0122176
:1065C000684601F033FB0DE01221684601F02EFB16
:1065D00008E01E21684601F029FB03E0122168460D
:1065E00001F024FB09F072FDA84FA94AE023388886
:1065F00000EB400102F821309DF805309DF806506F
:1066000002EB810103EB05234B8094F821C0A14BE1
:10661000A14A4FF4FA75BCF10B0F16D2DFE80CF06B
:106620001506162636469AF3F1F0EF009DF807207E
:106630009DF80A309DF8085002EB03629DF809307E
:106640001B0403EB05231A444A60B5E19DF80720BB
:106650009DF80A309DF8085002EB03629DF809305E
:106660001B0403EB05231A444A60A5E19DF80720AB
:106670009DF80A309DF8085002EB03629DF809303E
:106680001B0403EB05231A444A6095E19DF807209B
:106690009DF80A309DF8085002EB03629DF809301E
:1066A0001B0403EB05231A444A6085E11688AE42B9
:1066B000CBD29DF807109DF80A509DF8088001EB99
:1066C00005619DF809502D0405EB08250D4403EBE9
:1066D00046114D609DF80B309DF80E509DF80C80D2
:1066E00003EB05639DF80D502D0405EB08252B44A5
:1066F0008B609DF80F309DF812509DF8108003EBD1
:1067000005659DF811301B0403EB08232B44CB6077
:106710009DF813309DF816509DF8148003EB056327
:106720009DF815502D0405EB08252B440B619DF8B1
:1067300017309DF81A509DF8188003EB05639DF8FB
:1067400019502D0405EB08252B444B610880761C5D
:10675000168031E11688AE4287D29DF807109DF869
:106760000A509DF8088001EB05619DF809502D0441
:1067700005EB08250D4403EB46114D609DF80B30E9
:106780009DF80E509DF80C8003EB05639DF80D50AD
:106790002D0405EB08252B448B609DF80F309DF8E8
:1067A00012509DF8108003EB05639DF811502D04E5
:1067B00005EB08252B44CB609DF813309DF816504F
:1067C0009DF8148003EB05639DF815502D0405EB2F
:1067D00008252B440B619DF817309DF81A5003EBE8
:1067E00005659DF819304FEA03489DF8183008EB0D
:1067F00003232B444B610880761C1680DCE0B5E057
:1068000060E027E0FFE71188A94222D29DF80750F7
:106810009DF80A609DF8088005EB06659DF8096003
:1068200003EB4113360406EB082635445D609DF802
:106830000B509DF80E609DF80C8005EB06659DF8E9
:106840000D60360406EB082635449D601880491C0F
:106850001180B1E01188A94233D29DF807509DF80C
:106860000A609DF8088005EB06659DF8096003EB5A
:106870004113360406EB082635440FE024CD0120F1
:1068800068A702006CA802002083FF1F7083FF1F0F
:10689000F0B9FF1FA48E01207283FF1F5D609DF879
:1068A0000B509DF80E609DF80C8005EB06659DF879
:1068B0000D60360406EB082635449D601880491C9F
:1068C000118079E01688AE4276D29DF807109DF8C7
:1068D0000A509DF8088001EB05619DF809502D04D0
:1068E00005EB08250D4403EB46114D609DF80B3078
:1068F0009DF80E509DF80C8003EB05639DF80D503C
:106900002D0405EB08252B448B609DF80F309DF876
:1069100012509DF8108003EB05639DF811502D0473
:1069200005EB08252B44CB609DF813309DF81650DD
:106930009DF8148003EB05639DF815502D0405EBBD
:1069400008252B440B619DF817309DF81A509DF8CF
:10695000188003EB05639DF819502D0405EB0825FD
:106960002B444B610880761C168025E01188A942D3
:1069700022D29DF807509DF80A609DF8088005EB2B
:1069800006659DF8096003EB4113360406EB082603
:1069900035445D609DF80B509DF80E609DF80C80AD
:1069A00005EB06659DF80D60360406EB08263544B8
:1069B0009D601880491C118042F20F71884201D2FB
:1069C000401C388005480168491C01600CF1010C2D
:1069D00084F821C008B0BDE8F08100007883FF1F73
:1069E0002DE9F04188B0FE4C694694F82120072A31
:1069F00039D2DFE802F038040C151E2730000020E1
:106A0000F84B1D5C0D54401C0E28FADB2BE00020D7
:106A1000F44B0E331D5C0D54401C1E28FADB22E0A3
:106A20000020F04B2C331D5C0D54401C1E28FADB5B
:106A300019E00020EB4B4A331D5C0D54401C12281A
:106A4000FADB10E00020E74B5C331D5C0D54401C6A
:106A50001E28FADB07E00020E24B7A331D5C0D5460
:106A6000401C1228FADB9DF8060000F0F100DE4918
:106A7000CB7840EA43008DF806009DF80500897840
:106A800040EA81108DF80500072A26D2DFE802F0DF
:106A90002504090E131821000E21684601F0C6F8DE
:106AA0001BE01E21684601F0C1F816E01E21684671
:106AB00001F0BCF811E01221684601F0B7F80CE0D3
:106AC0001E21684601F0B2F8C8480068C849C8628B
:106AD00003E01221684601F0A9F809F0F7FAC54D64
:106AE000C54AE023288800EB400102F821309DF8D8
:106AF00005309DF8066003EB062602EB81035E80FD
:106B000094F82160BD49BE4A4FF4FA77072E14D29B
:106B1000DFE806F01304146CC5F0EE009DF80710D2
:106B20009DF80A209DF8087001EB02619DF809208C
:106B3000120402EB07221144596070E11388BB4232
:106B4000FBD29DF807709DF80AC09DF8088007EBFE
:106B50000C679DF809C001EB43114FEA0C4C0CEB9C
:106B6000082C67444F609DF80B709DF80EC09DF88F
:106B70000C8007EB0C679DF80DC04FEA0C4C0CEB3A
:106B8000082C67448F609DF80F709DF812C09DF827
:106B9000108007EB0C679DF811C04FEA0C4C0CEB12
:106BA000082C6744CF609DF813709DF816C09DF8BF
:106BB000148007EB0C679DF815C04FEA0C4C0CEBEA
:106BC000082C67440F619DF817709DF81AC007EBF9
:106BD0000C689DF819709DF818C03F0407EB0C274E
:106BE00047444F6108805B1C138018E11388BB4247
:106BF00054D29DF807709DF80AC09DF8088007EBF5
:106C00000C679DF809C001EB43114FEA0C4C0CEBEB
:106C1000082C67444F609DF80B709DF80EC09DF8DE
:106C20000C8007EB0C679DF80DC04FEA0C4C0CEB89
:106C3000082C67448F609DF80F709DF812C09DF876
:106C4000108007EB0C679DF811C04FEA0C4C0CEB61
:106C5000082C6744CF609DF813709DF816C09DF80E
:106C6000148007EB0C679DF815C04FEA0C4C0CEB39
:106C7000082C67440F619DF817709DF81AC09DF8A5
:106C8000188007EB0C679DF819C04FEA0C4C0CEB11
:106C9000082C67444F6108805B1C1380BFE0138899
:106CA000BB4224D29DF807709DF80AC09DF8088069
:106CB00007EB0C679DF809C001EB43114FEA0C4C40
:106CC0000CEB082C67444F609DF80B709DF80EC0CC
:106CD0009DF80C8007EB0C679DF80DC04FEA0C4C3B
:106CE0000CEB082C67448F6008805B1C138096E0D7
:106CF00059E0FFE71388BB4254D29DF807709DF816
:106D00000AC09DF8088007EB0C679DF809C001EBED
:106D100043114FEA0C4C0CEB082C67444F609DF874
:106D20000B709DF80EC09DF80C8007EB0C679DF86A
:106D30000DC04FEA0C4C0CEB082C67448F609DF89B
:106D40000F709DF812C09DF8108007EB0C679DF83E
:106D500011C04FEA0C4C0CEB082C6744CF609DF837
:106D600013709DF816C09DF8148007EB0C679DF812
:106D700015C04FEA0C4C0CEB082C67440F619DF8D2
:106D800017709DF81AC09DF8188007EB0C679DF8E6
:106D900019C04FEA0C4C0CEB082C67444F6108807B
:106DA0005B1C13803BE01388BB4238D29DF8077010
:106DB0009DF80AC09DF8088007EB0C679DF809C094
:106DC00001EB43114FEA0C4C0CEB082C67444F606D
:106DD0009DF80B709DF80EC007EB0C6712E00000E9
:106DE00024CD012068A702002083FF1F7C83FF1FA2
:106DF00044B7FF1F7083FF1FF0B9FF1FA48E01204F
:106E00007283FF1F9DF80DC09DF80C804FEA0C4C5B
:106E10000CEB082C67448F6008805B1C138042F2E7
:106E20000F71884201D2401C288005480168491C26
:106E30000160761C84F8216008B0BDE8F081000094
:106E40007883FF1F70B586B00020344A01A9135C17
:106E50000B54401CC0B21228F9D39DF80A0000F070
:106E6000F1002F49CA7840EA42008DF80A009DF8E7
:106E70000900897840EA81108DF80900122101A8E3
:106E800000F0D4FE09F022F9264D274AE023288895
:106E900000EB400102F821309DF809309DF80A40CE
:106EA00002EB810103EB04234B809DF80B209DF83E
:106EB0000E109DF80C3002EB01619DF80D201204BC
:106EC00002EB03228C1819490C609DF80F209DF8E5
:106ED00012309DF8106002EB03629DF811301B0424
:106EE00003EB062313444B60114E3188B1F5FA7F52
:106EF00007D2104A02EB4112546093601080491C83
:106F0000318042F20F71884201D2401C28800A4928
:106F10000868401C086006B070BD00001AA9020095
:106F20002083FF1F7083FF1FF0B9FF1F24CD0120B6
:106F30007283FF1FA48E01207883FF1F7FB500207E
:106F4000244A6946135C0B54401C0E28FADB9DF85A
:106F5000060000F0F1002049CA7840EA42008DF8AE
:106F600006009DF80500897840EA81108DF805003B
:106F70000E21684600F05AFE09F0A8F8174B184A8F
:106F8000E024188800EB400102F821409DF80540FC
:106F90009DF8065002EB810104EB05244C809DF81E
:106FA00007209DF80A409DF8085002EB04629DF806
:106FB0000940240404EB052422444A6042F20F7184
:106FC000884201D2401C188006480168491C0160B3
:106FD0007FBD0000E2A802002083FF1F7083FF1F17
:106FE000F0B9FF1F7883FF1F2DE9F04F85B0DFF860
:106FF000C89399F8287099F829103944491E81429C
:107000003EDBEE4CEE4D216A2A68511A502937D3E7
:10701000A17C0126012932D0DFF8A8C3411CCAB2E5
:107020008CF80520E8496B4691F81AA0BAF1010FD7
:1070300029D00021DFF8948318F801B003F801B0DB
:10704000491CC9B20E29F7D39DF8061001F0F101D1
:107050009CF8033041EA43018DF806109DF80510B5
:107060009CF8023041EA83118DF80510974216D33F
:107070009DF80A1041EA02118DF80A1018E0E67432
:1070800005B0BDE8F08F0021DFF8448318F801B0A7
:1070900003F801B0491CC9B21229F7D3D4E79DF80F
:1070A0000A10C7F107031A4441EA02118DF80A10C9
:1070B00009EB0001002291F8F830DFEDC60A9FEDE0
:1070C000C60A012B0DD0022B37D0BC4A4FF0090E57
:1070D000032B92F83470117B52895BD0042B78D04B
:1070E000F1E059F820108DF80710C1F3012343EAAD
:1070F00081038DF808309DF80930C1F383173B43B5
:107100008DF8093084F834202672C1F3892201EE0B
:10711000102AB8EE411A61EE200AFCEEE00A10EEE9
:10712000902A2270C1F3090100EE901AF8EE600A6D
:1071300020EE800A84ED010AC5E059F820108DF890
:107140000710C1F3012343EA81038DF808309DF84D
:107150000930C1F383173B438DF8093084F834209C
:1071600003222272C1F3892201EE102AB8EE411ADD
:1071700061EE200AFCEEE00A10EE902A2270C1F3C4
:10718000090100EE901AF8EE600A20EE800A84ED04
:10719000010A98E059F82080C8F3484303EB8303C1
:1071A000A382C8F3072C0CEB8C0CA4F816C008F0D3
:1071B000FF0884F80D804FF0020B84F808B027B95F
:1071C00084F83460854F87F800E09A4202D96381E1
:1071D00003E01CE00AB9FA2262816289624501D2A9
:1071E000A4F80AC0414500D809B984F80C80217B75
:1071F0008DF8071061894A008DF808209DF8092054
:1072000042EAD1118DF80910296821625BE059F832
:107210002030C3F3484C4FEA8C0CA4F814C0C3F3DD
:1072200007284FEA8808A4F81680637304232372A2
:1072300027B984F83460694B83F800E0624501D9CE
:10724000A4F80AC06289424501D2A4F80A80628982
:1072500002F00303D21A92B2628101EE102A99ED74
:107260003D0AF8EE411A9FED5E1A5E4F21EE812A2B
:10727000C0EE021A11EE903ABB4202DD6423637342
:107280000EE001EE902AF8EE611A61EE811A80EEAE
:10729000211A81EE200ABCEEC00A10EE103A637388
:1072A000637B994200D801B92373217B8DF80710C5
:1072B00051008DF808109DF8091041EAD2118DF89F
:1072C0000910296821625146DFF81C81DFF81CA1F2
:1072D000474F42F20F7B012930D00E21684600F063
:1072E000A5FC08F0F3FE3888E02200EB400108F826
:1072F00021209DF805209DF8063008EB810102EB66
:1073000003224A809DF807209DF80A309DF808C0A6
:1073100002EB03629DF809301B0403EB0C231A44B3
:107320004A60584501D2401C3880DAF80000401C01
:10733000CAF80000A67428682063A1E659F8200066
:10734000010E8DF80E10010C8DF80D10010A8DF84C
:107350000C108DF80B00286860621221684600F05E
:1073600065FC08F0B3FE3888E02200EB400108F825
:1073700021209DF805209DF8063008EB810102EBE5
:1073800003224A809DF807209DF80A309DF808C026
:1073900002EB03629DF809301B0403EB0C231A4433
:1073A0004A60584501D2401C3880DAF80000401C81
:1073B000CAF80000BEE70000E4B8FF1F44B7FF1F93
:1073C0007C83FF1F2083FF1F24CD0120A8A502007E
:1073D000F0A80200CDCC4C3D0AD7233CB183FF1F5F
:1073E000CDCCCC3C0000A040F0B9FF1F7883FF1F3C
:1073F0007083FF1F2DE9F04188B000205349544BA2
:107400006A4691F83910491EC1EB011103EB4101A5
:107410000B5C1354401CC0B21E28F9D39DF8060023
:1074200000F0F1004B490A7940EA42008DF806006D
:107430009DF80500897840EA81108DF805001E212D
:10744000684600F0F3FB08F04DFEDFF80CC1434A3C
:10745000C023BCF8001001EB410002F820309DF879
:1074600005309DF8064002EB800003EB04234380C7
:107470009DF807009DF80A209DF8083000EB026097
:107480009DF80920120402EB03228418344804609A
:107490009DF80B209DF80E309DF80C5002EB036216
:1074A0009DF80D301B0403EB0523D61846609DF8AC
:1074B0000F209DF812309DF8105002EB03629DF8EA
:1074C00011301B0403EB0523D71887609DF81320A8
:1074D0009DF816309DF8145002EB03629DF81530AC
:1074E0001B0403EB05231344C3609DF817209DF88C
:1074F0001A509DF8188002EB05629DF819502D0472
:1075000005EB082515440561DFF85880B8F8002020
:10751000B2F5FA7F0BD2144800EB4210446086604B
:10752000C760036145610180521CA8F8002042F247
:107530000F70814202D2491CACF800100B49086858
:10754000401C086008B0BDE8F081000074610220B2
:10755000CAA502002083FF1F7083FF1FF0B9FF1F21
:1075600024CD01207283FF1FA48E01207883FF1F8A
:1075700070B586B0002027496A460B5C1354401C46
:10758000C0B21628F9D39DF8060000F0F100224998
:107590000A7940EA42008DF806009DF805008978D6
:1075A00040EA81108DF805001621684600F03EFB88
:1075B00008F098FD194D1A4AC023288800EB4001B5
:1075C00002F821309DF805309DF8064002EB81015C
:1075D00003EB04234B80134C2288B2F5FA7F0CD2C4
:1075E000114B124901EB42111E684E605E688E60BD
:1075F0009B68CB600880521C228042F20F71884247
:1076000001D2401C28800A480168491C016006B06C
:1076100070BD0000D8A602002083FF1F7083FF1FEB
:10762000F0B9FF1F7283FF1F24CD0120A48E01201B
:107630007883FF1F70B586B00020304901AA0B5C2B
:107640001354401CC0B21228F9D39DF80A0000F070
:10765000F1002B490A7940EA42008DF80A009DF8B2
:107660000900897840EA81108DF80900254890F8D2
:107670002700012802D0022807D00CE09DF8110055
:1076800040F003008DF8110005E09DF8110040F076
:107690000B008DF81100122101A800F0C7FA08F0C4
:1076A00021FD194B194AC024188800EB400102F84B
:1076B00021409DF809409DF80A5002EB810104EB3E
:1076C00005244C80124C2188B1F5FA7F0AD2114D65
:1076D000114A02EB41122E6856606D689560108069
:1076E000491C218042F20F71884201D2401C18804F
:1076F0000A480168491C016006B070BDEEA6020090
:107700002083FF1F746102207083FF1FF0B9FF1FE9
:107710007283FF1F24CD0120A48E01207883FF1FD8
:1077200070B588B0002029496A460B5C1354401C90
:10773000C0B21E28F9D39DF8060000F0F1002449DC
:107740000A7940EA42008DF806009DF80500897824
:1077500040EA81108DF805001E21684600F066FAA7
:1077600008F0C0FC1B4D1C4AC023298801EB4100D6
:1077700002F820309DF805309DF8064002EB8000AD
:1077800003EB04234380154C2388B3F5FA7F10D212
:10779000134A144800EB431016684660566886602A
:1077A0009668C660D66806611269426101805B1CFA
:1077B000238042F20F70814201D2491C29800A487D
:1077C0000168491C016008B070BD000000A70200FC
:1077D0002083FF1F7083FF1FF0B9FF1F7283FF1FFD
:1077E00024CD0120A48E01207883FF1F70B588B0BE
:1077F000002029496A460B5C1354401CC0B21E2865
:10780000F9D39DF8060000F0F10024490A7940EA16
:1078100042008DF806009DF80500897840EA811045
:107820008DF805001E21684600F000FA08F05AFCA9
:107830001B4D1C4AC023298801EB410002F820306F
:107840009DF805309DF8064002EB800003EB042311
:107850004380154C2388B3F5FA7F10D2134A14489D
:1078600000EB431016684660566886609668C660EE
:10787000D66806611269426101805B1C238042F276
:107880000F70814201D2491C29800A480168491CB5
:10789000016008B070BD00001EA702002083FF1F1A
:1078A0007083FF1FF0B9FF1F7283FF1F24CD0120DB
:1078B000A48E01207883FF1F3EB500201C496A4634
:1078C0000B5C1354401C0A28FADB9DF8060000F0FC
:1078D000F1001849CA7840EA42008DF806009DF888
:1078E0000500897840EA81108DF805000A21684674
:1078F00000F09CF908F0EAFB0F4A104BE0241088D6
:1079000000EB400103F821409DF805409DF806502A
:1079100003EB810104EB05244C8042F20F71884295
:1079200001D2401C108006480168491C01603EBD20
:10793000AEA802002083FF1F7083FF1FF0B9FF1F56
:107940007883FF1F3EB500201C496A460B5C135428
:10795000401C0A28FADB9DF8060000F0F1001849E7
:10796000CA7840EA42008DF806009DF80500897843
:1079700040EA81108DF805000A21684600F056F9AA
:1079800008F0A4FB0F4A104BE024108800EB4001E4
:1079900003F821409DF805409DF8065003EB810156
:1079A00004EB05244C8042F20F71884201D2401C46
:1079B000108006480168491C01603EBD3CA70200DA
:1079C0002083FF1F7083FF1FF0B9FF1F7883FF1F05
:1079D0007FB50021324A6B46545C5C54491C0E2929
:1079E000FADB9DF8061001F0F1012E4AD37841EA46
:1079F00043018DF806109DF80510927841EA821136
:107A00008DF805108021012802D002280CD015E045
:107A100002208DF807008DF8081000208DF809006D
:107A2000FF208DF80A0009E003208DF807008DF88B
:107A3000081087208DF809008DF80A100E2168467D
:107A400000F0F4F808F042FB174A184BC0241088E5
:107A500000EB400103F821409DF805409DF80650D9
:107A600003EB810104EB05244C809DF807309DF861
:107A70000A409DF8085003EB04639DF80940240474
:107A800004EB052423444B6042F20F71884201D27B
:107A9000401C108006480168491C01607FBD000041
:107AA00050A702002083FF1F7083FF1FF0B9FF1F44
:107AB0007883FF1FF0B585B0002032496A460B5C21
:107AC0001354401C1228FADB9DF8060000F0F10068
:107AD0002D49CA7840EA42008DF806009DF805005D
:107AE000897840EA81108DF805001221684600F07F
:107AF0009DF808F0EBFA254B254AE024188800EBA6
:107B0000400102F821409DF805409DF8065002EB27
:107B1000810104EB05244C801E4C2188B1F5FA7FCD
:107B200023D29DF807209DF80A509DF8086002EBCB
:107B300005629DF809502D0405EB06251544164AEB
:107B400002EB411255609DF80B509DF80E609DF8B8
:107B50000C7005EB06659DF80D60360406EB0726F4
:107B6000354495601080491C218042F20F71884293
:107B700001D2401C188009480168491C016005B009
:107B8000F0BD0000B8A802002083FF1F7083FF1F14
:107B9000F0B9FF1F7283FF1FA48E01207883FF1F9F
:107BA0003EB500201C496A460B5C1354401C0A2851
:107BB000FADB9DF8060000F0F1001849CA7840EAA7
:107BC00042008DF806009DF80500897840EA811092
:107BD0008DF805000A21684600F028F808F076FACA
:107BE0000F4A104BE024108800EB400103F82140BD
:107BF0009DF805409DF8065003EB810104EB052438
:107C00004C8042F20F71884201D2401C108006481D
:107C10000168491C01603EBD46A702002083FF1F8A
:107C20007083FF1FF0B9FF1F7883FF1F38B504462C
:107C30000D464320009072B6222001F089FA38B92F
:107C40000121684601F0FAF92946204601F0F6F9CB
:107C500001F09CFA62B638BD08B58DF800008DF8C9
:107C60000110222001F074FA18B105490020887132
:107C700008BD0221684601F0E1F901F087FA08BD6C
:107C80002083FF1F38B53E4800903E483E490068BB
:107C90000860401C37D03D490120087000203C4C52
:107CA000810101F5FC210978A0292FD0401CC0B228
:107CB0007F28F5D31E2020710720E070042084F86F
:107CC00039004FF64D31282000F0D6F840F27961A6
:107CD0002A2000F0D1F84DF69A312C2000F0CCF893
:107CE000B1EE040A092000F0D1F8B1EE040A0D202B
:107CF00000F0CCF8B7EE000A1D2000F0C7F8BDE890
:107D0000384000F079B800200860C7E74FF4FC2144
:107D100001EB801140221E48F8F73CFB607800B16F
:107D200001201C490870112000F050F81A4880ED1D
:107D3000000A152000F04AF8184880ED000A1D20BE
:107D400000F044F8164880ED000A342000F03EF8B8
:107D5000144880ED000A282000F02CF800280ED0EE
:107D6000282000F027F8104908802A2000F022F887
:107D70000E4908802C2000F01DF80D49088038BD00
:107D800053AE0043080C00035491FF1FCC83FF1F28
:107D900074610220A683FF1F1C8DFF1F208DFF1F13
:107DA0004C83FF1F4483FF1FA883FF1FAA83FF1F6D
:107DB000AC83FF1F08B500210091034908440088E7
:107DC0000090BDF8000008BD7461022008B59FED69
:107DD000050A8DED000A04490844006800909DEDF5
:107DE000000A08BD00000000746102200149084437
:107DF00000687047746102202DE9F04100241D4F96
:107E0000A0264FF4FC25A10101F5FC210878FF28EC
:107E10000ED0641CE4B27F2CF5D3284600F048F85D
:107E20003E702846BDE8F04140221249F8F777BE7F
:107E30003E7005EB841040220E49F8F770FE002CCE
:107E400015D0601E810101F5FC210978A02907D019
:107E5000A41E05EB8410BDE8F041002100F03FB8FE
:107E600005EB8010BDE8F041002100F038B8BDE816
:107E7000F08100007461022003B503490844BDF895
:107E8000041001800CBD00007461022001B52DEDCD
:107E9000020B02490844009901600EBD7461022082
:107EA000014A1044016070477461022000F017B865
:107EB00070B50546FDF7BCFD0120FDF787FC4FF4CA
:107EC00080742046FDF7B0FC0128FAD172B628462E
:107ED000F8F72AFE62B6BDE87040FDF7DBBC70B56E
:107EE00005460E46FDF7A4FD0120FDF76FFC4FF49B
:107EF00080742046FDF798FC0128FAD172B631460D
:107F00002846FDF729FD62B6BDE87040FDF7C2BC0A
:107F100010B586B004466846FDF7C8FC9DE807002A
:107F200003AB07C3012C0DD0022C0DD0032C0DD0B8
:107F30000398049980B289B20844059900EB014086
:107F400006B010BD0398FBE70498F9E70598F7E73A
:107F50000EB509293BD2DFE801F0050B11171D23EF
:107F6000292F350002461CA168460DF017FA2EE0B5
:107F700002461AA168460DF011FA28E0024619A13E
:107F800068460DF00BFA22E0024618A168460DF093
:107F900005FA1CE0024617A168460DF0FFF916E04D
:107FA000024616A168460DF0F9F910E0024615A147
:107FB00068460DF0F3F90AE0024614A168460DF098
:107FC000EDF904E0024613A168460DF0E7F96846B2
:107FD00000F024F80EBD000025580000253031586F
:107FE00000000000253032580000000025303358D2
:107FF00000000000253034580000000025303558BE
:1080000000000000253036580000000025303758A9
:108010000000000025303858000000002DE9F0472E
:108020000023544D544E554FDFF85481DFF854C1AE
:108030009AE07E2925D94FF09B09427802EB012175
:108040008AB2002114E035F831A092450ED805EB34
:10805000C10ABAF802A0924508D335F8314005EBC1
:10806000C101121B898811448CB203E0491C89B2FA
:108070004945E8D3801C444931F8341019448BB287
:1080800072E098F80120102A06D01C2A27D00C2A6A
:1080900048D00020BDE8F0874FF01209002214E01C
:1080A00036F832A051450ED306EBC20ABAF802A048
:1080B000514508D836F8324006EBC202091B9288B7
:1080C00011448CB203E0521C92B24A45E8D3401CE2
:1080D0002949903131F8341019448BB244E04FF003
:1080E0000409002214E037F832A051450ED307EB03
:1080F000C20ABAF802A0514508D837F8324007EB57
:10810000C202091B928811448CB203E0521C92B245
:108110004A45E8D3401C1949203131F8341019443C
:108120008BB221E04FF00A09002214E03CF832A0A3
:1081300051450ED30CEBC20ABAF802A0514508D83B
:108140003CF832400CEBC202091B928811448CB2FD
:1081500003E0521C92B24A45E8D3401C0949503111
:1081600031F8341019448BB2017800297FF461AFE3
:1081700018468FE734E4020028BE02002CA9020052
:108180009C83FF1F545B03000CE902002DE9F843B8
:108190006B4800906B4C6C4800996C4E084483E02F
:1081A000217800297FD022781346082502E05B0859
:1081B0006D1EEDB2DF07FAD0F82A22D008DC802A43
:1081C00027D0C02A23D0E02A1FD0F02A06D11AE0F7
:1081D000FC2A14D0FE2A10D0FF2A0CD000225A4BC1
:1081E000009F08333B449C421DD31846231A12D0EB
:1081F000012B4FD112E0FE22F1E7FC22EFE7F8223B
:10820000EDE7F022EBE7E022E9E7C022E7E7802292
:10821000E5E70022E3E74E4911433BE06FF47F417D
:1082200041EA022136E0484B009F1B1D3B444FF0C2
:10823000FF0C4FF6FF776FF07F489C4214D318462F
:10824000231A06D0012B06D0022B07D0032B21D1F5
:1082500007E011461EE04CEA02211BE007EB024159
:1082600018E048EA026115E0844213D3231A06D0CD
:10827000012B06D0022B08D0032B0BD108E01146AE
:1082800008E04CEA022105E00DE007EB024101E0C5
:1082900048EA0261FFF70AFE0098201A133005EB46
:1082A000C000B07003E0641E8442BFF479AFB078C0
:1082B0000324B8B327480179427901EB022182797E
:1082C000C079120402EB0060084430610020FFF71F
:1082D0001FFE00F0070120FA01F2884010441E49F9
:1082E000884203D91D490844400803E01B4949421C
:1082F0000844400031690125814216D1124A009894
:10830000383A1044FFF7D2FD154900980844316906
:10831000D0F8B50D884206D11248057012490020E8
:10832000087006E003E0F47003E0F57001E002205D
:10833000F07020467471BDE8F84300F015B90000F4
:1083400053AE0043490C0003ED5DFFBFB882FF1F31
:108350000000FFFFB463022033DDD35334DDD3D3F9
:108360000050FFBFCB83FF1FB183FF1F04490522CD
:108370000A7011224A7009228A70C8707047000082
:10838000F463022010B5094CE079032809D860791C
:1083900000F0EAF8E079401CE0710548006860618F
:1083A00010BD0020A071E07110BD0000B882FF1F59
:1083B0007C83FF1F00200321044A535C1844C0B291
:1083C000491CC9B23F29F8D370470000B4630220AA
:1083D00006480178052905D14178112902D1817813
:1083E000092901D000207047C0787047B46302208B
:1083F0002DE9F041594C0027A771A07A0125584E6C
:10840000002802D0FFF7E4FF98B1FFF7D3FF96F8FA
:108410003F1088427ED1FFF7DBFF69287FD02BDC3D
:10842000652848D023DC78B3012875D0642830D182
:108430003BE0E089217A884203D9F420607100F0A2
:1084400093F80020474BE289315CA7890F44A7814C
:1084500000EB8217D955401CC0B24028F4D3521CFF
:10846000E28128466571BDE8F04100F07DB86728DB
:108470003BD068280DD12BE0F1285ED005DC6A28BE
:1084800053D0F02805D154E009E0F22859D0FF2854
:1084900061D0F1206071BDE8F04100F065B8F020D6
:1084A0006071BDE8F04100F05FB838466771BDE823
:1084B000F04100F059B8A781E781307920727079D6
:1084C00060722846A5726071BDE8F04100F04CB8BA
:1084D000A781E78130792072707960722846A57291
:1084E0006071BDE8F04100F03FB8A772A089317912
:1084F000C2B2914209D17179B1EB102F05D102209E
:108500006071BDE8F04100F02FB8F3206071BDE864
:10851000F04102E019E002E01DE000F025B8284635
:108520006571BDE8F04100F01FB8BDE8F041FFF70C
:108530002DBEBDE8F041FFF725BFBDE8F041FFF7D4
:1085400021BFBDE8F041FFF71DBFF2206071BDE81B
:10855000F04100F009B8BDE8F0810000B882FF1FCB
:10856000B46302204092FF1F10B504464021254805
:10857000F7F729FFF12C27D00BDC022C1CD003DCF1
:1085800084B1012C33D110E0032C12D0F02C2ED169
:1085900016E0F22C1CD0F32C1ED0F42C20D0FF2C93
:1085A00025D121E000F034F821E0012000F064F84A
:1085B0001DE000F083F81AE0022000F05DF816E0FC
:1085C000F02000F059F812E0F12000F055F80EE02C
:1085D000F22000F051F80AE0F32000F04DF806E038
:1085E000F42000F049F802E0FF2000F045F8012CEB
:1085F00007D0FF2C05D004480168044841610121DF
:10860000817110BDF46302207C83FF1FB882FF1FBD
:1086100070B5154D2878002825D0144890F8DC0056
:10862000032820D10020FFF773FC03460020FFF74A
:108630009DFE0F4C012020716371180AA071180C67
:10864000E071180E20720B4800786072CC20A07286
:1086500000F062F884F83F0040222146034811F000
:1086600005FF0020287070BDB882FF1F40B2FF1FB9
:10867000F4630220CB83FF1F70B504460C4D2978AC
:10868000002914D00B4991F8DC1003290FD10020E8
:10869000FFF73EFC2046FFF769FE074880F83F40A1
:1086A00001464022034811F0E1FE0020287070BD11
:1086B000B882FF1F40B2FF1FF463022070B5124C56
:1086C000207800281FD0114890F8DC0003281AD128
:1086D0000020FFF71DFC0320FFF748FE0C4803783D
:1086E0000C480371A1784171E2788271C578114418
:1086F0002B44194480F83F1001464022034811F0F2
:10870000B5FE0020207070BDB882FF1F40B2FF1F71
:10871000CB83FF1FF463022000200321044A535C33
:108720001844C0B2491CC9B23F29F8D370470000B1
:10873000F463022010B5134C2078002820D0124892
:1087400090F8DC0003281BD10020FFF7E1FB034673
:108750000020FFF70BFE0D49012008714B71180A2C
:108760008871180CC871180E087209480078487290
:10877000C92088724022044811F078FE0020207041
:1087800010BD0000B882FF1F40B2FF1FF46302203B
:10879000CB83FF1F70B51C481C4D1D4C90F8330057
:1087A000002824D02868B0F57A7F20D94FF40071D2
:1087B000002007F0A1FD012819D1607838B9154BC8
:1087C000154A164916480FF015FF012060702079F0
:1087D00001280CD1124890F8DC00032807D10020B2
:1087E000207100231A4681210D4810F085F8A079E8
:1087F000002808D028686169401A642803D9BDE8B8
:108800007040FFF7BFBD70BD746102207C83FF1F05
:10881000B882FF1F0483FF1F0C92FF1FD082FF1F2F
:1088200040B2FF1F10B5AFF3008010BD70B5044615
:108830000D460D4884420AD00C48844207D00C48AB
:10884000844204D04FF457710AA0FCF7E7FE35B11B
:10885000012D04D040F25D3106A0FCF7DFFE206858
:1088600065F38A20206070BD00E0044000E404400D
:1088700000E804402E2E5C2E2E5C2E2E5C2E2E5CEC
:108880002E2E5C6472697665725C7372635C6863D9
:108890003332663436305F6932632E630000000085
:1088A0002DE9F04704462DED028B0D46904600263B
:1088B00000274FF002099FED648A002D45D0B8F1E2
:1088C000000F42D0614884420AD06148844207D0F8
:1088D0006048844204D04FF496715FA0FCF79EFE7E
:1088E00068496868884204D940F22D115AA0FCF703
:1088F00095FE286890B1012810D002280ED00328D8
:108900000CD004280AD0052808D0062806D007284D
:1089100004D04FF4977150A0FCF780FE5A48006ACB
:10892000C0F3023159480068C8402A6801219140CB
:10893000D5ED020A95ED011A236BDB0603D5236BF7
:1089400003F003077F1C12B103E0042670E04FF030
:10895000030900EE100AB8EE412AB8EE400AC0EE54
:10896000021A00EE101AB8EE402A81EE820A01EED9
:10897000909AF8EE600AB8EE612AF0EE001A62EE04
:10898000212A02EE107AB8EE422A42EE212A32EE75
:10899000A02A70EE421AFCEEC00AF8EE602A30EE11
:1089A000620A10EE103AB3F17C5F06DBB8EE600AA3
:1089B000F7EE000A30EE200A01E0B8EE600AB4EEED
:1089C000C20AF1EE10FA01D8042631E011EE903A15
:1089D0002F4DAB4201DD04262AE0BCEEC00A10EEAA
:1089E000103AB0FBF3F0B0FBF1F000EE100AF8EE35
:1089F000410AB8EE400A70EEC00A00EE100AB8EE66
:108A0000400A80EE808AE06A62F31240E062BCEEC7
:108A1000E10A10EE100A4108E06A61F30400E06226
:108A200010EE100AA0EB5001E06A61F30C20E06246
:108A3000B8F1000F02D00EB988ED008A3046BDECC7
:108A4000028BBDE8F08700000000000000E0044059
:108A500000E4044000E804402E2E5C2E2E5C2E2EF6
:108A60005C2E2E5C2E2E5C6472697665725C73726D
:108A7000635C68633332663436305F6932632E6319
:108A800000000000801A060000400540B482FF1F6D
:108A90000000784270B504460D460A4884420AD068
:108AA0000948844207D00948844204D040F2F521A5
:108AB00007A0FCF7B3FD206A10490D40284320624F
:108AC00070BD000000E0044000E4044000E8044001
:108AD0002E2E5C2E2E5C2E2E5C2E2E5C2E2E5C649A
:108AE00072697665725C7372635C68633332663494
:108AF00036305F6932632E6300000000DF56F000FD
:108B000070B504460D460D4884420AD00C48844294
:108B100007D00C48844204D040F2FF110AA0FCF7B1
:108B20007DFD35B1012D04D04FF4007106A0FCF796
:108B300075FD206865F30000206070BD00E0044012
:108B400000E4044000E804402E2E5C2E2E5C2E2E05
:108B50005C2E2E5C2E2E5C6472697665725C73727C
:108B6000635C68633332663436305F6932632E6328
:108B7000000000001FB5002331224FF40041012006
:108B800007F05CFD002330224FF48041012007F004
:108B900055FD0121402008F069F80A4C204600F0FC
:108BA00015F8002101910391074902916A4601A934
:108BB000204600F019F901212046FFF7A1FF04B07B
:108BC000284610BD00E80440801A060010B504468F
:108BD0000B4884420AD00B48844207D00A4884429A
:108BE00004D04FF4BD7109A0FCF718FD206820F0F7
:108BF00001002060206840F400402060002010BD8B
:108C000000E0044000E4044000E804402E2E5C2E06
:108C10002E5C2E2E5C2E2E5C2E2E5C647269766588
:108C2000725C7372635C68633332663436305F69DA
:108C300032632E630000000070B504460D460C48F8
:108C4000844209D00B48844206D00B48844203D0AA
:108C5000D5210AA0FCF7E2FC2DB1012D03D0D621CD
:108C600006A0FCF7DBFC206865F30820206070BDDF
:108C700000E0044000E4044000E804402E2E5C2E96
:108C80002E5C2E2E5C2E2E5C2E2E5C647269766518
:108C9000725C7372635C68633332663436305F696A
:108CA00032632E630000000070B504460D460C4888
:108CB000844209D00B48844206D00B48844203D03A
:108CC000F8210AA0FCF7AAFC2DB1012D03D0F9214F
:108CD00006A0FCF7A3FC206865F34920206070BD66
:108CE00000E0044000E4044000E804402E2E5C2E26
:108CF0002E5C2E2E5C2E2E5C2E2E5C6472697665A8
:108D0000725C7372635C68633332663436305F69F9
:108D100032632E630000000070B505460C46002645
:108D2000234885420AD02348854207D022488542FD
:108D300004D040F2CD2121A0FCF770FC012C31D0F1
:108D4000022C2FD0042C2DD0082C2BD0102C29D065
:108D5000402C27D0802C25D0B4F5007F22D0B4F54C
:108D6000806F1FD0B4F5805F1CD0B4F5804F19D050
:108D7000B4F5803F16D0B4F5003F13D0B4F5802F82
:108D800010D0B4F5801F0DD0B4F5001F0AD0B4F593
:108D9000800F07D0B4F5000F04D040F2CE2107A019
:108DA000FCF73CFCE869204200D00126304670BD4B
:108DB00000E0044000E4044000E804402E2E5C2E55
:108DC0002E5C2E2E5C2E2E5C2E2E5C6472697665D7
:108DD000725C7372635C68633332663436305F6929
:108DE00032632E630000000070B504460D4616463F
:108DF000002D4BD0002C49D0254884420AD025486C
:108E0000844207D02448844204D040F2A31123A016
:108E1000FCF704FC2C496868884204D94FF4D271ED
:108E20001EA0FCF7FBFB286890B1012810D0022897
:108E30000ED003280CD004280AD0052808D0062814
:108E400006D0072804D040F2A51114A0FCF7E6FBD9
:108E5000206820F001002060206840F4004020607D
:108E6000206840F001002060324629462046FFF786
:108E700017FD216821F040012160216821F40041A3
:108E80002160216821F00101216070BD042070BDC6
:108E900000E0044000E4044000E804402E2E5C2E74
:108EA0002E5C2E2E5C2E2E5C2E2E5C6472697665F6
:108EB000725C7372635C68633332663436305F6948
:108EC00032632E6300000000801A060010B50446CD
:108ED000084884420AD00848844207D007488442A0
:108EE00004D040F24B3106A0FCF798FB94F8280020
:108EF00010BD000000E0044000E4044000E804402D
:108F00002E2E5C2E2E5C2E2E5C2E2E5C2E2E5C6465
:108F100072697665725C7372635C6863333266345F
:108F200036305F6932632E63000000002DE9F05F88
:108F300007460E4691464FF47A7AD0463E4D0121BF
:108F4000284600F085F80021284600F081F84FF40B
:108F5000003B07E0B8F1010804D200F017F9002047
:108F6000BDE8F09F59462846FFF7D6FE0128F1D00C
:108F700001212846FFF760FE5446D8464146284660
:108F8000FFF7CAFE834601212846FFF7C5FEBBF165
:108F9000000F05D020B1012000EB4700C7B206E06A
:108FA000641E601CEAD1DBE7641E601C0ED08021C9
:108FB0002846FFF7B1FE0028F6D02C463946204659
:108FC00000F0F2F957464FF4806504E00020C7E74F
:108FD0007F1E781C0AD029462046FFF79DFE0128F7
:108FE000F6D00025A9F1010827461AE000F0CEF8D6
:108FF0000020B5E7454503D101213846FFF716FCAF
:10900000544602E0641E601C11D040213846FFF730
:1090100083FE0028F6D03846FFF758FF06F8010B0C
:109020006D1C4D45E6D300F0B1F8012098E700F043
:10903000ADF8002094E7000000E804400A4601462D
:109040004FF47A73014800F037B9000000E804409B
:1090500070B504460D460D4884420AD00C4884423F
:1090600007D00C48844204D040F205310AA0FCF736
:10907000D5FA35B1012D04D040F2063106A0FCF737
:10908000CDFA206865F3CF30206070BD00E0044069
:1090900000E4044000E804402E2E5C2E2E5C2E2EB0
:1090A0005C2E2E5C2E2E5C6472697665725C737227
:1090B000635C68633332663436305F6932632E63D3
:1090C0000000000070B504460D46124884420AD0E4
:1090D0001148844207D01148844204D040F28F31B5
:1090E0000FA0FCF79BFA2B4600224FF400312046DC
:1090F00000F046F900280BD101212046FFF79CFD26
:109100002B462046BDE870400122104900F038B9D6
:1091100070BD000000E0044000E4044000E80440AA
:109120002E2E5C2E2E5C2E2E5C2E2E5C2E2E5C6443
:1091300072697665725C7372635C6863333266343D
:1091400036305F6932632E630000000001000200C8
:1091500070B506460C4C01212046FFF779FF00212F
:109160002046FFF775FF4FF47A7529462046FFF732
:10917000A9FF002807D12B4631462046BDE87040A4
:10918000002200F02DB870BD00E804402DE9F04148
:109190004FF47A752C464FF40037104E02E0641EEF
:1091A000601C0BD039463046FFF7B6FD0028F6D0DC
:1091B000344601212046FFF777FD05E00020BDE899
:1091C000F0816D1E681C07D010212046FFF7A4FD1A
:1091D0000028F6D00120F2E70020F0E700E8044084
:1091E0002DE9F04106460F4615469846244886422A
:1091F0000AD02448864207D02348864204D040F251
:10920000C93122A0FCF70AFA7F2F04D940F2CA31F3
:109210001EA0FCF703FA012D05D025B140F2CB3199
:109220001AA0FCF7FBF9434601228021304600F0EA
:10923000A7F8044604BB45EA4700C1B2304600F037
:10924000B3F84DB1434600224FF48021304600F080
:1092500097F8044644B10FE0434601220821304606
:1092600000F08EF80446F5E74FF480613046FFF7D2
:1092700053FD012800D101242046BDE8F081000003
:1092800000E0044000E4044000E804402E2E5C2E80
:109290002E5C2E2E5C2E2E5C2E2E5C647269766502
:1092A000725C7372635C68633332663436305F6954
:1092B00032632E63000000002DE9F84305460E4698
:1092C00017469946204885420AD02048854207D053
:1092D0001F48854204D040F24B411EA0FCF79EF986
:1092E00000240020009056B34FF480581CE04B46F9
:1092F00001228021284600F043F80446A4B90098D2
:10930000315C284600F050F84B46012208212846DF
:1093100000F036F8044641462846FFF7FDFC0128D8
:1093200008D00098401C00900098B84208D0002C4B
:10933000DDD005E041462846FFF7ACFB00E0042401
:109340002046BDE8F883000000E0044000E404404B
:1093500000E804402E2E5C2E2E5C2E2E5C2E2E5C01
:109360002E2E5C6472697665725C7372635C6863EE
:109370003332663436305F6932632E63000000009A
:1093800030B505460920EC690C40012A01D1A14203
:1093900001D0144300D10020002803D0002B01D0BD
:1093A0005B1EF0E730BD000070B504460D4608486E
:1093B00084420AD00748844207D00748844204D038
:1093C00040F23D3105A0FCF729F984F8245070BD26
:1093D00000E0044000E4044000E804402E2E5C2E2F
:1093E0002E5C2E2E5C2E2E5C2E2E5C6472697665B1
:1093F000725C7372635C68633332663436305F6903
:1094000032632E630000000010B5042000F0CFF995
:1094100001040FD5401EC04380B2F7F767F99FEDF6
:109420000C1B53EC112BF7F780F8F7F7C9F900EE96
:10943000100A10BDF7F75AF99FED071B53EC112BDB
:10944000F7F773F8F7F7BCF900EE100A10BD00004B
:10945000FCA9F1D24D6240BFFCA9F1D24D62403F60
:1094600010B5022000F0A3F9F7F740F99FED051BB6
:1094700053EC112BF7F759F8F7F7A2F900EE100AA1
:1094800010BD00007B14AE47E17A543F10B540EAAE
:109490000102072A1DD844F2070242EA402080B2A6
:1094A00040EA811040EAC101002000F099F94FF430
:1094B0008061062000F094F94FF40061052000F06F
:1094C0008FF90448006804498861BDE8104000F045
:1094D0000DB810BD7C83FF1F3083FF1F10B500F057
:1094E00061F8BDE810400820FCF704BB70B586B0F9
:1094F00000240594039404940194029408268DF8A2
:10950000146001258DF815508DF816508DF8174010
:1095100005A8FCF797FA019402948DF804408DF8A1
:1095200006508DF8085001AA2902002006F046FFD7
:10953000ADF80C600320ADF80E001948049003A8A4
:109540000EF0AEFDBDF90E00002809DB00F01F0192
:1095500005FA01F14009800000F1E020C0F8801216
:10956000BDF90E00F021002804DB00F1E02080F8B6
:10957000001405E000F00F0000F1E02080F8141D59
:10958000BDF90E00002808DB00F01F018D404009E6
:10959000800000F1E020C0F8005106B070BD00006E
:1095A000DD94010070B5FFF75BFF754C84ED010A97
:1095B000FFF72AFF84ED020A00F0F6F894ED020AA4
:1095C000704910EE100A884202D80120207001E094
:1095D0000020207094ED020A10EE100AF7F7ACF8A4
:1095E00041EC100B0BF084FF51EC100BF7F7E8F88F
:1095F00000EE100A84ED020A94ED020AD4ED050A89
:10960000B4EEE00AF1EE10FA04DD94ED020A84ED06
:10961000030A03E09FED5C0A84ED030A94ED070A58
:10962000B5EEC00AF1EE10FA0ED094ED070A10EE76
:10963000100AB0F17E5F07D094ED030AD4ED070A5B
:1096400020EE200A84ED030A94ED010AD4ED030A0A
:1096500020EE200A84ED040A4C4D2868A169D4ED5F
:10966000040A401A00EE100AB8EE400A60EE200A22
:109670009FED471A80EE810A10EE100AF7F75CF8AA
:1096800094ED081B53EC112BF6F7A8FE41EC100BE0
:1096900084ED080B94ED010A3E4A10EE100A904248
:1096A0001DDC2868A169D4ED030A401A00EE100AF7
:1096B0009FED391AB8EE400A60EE200A80EE810A6A
:1096C00010EE100AF7F738F894ED0A1B53EC112B43
:1096D000F6F784FE41EC100B84ED0A0B4DE094ED9F
:1096E000010A2E4810EE101A914223DD94ED010A72
:1096F00010EE101A81421DDC2868A169D4ED030A1E
:10970000401A00EE100A9FED261AB8EE400A60EEED
:10971000200A80EE810A10EE100AF7F70DF894ED9A
:109720000A1B53EC112BF6F759FE41EC100B84ED9C
:109730000A0B22E094ED010A10EE101A81421CDDA2
:109740002868A169D4ED030A401A00EE100A9FEDC3
:10975000151AB8EE400A60EE200A80EE810A10EE7B
:10976000100AF6F7E9FF94ED0A1B53EC112BF6F7FC
:1097700035FE41EC100B84ED0A0B2868A06170BD2A
:109780003083FF1F6F1203BB000000007C83FF1FAC
:1097900000BA5B4A0000C040000061450000404143
:1097A0000000E144000061440620AFF3008001B5F1
:1097B00082B04020FFF7CCFC18B9012102A8FFF7C6
:1097C0003DFCFFF7E3FC022201A94020FFF7AEFBBE
:1097D0009DF805009DF8041000EB012080B20EBD3D
:1097E00008B58DF80000080A8DF801008DF8021008
:1097F0004020FFF7ADFC18B105490020487008BDB6
:1098000003216846FFF71AFCFFF7C0FC08BD000003
:109810003083FF1F02480068002800D000477047CF
:10982000B461022002484068002800D00047704719
:10983000B461022002488068002800D000477047C9
:10984000B46102200248C068002800D00047704779
:10985000B461022002480069002800D00047704728
:10986000B461022002484069002800D000477047D8
:10987000B461022002488069002800D00047704788
:10988000B46102200248C069002800D00047704738
:10989000B46102200248006A002800D000477047E7
:1098A000B46102200248406A002800D00047704797
:1098B000B46102200248806A002800D00047704747
:1098C000B46102200248C06A002800D000477047F7
:1098D000B46102200248006B002800D000477047A6
:1098E000B46102200248406B002800D00047704756
:1098F000B46102200248806B002800D00047704706
:10990000B46102200248C06B002800D000477047B5
:10991000B46102200248006C002800D00047704764
:10992000B46102200248406C002800D00047704714
:10993000B46102200248806C002800D000477047C4
:10994000B46102200248C06C002800D00047704774
:10995000B46102200248006D002800D00047704723
:10996000B46102200248406D002800D000477047D3
:10997000B46102200248806D002800D00047704783
:10998000B46102200248C06D002800D00047704733
:10999000B46102200248006E002800D000477047E2
:1099A000B46102200248406E002800D00047704792
:1099B000B46102200248806E002800D00047704742
:1099C000B46102200248C06E002800D000477047F2
:1099D000B46102200248006F002800D000477047A1
:1099E000B46102200248406F002800D00047704751
:1099F000B46102200248806F002800D00047704701
:109A0000B46102200248C06F002800D000477047B0
:109A1000B46102200348D0F88000002800D000473D
:109A200070470000B46102200348D0F88400002889
:109A300000D0004770470000B46102200348D0F80E
:109A40008800002800D0004770470000B461022061
:109A50000348D0F88C00002800D000477047000071
:109A6000B46102200348D0F89000002800D00047DD
:109A700070470000B46102200348D0F89400002829
:109A800000D0004770470000B46102200348D0F8BE
:109A90009800002800D0004770470000B461022001
:109AA0000348D0F89C00002800D000477047000011
:109AB000B46102200348D0F8A000002800D000477D
:109AC00070470000B46102200348D0F8A4000028C9
:109AD00000D0004770470000B46102200348D0F86E
:109AE000A800002800D0004770470000B4610220A1
:109AF0000348D0F8AC00002800D0004770470000B1
:109B0000B46102200348D0F8B000002800D000471C
:109B100070470000B46102200348D0F8B400002868
:109B200000D0004770470000B46102200348D0F81D
:109B3000B800002800D0004770470000B461022040
:109B40000348D0F8BC00002800D000477047000050
:109B5000B46102200348D0F8C000002800D00047BC
:109B600070470000B46102200348D0F8C400002808
:109B700000D0004770470000B46102200348D0F8CD
:109B8000C800002800D0004770470000B4610220E0
:109B90000348D0F8CC00002800D0004770470000F0
:109BA000B46102200348D0F8D000002800D000475C
:109BB00070470000B46102200348D0F8D4000028A8
:109BC00000D0004770470000B46102200348D0F87D
:109BD000D800002800D0004770470000B461022080
:109BE0000348D0F8DC00002800D000477047000090
:109BF000B46102200348D0F8E000002800D00047FC
:109C000070470000B46102200348D0F8E400002847
:109C100000D0004770470000B46102200348D0F82C
:109C2000E800002800D0004770470000B46102201F
:109C30000348D0F8EC00002800D00047704700002F
:109C4000B46102200348D0F8F000002800D000479B
:109C500070470000B46102200348D0F8F4000028E7
:109C600000D0004770470000B46102200348D0F8DC
:109C7000F800002800D0004770470000B4610220BF
:109C80000348D0F8FC00002800D0004770470000CF
:109C9000B46102200348D0F80001002800D000473A
:109CA00070470000B46102200348D0F80401002886
:109CB00000D0004770470000B46102200348D0F88C
:109CC0000801002800D0004770470000B46102205E
:109CD0000348D0F80C01002800D00047704700006E
:109CE000B46102200348D0F81001002800D00047DA
:109CF00070470000B46102200348D0F81401002826
:109D000000D0004770470000B46102200348D0F83B
:109D10001801002800D0004770470000B4610220FD
:109D20000348D0F81C01002800D00047704700000D
:109D3000B46102200348D0F82001002800D0004779
:109D400070470000B46102200348D0F824010028C5
:109D500000D0004770470000B46102200348D0F8EB
:109D60002801002800D0004770470000B46102209D
:109D70000348D0F82C01002800D0004770470000AD
:109D8000B46102200348D0F83001002800D0004719
:109D900070470000B46102200348D0F83401002865
:109DA00000D0004770470000B46102200348D0F89B
:109DB0003801002800D0004770470000B46102203D
:109DC0000348D0F83C01002800D00047704700004D
:109DD000B46102200348D0F84001002800D00047B9
:109DE00070470000B46102200348D0F84401002805
:109DF00000D0004770470000B46102200348D0F84B
:109E00004801002800D0004770470000B4610220DC
:109E10000348D0F84C01002800D0004770470000EC
:109E2000B46102200348D0F85001002800D0004758
:109E300070470000B46102200348D0F854010028A4
:109E400000D0004770470000B46102200348D0F8FA
:109E50005801002800D0004770470000B46102207C
:109E60000348D0F85C01002800D00047704700008C
:109E7000B46102200348D0F86001002800D00047F8
:109E800070470000B46102200348D0F86401002844
:109E900000D0004770470000B46102200348D0F8AA
:109EA0006801002800D0004770470000B46102201C
:109EB0000348D0F86C01002800D00047704700002C
:109EC000B46102200348D0F87001002800D0004798
:109ED00070470000B46102200348D0F874010028E4
:109EE00000D0004770470000B46102200348D0F85A
:109EF0007801002800D0004770470000B4610220BC
:109F00000348D0F87C01002800D0004770470000CB
:109F1000B46102200348D0F88001002800D0004737
:109F200070470000B46102200348D0F88401002883
:109F300000D0004770470000B46102200348D0F809
:109F40008801002800D0004770470000B46102205B
:109F50000348D0F88C01002800D00047704700006B
:109F6000B46102200348D0F89001002800D00047D7
:109F700070470000B46102200348D0F89401002823
:109F800000D0004770470000B46102200348D0F8B9
:109F90009801002800D0004770470000B4610220FB
:109FA0000348D0F89C01002800D00047704700000B
:109FB000B46102200348D0F8A001002800D0004777
:109FC00070470000B46102200348D0F8A4010028C3
:109FD00000D0004770470000B46102200348D0F869
:109FE000A801002800D0004770470000B46102209B
:109FF0000348D0F8AC01002800D0004770470000AB
:10A00000B46102200348D0F8B001002800D0004716
:10A0100070470000B46102200348D0F8B401002862
:10A0200000D0004770470000B46102200348D0F818
:10A03000B801002800D0004770470000B46102203A
:10A040000348D0F8BC01002800D00047704700004A
:10A05000B46102200348D0F8C001002800D00047B6
:10A0600070470000B46102200348D0F8C401002802
:10A0700000D0004770470000B46102200348D0F8C8
:10A08000C801002800D0004770470000B4610220DA
:10A090000348D0F8CC01002800D0004770470000EA
:10A0A000B46102200348D0F8D001002800D0004756
:10A0B00070470000B46102200348D0F8D4010028A2
:10A0C00000D0004770470000B46102200348D0F878
:10A0D000D801002800D0004770470000B46102207A
:10A0E0000348D0F8DC01002800D00047704700008A
:10A0F000B46102200348D0F8E001002800D00047F6
:10A1000070470000B46102200348D0F8E401002841
:10A1100000D0004770470000B46102200348D0F827
:10A12000E801002800D0004770470000B461022019
:10A130000348D0F8EC01002800D000477047000029
:10A14000B46102200348D0F8F001002800D0004795
:10A1500070470000B46102200348D0F8F4010028E1
:10A1600000D0004770470000B46102200348D0F8D7
:10A17000F801002800D0004770470000B4610220B9
:10A180000348D0F8FC01002800D0004770470000C9
:10A19000B46102202DE9FC5F00260327DFF88C83E1
:10A1A000DFF88CA3DFF88CB3E34DE44C47F6EF31D6
:10A1B0004FF44879092828D2DFE800F02705294C18
:10A1C000A1D6FEFDFC000022DC200CF0E1FECDE972
:10A1D000007030237F2210210F20F7F7CDFF2021C0
:10A1E0003520F8F7DBFF1020F8F7DEFFB8F80000A5
:10A1F000F8F7E0FFD2A0F8F7B7F82868216B401A0B
:10A20000484502D9112060702670BDE8FC9F0022ED
:10A21000DC200CF0BDFECDE900703023822210213D
:10A220000F20F7F7A9FF20213220F8F7B7FF102001
:10A23000F8F7BAFFB8F80000F8F7BCFFC3A0F8F7CA
:10A2400093F82968206B081A4845DED91E206070F3
:10A250002670DAE70022DC200CF09AFECDE90070CF
:10A260003023822210210F20F7F786FF1020F8F705
:10A270009BFFB9480088F8F79DFF10210F20F8F7E1
:10A280008DFFB648007868B9B5A0F8F71FFC00212B
:10A290000420F7F717FEB4A0F8F718FC10210F20E0
:10A2A000F7F71AFEB248007868B9B2A0F8F70EFCCA
:10A2B00000210420F7F706FEABA0F8F707FC1021F9
:10A2C0000F20F7F709FEE07E80B9AC48006868B15E
:10A2D000ABA0F8F7FBFB00210420F7F7F3FDA2A0E9
:10A2E000F8F7F4FB10210F20F7F7F6FD2868216B33
:10A2F000401A41F28831884287D9267085E70022CA
:10A30000DC200CF045FECDE90070302382221021C4
:10A310000F20F7F731FF20211F20F8F73FFF102013
:10A32000F8F742FFB8F80000F8F744FF95A0F8F7F7
:10A330001BF8DAF800004FF07C51884209DADBF8AC
:10A340000000884205DD26700B2060700120A0709F
:10A350005BE72868216B401AB0F5FA6FCED906206A
:10A3600020702868206350E70022DC200CF010FEEB
:10A37000CDE900703023822210210F20F7F7FCFE78
:10A3800020211F20F8F70AFF1020F8F70DFFB8F87A
:10A390000000F8F70FFF7BA0F7F7E6FFDAF8000000
:10A3A0004FF07C51884210DADBF8000088420CDD67
:10A3B000267002E07BE035E013E006F0E3FE0C20BF
:10A3C00060700120A07020711FE72868216B401A7F
:10A3D00040F6C411884291D9062020702868206375
:10A3E00013E70022DC200CF0D3FDCDE90070302310
:10A3F000822210210F20F7F7BFFE20213A20F8F724
:10A40000CDFE1020F8F7D0FEB8F80000F8F7D2FE25
:10A4100061A0F7F7A9FF2868216B401A484597D932
:10A420002670F2E60022DC200CF0B2FDCDE90070CF
:10A430003222142311463720F7F79EFE1020F8F73A
:10A44000B3FEB8F80000F8F7B5FE5548807830B193
:10A4500001280CD0022812D003281FD117E0352183
:10A460003E20F8F79BFE4FA0F8F730FB16E03521B1
:10A470003920F8F793FE4DA0F8F728FB0EE03521C0
:10A480003920F8F78BFE4BA0F8F720FB06E03521CA
:10A490003E20F8F783FE49A0F8F718FB2868216BE7
:10A4A000401A40F2DC5188428ED92670ADE6002277
:10A4B000DC200CF06DFDCDE90070302382221021EC
:10A4C0000F20F7F759FE20212F20F8F767FE102004
:10A4D000F8F76AFEB8F80000F8F76CFE3948807BA0
:10A4E000022804D003280AD0012810D016E0202129
:10A4F0003120F8F753FE34A0F7F736FF0EE02021A5
:10A500002620F8F74BFE33A0F7F72EFF06E02021B8
:10A510002620F8F743FE33A0F7F726FF2868216BC3
:10A52000401A4845C2D926706FE60000AA83FF1F73
:10A530008C83FF1F8883FF1F7C83FF1FB083FF1F57
:10A54000C9E8D6C3B3C9B9A621000000D7A2B2E1B9
:10A55000C2EBB4EDCEF32100AE83FF1F3183FF1FAA
:10A56000494E4132323600004552524F52210000CE
:10A570002683FF1F46555342333032005491FF1F4C
:10A580004F545000D5FDD4DABDF8C8EB5143D3D5B4
:10A59000C6AD2E2E2E000000B2BBD6A7B3D621002A
:10A5A0007461022037535053000000003230535082
:10A5B00053000000353053505300000033535053C4
:10A5C0000000000044B7FF1FD3D5C6ADD2D1BDFBFC
:10A5D000D3C321005044D3D5C6ADD2D1BDFBD3C324
:10A5E000210000005143D3D5C6ADD2D1BDFBD3C3AA
:10A5F0002100000010B50121052005F07DFE38B1D5
:10A6000015480178022909D001780B2906D01EE0EF
:10A6100001221146114809F0FDFC18E010490A68B2
:10A620008368D21AFA2A02D2052101700FE00A6863
:10A630008368D21AFA2A08D309688268891AB1F5A0
:10A640007A7F02D20821017001E000210170BDE88B
:10A6500010400020FBF74EBA6083FF1F0044024009
:10A660007C83FF1F10B54FF48041022005F044FEAB
:10A6700038B116480178032909D001780C2906D091
:10A680001EE001221146124809F0C4FC18E01149ED
:10A690000A68C368D21AFA2A02D2062101700FE0B2
:10A6A0000A68C368D21AFA2A08D30968C268891AE4
:10A6B000B1F57A7F02D20921017001E00021017019
:10A6C000BDE810400E20FBF715BA00006083FF1FA5
:10A6D000004402407C83FF1F10B54FF480610020CE
:10A6E00005F00AFE38B116480178012909D0017831
:10A6F0000A2906D01EE001221146124809F08AFC00
:10A7000018E011490A684368D21AFA2A02D20421D1
:10A7100001700FE00A684368D21AFA2A08D3096860
:10A720004268891AB1F57A7F02D20721017001E0EF
:10A7300000210170BDE810400A20FBF7DBB90000E2
:10A740006083FF1F004402407C83FF1FF0B585B08B
:10A750000024049402940394009401940A268DF832
:10A7600010608DF8004001258DF802508DF80450DE
:10A770006A460121052005F021FE6A46A902002053
:10A7800005F01CFE6A46A903022005F017FE01230E
:10A7900000225F023946104605F050FF8DF8024056
:10A7A0006A463946002005F009FE8DF811508DF8F3
:10A7B000125002208DF8130004A8FBF743F90E2570
:10A7C0008DF8105004A8FBF73DF98DF8104004A84F
:10A7D000FBF738F9ADF808600620ADF80A0021480B
:10A7E000039002A80DF05CFCBDF90A000AF002FE1D
:10A7F000BDF90A000F210AF04BFEBDF90A000AF06C
:10A8000020FEADF808500720ADF80A001648039066
:10A8100002A80DF045FCBDF90A000AF0EBFDBDF9F8
:10A820000A000F210AF034FEBDF90A000AF009FE01
:10A83000ADF808400820ADF80A000C48039002A8C3
:10A840000DF02EFCBDF90A000AF0D4FDBDF90A0096
:10A850000F210AF01DFEBDF90A000AF0F2FD05B055
:10A86000F0BD0000D9A6010065A60100F5A5010014
:10A8700010B51248037812494FF47A72032B07D1AE
:10A880000B68C4681B1B934202D90C21017010BDD8
:10A890000378012B07D10B6844681B1B934202D934
:10A8A0000A21017010BD0378022BFBD1096883686F
:10A8B000C91A9142F6D90B21017010BD6083FF1FA8
:10A8C0007C83FF1F10B500F0BFF94FF40044214610
:10A8D000002005F04BFE0A20FAF7D4FE21460020A6
:10A8E00005F078FE0AF0A2FA00F008FA00F05EF92E
:10A8F000112000F055FAAC48807901287ED0B120B3
:10A9000000F04EFA012000F061FA2C2000F05EFA0F
:10A910002D2000F05BFAB22000F042FA012000F096
:10A9200055FA2C2000F052FA2D2000F04FFAB320F7
:10A9300000F036FA012000F049FA2C2000F046FA27
:10A940002D2000F043FA012000F040FA2C2000F006
:10A950003DFA2D2000F03AFAB42000F021FA072049
:10A9600000F034FAC02000F01BFAA22000F02EFA0A
:10A97000022000F02BFA842000F028FAC12000F019
:10A980000FFAC52000F022FAC22000F009FA0A20CE
:10A9900000F01CFA002000F019FAC32000F000FAC1
:10A9A0008A2000F013FA2A2000F010FAC42000F0E8
:10A9B000F7F98A2000F00AFAEE2000F007FAC52025
:10A9C00000F0EEF90E2000F001FA212000F0E8F985
:10A9D0003A2000F0E5F9052000F0F8F9E02000F059
:10A9E000DFF9022000F0F2F91C2000F0EFF9072057
:10A9F00000F0ECF9122000F0E9F900E064E0372003
:10AA000000F0E4F9322000F0E1F9292000F0DEF94D
:10AA10002D2000F0DBF9292000F0D8F9252000F0E6
:10AA2000D5F92B2000F0D2F9392000F0CFF9002021
:10AA300000F0CCF9012000F0C9F9032000F0C6F9BC
:10AA4000102000F0C3F9E12000F0AAF9032000F083
:10AA5000BDF91D2000F0BAF9072000F0B7F9062073
:10AA600000F0B4F92E2000F0B1F92C2000F0AEF97E
:10AA7000292000F0ABF92D2000F0A8F92E2000F0DD
:10AA8000A5F92E2000F0A2F9372000F09FF93F2011
:10AA900000F09CF9002000F099F9002000F096F9F0
:10AAA000022000F093F9102000F090F9F02000F05F
:10AAB00077F9012000F08AF9132000F071F9BDE860
:10AAC0001040292000F06CB9B12000F069F9052090
:10AAD00000F07CF93C2000F079F93C2000F076F998
:10AAE000B22000F05DF9052000F070F93C2000F084
:10AAF0006DF93C2000F06AF9B32000F051F905200F
:10AB000000F064F93C2000F061F93C2000F05EF9AF
:10AB1000052000F05BF93C2000F058F93C2000F0E3
:10AB200055F9B42000F03CF9032000F04FF9C020A3
:10AB300000F036F90E2000F049F90E2000F046F939
:10AB4000042000F043F9C12000F02AF9C52000F0EC
:10AB50003DF9C22000F024F90D2000F037F9002063
:10AB600000F034F9C32000F01BF98D2000F02EF91D
:10AB70002A2000F02BF9C42000F012F98D2000F0FB
:10AB800025F9EE2000F022F9C52000F009F9062091
:10AB900000F01CF9202000F003F93A2000F000F941
:10ABA000552000F013F919E77461022010B58EB03A
:10ABB000302102A8F5F707FC0121C80306F016F8BA
:10ABC0000121480406F012F80120ADF80800ADF8A4
:10ABD0000A0000210391194A04928DF82C008DF887
:10ABE0002D108DF832108DF83500154C02AA204634
:10ABF000FAF7E4FA4FF49B7200212046FAF75EFC64
:10AC000001212046FAF7A4FA0220ADF802000D480F
:10AC100001902420ADF8000068460DF041FABDF91E
:10AC200002000F210AF054FCBDF902000AF0FCFBFF
:10AC3000BDF902000AF01FFC0EB010BD000002407A
:10AC400000340540E1AC01001CB5002000900190EB
:10AC500001248DF8004002208DF805006A4680210D
:10AC6000012005F0ABFB6A46E103002005F0A6FBDE
:10AC70008DF802406A460421052005F09FFB04215F
:10AC8000052005F073FC1CBD10B50B4CA079012804
:10AC900004D10A480021017118214171FFF712FE09
:10ACA000607800B1012000F0DBF8207900F0A4F812
:10ACB000BDE8104000F004B8746102209C83FF1FBF
:10ACC00010B500214F239F22084600F0D9F8034811
:10ACD000BDE810404FF4C84100F01EB94CD501202A
:10ACE00010B5022200210348FAF7C6F902490120F3
:10ACF000087010BD003405409C83FF1F10B588B05C
:10AD00001C2101A8F5F75FFB0121880405F0AEFFC7
:10AD100000232B224021012005F090FC0023282253
:10AD20002021012005F08AFC00208DF812008DF80A
:10AD3000150004218DF813108DF814008DF8100003
:10AD40008DF811008DF80F0001218DF816108DF887
:10AD500017108DF819008DF81A008DF81B008DF86A
:10AD60001C008DF81D008DF818108DF804108DF85A
:10AD700005008DF806108DF807008DF808100520E5
:10AD80008DF80900054C01A9204607F063FE01215A
:10AD9000204607F0BDFD08B010BD000000000240D5
:10ADA00070B50546084C0521204607F0EDFD00284A
:10ADB000F9D08021012005F0D9FB29462046BDE8C5
:10ADC000704008F073B800000000024070B50546FE
:10ADD000084C0521204607F0D7FD0028F9D0802136
:10ADE000012005F0F7FB29462046BDE8704008F039
:10ADF0005DB800000000024010B504462046F5F79B
:10AE000075FC9FED101B53EC112BF5F700FC41EC8A
:10AE1000100B9FED0E1B0AF05BFD5CB19FED0D1B4F
:10AE200051EC100B53EC112BF5F77FFBF5F76BFC96
:10AE300082B200E00122BDE810400621074809F077
:10AE400077BD00000000000000005940175D74D17C
:10AE50004517DD3F0000000000489D40005C0140B8
:10AE600010B504463620FFF79BFF24B1BDE8104023
:10AE7000A820FFF7ABBFBDE810406820FFF7A6BFD2
:10AE80002DE9F0410746884615461E462A20FFF761
:10AE900087FF1F4C20793844000AFFF797FF20797D
:10AEA0003844C0B2FFF792FF20792844C0F307204E
:10AEB000FFF78CFF20792844C0B2FFF787FF2B20D3
:10AEC000FFF76EFF60794044000AFFF77FFF60796B
:10AED0004044C0B2FFF77AFF60793044C0F30720E6
:10AEE000FFF774FF60793044C0B2FFF76FFF2C208A
:10AEF000FFF756FF074C0521204607F045FD0028C7
:10AF0000F9D02046BDE8F041002107F001BD000066
:10AF10009C83FF1F0000024070B50D460C4C02469A
:10AF200000212046FAF72CFA2A4600212046FAF79B
:10AF300073FA8021012005F04DFB012200212046FB
:10AF4000F9F7C0FFBDE870400121024807F0E0BCFE
:10AF500000340540000002402DE9F0412DED028B48
:10AF600082B01020F8F720F900210846F8F716F90A
:10AF7000C04C2088F8F71EF9BFA0F7F7F5F90021BB
:10AF80005820F8F70BF9BF49012091ED000AF8F7B6
:10AF90004DF8BDA0F7F79AFDBC4F3878BC4E4FF086
:10AFA00010053178084208D02088CDE9000500233B
:10AFB000B8A219469020F8F703F938783178884319
:10AFC00008D02088CDE900050023B3A219469020BF
:10AFD000F8F7F6F830783978884308D02088CDE93A
:10AFE00000050023ACA219469020F8F7E9F838785C
:10AFF00050B9307840B92088CDE900050023A5A2DA
:10B0000019469020F8F7DCF8A449FF20122309889C
:10B01000CDE900109F2219460020F7F76BF8A048F1
:10B020000088F8F7C7F814210020F8F7B7F89DA0BA
:10B03000F7F74CFD0C20F8F7B7F803210020F6F7DE
:10B0400041FF99A0F7F742FD6FF00208414600204A
:10B05000F6F738FF1020F8F7A7F8944F944D97EDC6
:10B06000000AD5ED000A9FED938A934CB4EEE00AF6
:10B07000F1EE10FA0BDD30EE600A0520C0EE080A92
:10B0800094ED000A20EE800AF7F7D0FF0AE070EE98
:10B09000C00A052080EE880AD4ED000A20EE200ABE
:10B0A000F7F7C4FF85A0F7F711FD00210520F6F79B
:10B0B00009FF83A0F7F70AFD0C20F8F775F80321C4
:10B0C0000020F6F7FFFE7FA0F7F700FD41460020C5
:10B0D000F6F7F8FE1020F8F767F897ED000A02205F
:10B0E000C0EE080A94ED000A20EE800AF7F79EFFF2
:10B0F00072A0F7F7EBFC24210120F8F74FF872A0BB
:10B10000F7F7E4FC0C20F8F74FF803210020F6F7DE
:10B11000D9FE6EA0F7F7DAFC41460020F6F7D2FE22
:10B120001020F8F741F86B4E042096ED000AF7F76F
:10B130007DFF69A0F7F7CAFC00210520F6F7C2FEE3
:10B140005FA0F7F7C3FC0C20F8F72EF803210020CE
:10B15000F6F7B8FE61A0F7F7B9FC41460020F6F714
:10B16000B1FE1020F8F720F895ED000A0220C0EE9D
:10B17000080A94ED000A20EE800AF7F757FF4FA067
:10B18000F7F7A4FC36210020F8F708F896ED000A3E
:10B19000534910EE100A884258DD38684FF08A4152
:10B1A000884202DB2868884250DA1C20F7F7FCFF4F
:10B1B0004C4D4D494D4C95ED000A10EE100A884259
:10B1C00003DA0320F7F732FF26E010EE100A4849B1
:10B1D000884203DA0220F7F729FF1DE010EE100A7B
:10B1E000A04203DA0120F7F721FF15E010EE100A64
:10B1F00040499FED411A884207DAC0EE010A032058
:10B20000B0EE600AF7F712FF06E0C0EE010A022076
:10B21000B0EE600AF7F70AFF1020F7F7C5FF042128
:10B220000320F6F74FFE2868A04207DA02B033A0E9
:10B23000BDEC028BBDE8F041F7F748BC02B030A08E
:10B24000BDEC028BBDE8F041F7F740BC392100208E
:10B25000F7F7A4FF4220F7F7A7FF2A480088F7F77F
:10B26000A9FF02B028A0BDEC028BBDE8F041F7F7C2
:10B270002DBC0000AC83FF1FBFAAB6FBCEC4B2E258
:10B28000CFDF00008483FF1FA1E600003083FF1F93
:10B29000A683FF1F3E0000003C000000A883FF1FA4
:10B2A000AA83FF1F44000000753A00009083FF1F2F
:10B2B0009483FF1F00F07F458083FF1F560000002E
:10B2C00055000000313A0000490000006275733AF1
:10B2D000000000003C83FF1F41000000323A0000E4
:10B2E000CDCCCC3E588DFF1F0000204100007A4499
:10B2F0000000C84200401C4600007A446DA6B80019
:10B30000A6B80000AE83FF1FC7EBD5FDC8B7BDD3FD
:10B31000C8EBBFAAB6FBCEC4B2E2CAD4D2C7000003
:10B320002DE9F04F2DED028B83B0FD48017800250B
:10B33000FC4EFD4CDFF8F49304290CD0017805296C
:10B340000DD0017806290ED001780A290FD0017896
:10B350000B2918D021E00570012060701DE00570F8
:10B360000220607019E005700A20607015E0057019
:10B37000307880F001003070ED494870FFF770FDC3
:10B38000FCF73AFD09E0057099F80E00012813D08A
:10B39000A07810B106F0EFF8A5701020F7F704FFC1
:10B3A000E44F3888F7F706FFE3490A78307802421D
:10B3B0004DD1097839B107E072B600210220FCF7BF
:10B3C0004BFC62B6E9E7E8B394ED0D0A4121BCEE0F
:10B3D000C00A10EE100AC0B2F7F7E0FED7A0F7F7E8
:10B3E00075FB94ED0E0A4121BCEEC00A10EE100A66
:10B3F000C0B2F7F7D3FED1A0F7F768FB4FF0FF0A12
:10B40000CDE9005A4F23682241215820F6F772FEF9
:10B41000CDE9005A4F238F2241217F20F6F76AFEA3
:10B42000DFF81CB39BED000A9FEDC61AB5EEC00A0B
:10B43000F1EE10FA71DD94ED0D0AC34910EE100A19
:10B44000884200E003E023DC84ED0D1A6BE094ED0C
:10B450000D0ADFEDBE0A30EEC00ABDEEC00A10EEE6
:10B46000100A94ED0E0A30EEC00ABDEEC00A10EECE
:10B47000106AC0B24121F7F791FEB5A0F7F726FB9D
:10B48000F0B24121F7F78AFEB1A0F7F71FFBB5E74D
:10B49000D4ED0E0A10EE900A884202DC84ED0E1AFA
:10B4A00041E09BED001AAB4911EE100A88420ADA1E
:10B4B0009FEDA91A30EE410A84ED0D0A30EEC10A63
:10B4C00084ED0E0A2FE09BED001AA44911EE100A3C
:10B4D000B0EE041A884216DADBED001A61EE812A1A
:10B4E000DFED9F1A82EEA12A30EE420A84ED0D0AAA
:10B4F0009BED000A20EE011A81EE210A30EEC00A0F
:10B5000084ED0E0A0FE030EE410A84ED0D0A30EEB4
:10B51000C10A84ED0E0A06E0FFE79FED920A84ED72
:10B520000D0A84ED0E1A9048DFF840821C2490ED3D
:10B53000000A8F4E10EE101A41450BDA3188CDE922
:10B540000014002390ED000A042219461846F8F76B
:10B55000A1F80AE03188CDE90014002390ED000A3B
:10B56000032219461846F8F795F83088CDE900040B
:10B57000002380A219465320F7F722FE7E487F4D14
:10B5800090ED000A10EE101A41450BDA2988CDE93A
:10B590000014002390ED000A04221B211846F8F73E
:10B5A00079F80AE02988CDE90014002390ED000A1B
:10B5B00003221B211846F8F76DF82888CDE900040E
:10B5C00000236FA21B215320F7F7FAFD9BED000A21
:10B5D00010EE100A40450BDA3888CDE9000400234C
:10B5E00004229BED000A37211846F8F753F823E0B0
:10B5F0009BED000A10EE100A404512DB9BED000A9D
:10B60000604910EE100A88420BDA3888CDE9000450
:10B61000002303229BED000A37211846F8F73AF879
:10B620000AE03888CDE90004002302229BED000ADD
:10B6300037211846F8F72EF83888CDE900040023A2
:10B6400051A237215320F7F7BBFD2888CDE9000A26
:10B650004F23682200216720F6F74CFD99F8080077
:10B66000DFED4A8A1024022838D0042857D03088C9
:10B67000CDE90004002346A219466C20F7F7A0FD8F
:10B680003088CDE9000443480023022290ED000AEF
:10B6900019468020F7F7FEFF3088CDE9000400232B
:10B6A0003DA211216C20F7F78BFD3088CDE9000415
:10B6B0003A480023022290ED000A11218020F7F77A
:10B6C000E9FF0CF051FB801E0C286DD2DFE800F082
:10B6D000FCFBFAF9F8F7F6F5F4F3F2F1B9F80A0021
:10B6E0009FED2F8A00EE100AB8EE400A20EE080AFD
:10B6F00010EE101A41456BDA3088CDE900040023C2
:10B7000028A201216B20F7F75BFD3088CDE900040A
:10B71000B9F80A0000EE100AB8EE400A45E096E0DB
:10B720006083FF1FA683FF1FB083FF1F44B7FF1F67
:10B7300074610220AC83FF1F3083FF1F3C000000B8
:10B740004083FF1F0000FE420000B042000058434B
:10B750003E00000000004041CDCC4C3E00001643AE
:10B76000000016430000D8423483FF1F0000204130
:10B77000A883FF1F560000003C83FF1FAA83FF1F02
:10B78000410000000000C84257000000CDCC4C3DF5
:10B79000442B00008883FF1F442D00008C83FF1F73
:10B7A0000AD7A33C3000000087E120EE080A0023FE
:10B7B000022201217420F7F76DFF30880023AFF2D9
:10B7C0004C02CDE9000401219420F7F7F9FC18E0C0
:10B7D00000EE100A3188CDE90014B8EE400A0023CB
:10B7E0000222012120EE080A6B20F7F753FF308870
:10B7F0000023AFF28002CDE9000401219420F7F785
:10B80000DFFC30880023AFF26402CDE9000411218F
:10B810006B20F7F7D5FC3088CDE9000499F80C00CF
:10B82000002300EE100A02221121B8EE400A742013
:10B8300020EE280AF7F72EFF30880023AFF2C0026F
:10B84000CDE9000411219420F7F7BAFC39E7B9F8E3
:10B850000A0000EE100AB8EE400A9FEDBB8A20EE07
:10B86000080A10EE101A414532DA30880023AFF290
:10B87000CC02CDE9000401216B20F7F7A1FC308850
:10B88000CDE90004B9F80A00002300EE100A0222F4
:10B890000121B8EE400A742020EE080AF7F7FAFEFC
:10B8A00030880023AFF23412CDE900040121942046
:10B8B0000BE0F8E0EDE0E2E0D7E08EE083E078E056
:10B8C0006DE062E057E04CE041E0F7F779FC18E00A
:10B8D00000EE100A3188CDE90014B8EE400A0023CA
:10B8E0000222012120EE080A6B20F7F7D3FE3088F0
:10B8F0000023AFF28012CDE9000401219420F7F774
:10B900005FFC30880023AFF26412CDE900041121FE
:10B910006B20F7F755FC3088CDE9000499F80C004E
:10B92000002300EE100A02221121B8EE400A742012
:10B9300020EE280AF7F7AEFE30880023AFF2C012DF
:10B94000CDE9000411219420F7F73AFCB9E62888E4
:10B95000CDE9000400237DA221217020F7F730FCFF
:10B96000B4E02888CDE9000400237AA221217020C8
:10B97000F7F726FCAAE02888CDE90004002377A287
:10B9800021216C20F7F71CFCA0E02888CDE90004F9
:10B99000002374A221216C20F7F712FC96E028887E
:10B9A000CDE90004002371A221216F20F7F708FCE4
:10B9B0008CE02888CDE9000400236EA221217520A7
:10B9C000F7F7FEFB82E02888CDE9000400236AA295
:10B9D00021217320F7F7F4FB78E099F800000A289A
:10B9E00021D22888CDE90004002364A221217120FE
:10B9F000F7F7E6FB2888CDE9000499F8000000235A
:10BA000000EE100A1A462121B8EE400A8620F7F708
:10BA100041FE2888CDE90004002351A221218F2076
:10BA2000F7F7CEFB52E02888CDE90004002353A2AB
:10BA300021216C20F7F7C4FB2888CDE9000499F890
:10BA40000000002300EE100A1A462121B8EE400A39
:10BA50008120F7F71FFE2888CDE90004002340A2CB
:10BA600021219320F7F7ACFB30E02888CDE90004D2
:10BA7000002343A221217520F7F7A2FB26E02888A6
:10BA8000CDE9000400233FA221217420F7F798FBA1
:10BA90001CE02888CDE9000400233BA22121752069
:10BAA000F7F78EFB12E02888CDE90004002337A2C7
:10BAB00021217520F7F784FB08E02888CDE90004F0
:10BAC000002333A221216C20F7F77AFB3888CDE9D7
:10BAD000000431480023012290ED000A31216D203D
:10BAE000F7F7D8FD3888CDE9000400232BA23121D7
:10BAF0008E20F7F765FB2A48007888B1012819D015
:10BB0000022808D13888CDE90004002325A241216C
:10BB10007F20F7F755FB03B0BDEC028BBDE8F08F3B
:10BB20003888CDE9000400231AA240218220F7F7CB
:10BB300047FBF0E73888CDE9000400231AA2412131
:10BB40007F20F7F73DFBE6E7CDCCCC3C51433556A3
:10BB500000000000514339560000000051433132CB
:10BB60005600000051433230560000005143332E3E
:10BB70003000000053435000464350005044000042
:10BB80005050530044435000564152004156530018
:10BB90002D2D2D2D2D2D2D008483FF1FA1E60000BE
:10BBA0002083FF1F434332004343310002490020FA
:10BBB00008700249487070476083FF1FB083FF1F01
:10BBC0002DE9F04F2DED108B83B0F6480178F64D3E
:10BBD000F64C4FF0000A04290CD0017805290ED04C
:10BBE0000178062910D001780A2912D001780B2992
:10BBF0001CD027E080F800A00220607022E080F8CE
:10BC000000A084F801A01DE080F800A00A20607068
:10BC100018E080F800A0287880F001002870E4493E
:10BC20004870FFF71DF9FCF7E7F80BE080F800A07B
:10BC3000E048807B012814D0A07818B105F09BFC67
:10BC400084F802A01020F7F7AFFADB4E3088F7F740
:10BC5000B1FADA490A78287802424AD1097839B12A
:10BC600007E000210220FBF7F7FFF9F7C9FFE9E73A
:10BC7000F0B394ED0D0AB0EE008A422130EE480A8E
:10BC8000BCEEC00A10EE100AC0B2F7F787FACCA0DB
:10BC9000F6F71CFF94ED0E0A422130EE480ABCEE86
:10BCA000C00A10EE100AC0B2F7F778FAC4A0F6F78F
:10BCB0000DFF4FF0FF0B4F23682242215820CDE9A2
:10BCC00000ABF6F717FADFF8FC8298ED000A9FED5B
:10BCD000BE1AB5EEC00AF1EE10FA72DD94ED0D0A4F
:10BCE000BA4810EE101A814226DC84ED0D1A6EE07F
:10BCF000FFE7D4ED0D0A9FEDB60A70EE600AFDEE87
:10BD0000E00A10EE900AD4ED0E0A30EE600ABDEEA5
:10BD1000C00A10EE105A801EC0B24221F7F73EFA58
:10BD2000ACA0F6F7D3FEAD1EE8B24221F7F736FA23
:10BD3000A8A0F6F7CBFEBCE7D4ED0E0A10EE901AE1
:10BD4000814202DC84ED0E1A41E098ED001AA2490E
:10BD500011EE100A88420ADA9FEDA01A30EE410A6D
:10BD600084ED0D0A30EEC10A84ED0E0A2FE098ED45
:10BD7000001A9B4911EE100AB0EE041A884216DA36
:10BD8000D8ED001A61EE812ADFED961A82EEA12A23
:10BD900030EE420A84ED0D0A98ED000A20EE011AF9
:10BDA00081EE210A30EEC00A84ED0E0A0FE030EE7B
:10BDB000410A84ED0D0A30EEC10A84ED0E0A06E058
:10BDC000FFE79FED890A84ED0D0A84ED0E1A87487E
:10BDD000874C1C2790ED000A864D10EE101AA142E8
:10BDE0000BDA2988CDE90017002390ED000A042220
:10BDF00019461846F7F74EFC0AE02988CDE90017E6
:10BE0000002390ED000A032219461846F7F742FC7A
:10BE10002888CDE90007002377A219465320F7F7B9
:10BE2000CFF97648DFF8D89190ED000A10EE101A9D
:10BE3000A1420CDAB9F80010CDE90017002390ED0B
:10BE4000000A04221B211846F7F724FC0BE0B9F87E
:10BE50000010CDE90017002390ED000A03221B21FA
:10BE60001846F7F717FCB9F80000CDE900070023E2
:10BE700064A21B215320F7F7A3F998ED000A40466E
:10BE800010EE102A21469FED60CB9FED61BB9FED28
:10BE900062DBDFF88C819FED63EB9FED64FB9FED30
:10BEA000659B9FED66AB9FED678B10248A420BDA92
:10BEB0003188CDE90017002390ED000A04223721D4
:10BEC0001846F7F7E7FB23E090ED000A10EE102A82
:10BED0008A4212DB90ED000A5C4A10EE101A914281
:10BEE0000BDA3188CDE90017002390ED000A032218
:10BEF00037211846F7F7CEFB0AE03188CDE9001765
:10BF0000002390ED000A022237211846F7F7C2FB02
:10BF10003088CDE9000700234DA237215320F7F7E1
:10BF20004FF9B9F80000CDE9000B4F23682200213A
:10BF30006720F6F7DFF898ED000B53EC1B2B51EC64
:10BF4000100BF4F70DFC09D22888CDE9000400237A
:10BF500040A219467220F7F733F908E02888CDE9A6
:10BF6000000400233DA219467820F7F729F998ED3F
:10BF7000000B53EC192B51EC100BF4F7F1FB70D2C2
:10BF800098ED000B51EC100BF4F71AFC00EE100AC0
:10BF90002888CDE90004002304220E216B20F7F746
:10BFA00079FB61E16083FF1FA683FF1FB083FF1F42
:10BFB0007461022044B7FF1FAC83FF1F3083FF1F53
:10BFC0003C0000004083FF1F0000FE420000B04222
:10BFD000000058433E00000000004041CDCC4C3EE4
:10BFE00000001643000016430000D8423483FF1FB0
:10BFF00000002041A883FF1F560000003C83FF1F64
:10C00000AA83FF1F41000000000000000088C34019
:10C0100000000000006AF8400000000080842E410B
:10C020005883FF1F9A9999999999B93F0000000088
:10C030000000F03F0000000000002440000000006D
:10C04000000059400000000000408F400000C8423E
:10C05000570000006D41683A0000000041683A0056
:10C06000FFE798ED000B53EC192B51EC100BF4F794
:10C070008FFB1AD898ED000B53EC1A2B51EC100BD8
:10C08000F4F76EFB11D298ED000B51EC100BF4F7A6
:10C0900097FB00EE100A2888CDE900040023032254
:10C0A0000E216B20F7F7F6FADEE098ED000B53EC6B
:10C0B0001A2B51EC100BF4F76BFB1AD898ED000B10
:10C0C00053EC182B51EC100BF4F74AFB11D298EDFE
:10C0D000000B51EC100BF4F773FB00EE100A2888EC
:10C0E000CDE90004002302220E216B20F7F7D2FADB
:10C0F000BAE098ED000B53EC182B51EC100BF4F751
:10C1000047FB1AD898ED000B53EC1C2B51EC100B8D
:10C11000F4F726FB11D298ED000B51EC100BF4F75D
:10C120004FFB00EE100A2888CDE90004002301220D
:10C130000E216B20F7F7AEFA96E098ED000B53EC6A
:10C140001C2B51EC100BF4F723FB1AD898ED000BC5
:10C1500053EC1B2B51EC100BF4F702FB11D298EDB2
:10C16000000B51EC100BF4F72BFB00EE100A2888A3
:10C17000CDE9000400231A460E216B20F7F78AFA56
:10C1800072E098ED000B53EC1B2B51EC100BF4F705
:10C19000FFFA22D898ED000B53EC1D2B51EC100B3D
:10C1A000F4F7DEFA19D2B0EE480AF0EE680A53EC62
:10C1B000102B98ED000B51EC100BF4F728FAF4F764
:10C1C000FFFA00EE100A2888CDE9000400230222BD
:10C1D0000E216B20F7F75EFA46E098ED000B53EC6A
:10C1E0001D2B51EC100BF4F7D3FA24D89FEDE20B82
:10C1F00053EC102B98ED000B51EC100BF4F7B0FA48
:10C2000019D2B0EE480AF0EE680A53EC102B98ED04
:10C21000000B51EC100BF4F7FAF9F4F7D1FA00EE39
:10C22000100A2888CDE90004002301220E216B208A
:10C23000F7F730FA18E0B0EE480AF0EE680A53EC6F
:10C24000102B98ED000B51EC100BF4F7E0F9F4F71C
:10C25000B7FA00EE100A2888CDE9000400231A4638
:10C260000E216B20F7F716FAC54D53EC1F2B95EDF9
:10C27000000B51EC100BF4F773FA0AD2B9F8000076
:10C28000CDE900040023BFA21B217220F6F798FF1E
:10C2900009E0B9F80000CDE900040023BBA21B218E
:10C2A0007820F6F78DFF9FEDBABB95ED000B53ECB0
:10C2B0001B2B51EC100BF4F753FA16D295ED000B33
:10C2C00053EC182B51EC100BF4F72FF9F4F778FA24
:10C2D00000EE100AB9F80000CDE9000400230422A2
:10C2E00029216B20F7F7D6F9F7E095ED000B53EC19
:10C2F0001B2B51EC100BF4F74BFA1FD895ED000BEC
:10C3000053EC1E2B51EC100BF4F72AFA16D295EDD4
:10C31000000B53EC182B51EC100BF4F706F9F4F763
:10C320004FFA00EE100AB9F80000CDE9000400232E
:10C33000032229216B20F7F7ADF9CEE095ED000B34
:10C3400053EC1E2B51EC100BF4F722FA1FD895ED8D
:10C35000000B53EC1F2B51EC100BF4F701FA16D223
:10C3600095ED000B53EC182B51EC100BF4F7DDF8A6
:10C37000F4F726FA00EE100AB9F80000CDE900043F
:10C380000023022229216B20F7F784F9A5E095ED1F
:10C39000000B53EC1F2B51EC100BF4F7F9F91BD8E1
:10C3A00095ED000B53EC192B51EC100BF4F7D8F969
:10C3B00012D295ED000B51EC100BF4F701FA00EEE0
:10C3C000100AB9F80000CDE9000400230422292155
:10C3D0006B20F7F75FF980E095ED000B53EC192B1C
:10C3E00051EC100BF4F7D4F91BD895ED000B53EC7E
:10C3F0001A2B51EC100BF4F7B3F912D295ED000B98
:10C4000051EC100BF4F7DCF900EE100AB9F800005B
:10C41000CDE900040023032229216B20F7F73AF924
:10C420005BE095ED000B53EC1A2B51EC100BF4F77D
:10C43000AFF91BD895ED000B53EC182B51EC100BFA
:10C44000F4F78EF912D295ED000B51EC100BF4F7C6
:10C45000B7F900EE100AB9F80000CDE90004002396
:10C46000022229216B20F7F715F936E095ED000B34
:10C4700053EC182B51EC100BF4F78AF91BD895EDFF
:10C48000000B53EC1C2B51EC100BF4F769F912D292
:10C4900095ED000B51EC100BF4F792F900EE100A39
:10C4A000B9F80000CDE900040023012229216B2006
:10C4B000F7F7F0F811E095ED000B51EC100BF4F7E5
:10C4C0007FF900EE100AB9F80000CDE9000400235E
:10C4D0001A4629216B20F7F7DDF830880C25CDE9C5
:10C4E00000A02D4802950223027837216920F7F732
:10C4F00051F93088CDE90005002328A238217720A2
:10C50000F6F75EFE30880295CDE900A024480223AC
:10C51000372102787D20F7F73DF93088CDE9000515
:10C5200000231EA238218B20F6F74AFE30880295A0
:10C53000CDE900A01B480223372102789120F7F7AC
:10C5400029F93088CDE90004174800231A4690EDF8
:10C55000000A42217C20F7F79DF83088CDE90004DD
:10C56000002312A242218E20F6F72AFE03B0BDEC72
:10C57000108BBDE8F08F000000000000D012634176
:10C580005083FF1F6D57683A0000000057683A005B
:10C590007B14AE47E17A843FF58CFF1F3A00000020
:10C5A000F68CFF1FF78CFF1F8483FF1FA1E600009E
:10C5B0002DE9F04F2DED028B83B0FE480178002568
:10C5C000FD4EFE4C04290CD0017805290CD00178D1
:10C5D00006290DD001780A290ED001780B2917D031
:10C5E00020E0057065701DE005700120607019E0A5
:10C5F00005700A20607015E00570307880F0010049
:10C600003070EF494870FEF72BFCFBF7F5FB09E0B3
:10C610000570EC48807B012813D0A07810B104F09D
:10C62000AAFFA5701020F6F7BFFDE74D2888F6F7A2
:10C63000C1FDE6490A783078024238D1097839B12B
:10C6400007E000210220FBF707FBF9F7D9FAE9E739
:10C6500068B394ED0F0A0021BCEEC00A10EE100A78
:10C66000C0B2F6F79BFDDAA0F6F730FA94ED100AA7
:10C670000021BCEEC00A10EE100AC0B2F6F78EFD23
:10C68000D3A0F6F723FAD34890ED000AB5EEC00A1E
:10C69000F1EE10FA71DD94ED0F0ACF4910EE102A79
:10C6A0009FEDCE1A8A4223DC84ED0F1A6DE094EDE3
:10C6B0000F0ADFEDCB0A30EEC00ABDEEC00A10EE65
:10C6C000100A94ED100A30EEC00ABDEEC00A10EE5A
:10C6D000106AC0B20021F6F761FDC2A0F6F7F6F9C4
:10C6E000F0B20021F6F75AFDBEA0F6F7EFF9CAE75F
:10C6F000D4ED100A10EE902A8A4202DC84ED101A62
:10C7000043E090ED001AB84A11EE101A91420ADA8D
:10C710009FEDB61A30EE410A84ED0F0A30EEC10AE1
:10C7200084ED100A31E090ED001AB14A11EE101AB2
:10C73000B0EE041A914216DAD0ED001A61EE812AA9
:10C74000DFEDAC1A82EEA12A30EE420A84ED0F0A28
:10C7500090ED000A20EE011A81EE210A30EEC00AA7
:10C7600084ED100A11E030EE410A84ED0F0A30EE3C
:10C77000C10A84ED100A08E0FFE79FED9F0A84EDEF
:10C780000F0A9FED9E0A84ED100A10242888CDE937
:10C7900000049B4800231A4690ED000A19466B20BE
:10C7A000F6F778FF2888CDE90004002395A2194602
:10C7B0007D20F6F705FD9448944EDFF854B290EDD5
:10C7C000000A10EE101AB1420CDABBF80010CDE9E5
:10C7D0000014002390ED000A032219461846F6F7CC
:10C7E00059FF0BE0BBF80010CDE90014002390EDD9
:10C7F000000A022219461846F6F74CFFBBF8000063
:10C80000CDE90004002383A219462920F6F7D8FCBD
:10C810008148DFF808A290ED000A10EE101AB1422C
:10C820000CDABAF80010CDE90014002390ED000AEC
:10C83000032219463520F6F72DFF0BE0BAF8001059
:10C84000CDE90014002390ED000A0222194635209C
:10C85000F6F720FFBAF80000CDE90004002370A22B
:10C8600019465E20F6F7ACFCFF20BAF80010CDE9BF
:10C87000001013239F2212210020F5F73BFC4FF0FC
:10C880004209BBF80000CDE90009002365A2172189
:10C890001846F6F795FC654890ED000A10EE100A70
:10C8A000B0420ADABBF80000CDE9000400230222FE
:10C8B00018211920F6F7EEFE09E0BBF80000CDE9DB
:10C8C00000040023012218211920F6F7E3FEBBF82B
:10C8D0000000CDE9000400234EA218213920F6F70C
:10C8E0006FFC534890ED000A10EE100AB0420ADACD
:10C8F000BBF80000CDE900040023022218214520E6
:10C90000F6F7C8FE09E0BBF80000CDE900040023FB
:10C91000012218214520F6F7BDFEBBF80000CDE945
:10C92000000400233EA218216520F6F749FC414887
:10C93000364F4FF0D47890ED000A7F4210EE100A87
:10C94000B0420ADABBF80000CDE90004002302225D
:10C9500018217120F6F79EFE19E010EE100A3844F7
:10C9600040450AD2BBF80000CDE9000400230122B3
:10C9700018217120F6F78EFE09E0BBF80000CDE922
:10C98000000400231A4618217120F6F783FEBBF835
:10C990000000CDE90004002327A218219120F6F71A
:10C9A0000FFCBAF80000CDE90009002323A22B21D7
:10C9B000184647E06083FF1FA683FF1FB083FF1F59
:10C9C0007461022044B7FF1FAC83FF1F3083FF1F39
:10C9D0003C0000004083FF1F0000F44200001F43A2
:10C9E00000808C433E00000000004041CDCC4C3E16
:10C9F000000016430000164300000F4300002243CE
:10CA00008483FF1FA1E600003483FF1F0000204144
:10CA1000A883FF1F560000003C83FF1FAA83FF1F4F
:10CA200041000000D7EEB8DF00000000288DFF1F96
:10CA30002C8DFF1F308DFF1F57000000C6BDBEF9B3
:10CA400000000000F6F7BCFBA04890ED000A10EED5
:10CA5000100AB0420ADABAF80000CDE90004002357
:10CA600002222C211920F6F715FE09E0BAF8000081
:10CA7000CDE90004002301222C211920F6F70AFE3B
:10CA8000BAF800000023AFF27402CDE900042C21B3
:10CA90003920F6F795FB8E4890ED000A10EE100A4B
:10CAA000B0420ADABAF80000CDE9000400230222FD
:10CAB0002C214520F6F7EEFD09E0BAF80000CDE99B
:10CAC0000004002301222C214520F6F7E3FDBAF8EB
:10CAD00000000023AFF2B802CDE900042C2165204C
:10CAE000F6F76EFB7B4890ED000A10EE100AB0429C
:10CAF0000ADABAF80000CDE90004002302222C2152
:10CB00007120F6F7C7FD19E010EE100A38444045D1
:10CB10000AD2BAF80000CDE90004002301222C213A
:10CB20007120F6F7B7FD09E0BAF80000CDE900047E
:10CB300000231A462C217120F6F7ACFDBAF800004C
:10CB40000023AFF20C12CDE900042C219120F6F75E
:10CB500037FB2888CDE9000900235FA23F21184652
:10CB6000F6F72EFB5E48DFF87C9190ED000A10EEA0
:10CB7000100A9FED5D8A48450BD12888CDE9000455
:10CB800000230222B0EE480A40211920F6F782FD68
:10CB900016E010EE100AB04209DA2888CDE9000448
:10CBA0000023022240211920F6F774FD08E02888AE
:10CBB000CDE900040023012240211920F6F76AFD87
:10CBC00028880023AFF2B412CDE9000440213920B7
:10CBD000F6F7F6FA454890ED000A10EE100A4845BF
:10CBE0000BD12888CDE9000400230222B0EE480AC8
:10CBF00040214520F6F74EFD16E010EE100AB04237
:10CC000009DA2888CDE900040023022240214520CA
:10CC1000F6F740FD08E02888CDE900040023012252
:10CC200040214520F6F736FD28880023AFF2102278
:10CC3000CDE9000440216520F6F7C2FA2C4890EDBA
:10CC4000000A10EE100A48450BD12888CDE90004EF
:10CC500000230222B0EE480A40217120F6F71AFDA7
:10CC600025E010EE100AB04209DA2888CDE9000468
:10CC70000023022240217120F6F70CFD17E010EE90
:10CC8000100A3844404509D22888CDE90004002321
:10CC9000012240217120F6F7FDFC08E02888CDE94B
:10CCA000000400231A4640217120F6F7F3FC28887F
:10CCB0000023AFF27C22CDE9000440219120F6F759
:10CCC0007FFA03B0BDEC028BBDE8F08F348DFF1FFF
:10CCD000388DFF1F3C8DFF1FD7EEB5CD0000000043
:10CCE000408DFF1F00007A4400000000448DFF1FAC
:10CCF000488DFF1FF0EE401AB0EE410AF4EEE01A44
:10CD0000F1EE10FA07DDF4EEC01AF1EE10FA01DDD3
:10CD1000B0EE610A7047F4EEC00AF1EE10FAF9DDE8
:10CD2000B0EE600A704710B5AFF3008010BD000090
:10CD30002DE9FC4100F05CF81020F6F735FA0024EC
:10CD4000284D274E05F59A773088F6F733FA2007F5
:10CD5000010E0020F6F722FAE87A844212D102216D
:10CD60000020F5F7AFF80C20F6F71EFA1E480088F1
:10CD7000F6F720FA1DA0F5F7A9FE6FF001010020DB
:10CD8000F5F7A0F81020F6F70FFA287B204400EB07
:10CD9000400101EB001057F82000F5F7E5FA641C9C
:10CDA000E4B2052CD0D3FF243088CDE900049E22C4
:10CDB0004F2300211046F5F79DF93088CDE9000496
:10CDC000E87A297B9F22084400EB400101EBC00375
:10CDD0009B1C00219D20F5F78DF9BDE8FC8100002A
:10CDE000AA83FF1FB083FF1FA883FF1F3E00000020
:10CDF00070B5324C2578324A0023042DD07A117B4D
:10CE00000FD026780325052E19D02678062E12D1AC
:10CE10000844082850D2DFE800F01F21244144478D
:10CE20004A4D042802D2401CD07203E0032903D0EB
:10CE3000491C1173237070BDD3721373FAE710B1DC
:10CE4000401ED07202E019B1491E1173237070BDEB
:10CE50000420D0721573F9E755702DE0162050703C
:10CE60002AE01848807B022815D1907898B9164896
:10CE700090ED000A10EE100AB0F17C5F0BDD134854
:10CE80000168156B491BB1F5487F15D90821117050
:10CE90000068106310E0072050700DE00E20507005
:10CEA0000AE01020507007E00D20507004E00F20C1
:10CEB000507001E011205070237070BD6083FF1F1F
:10CEC000B083FF1F44B7FF1F4083FF1F7C83FF1FFA
:10CED00003490020087003490A2048707047000089
:10CEE0006083FF1FB083FF1F10B500F001F810BD75
:10CEF00010B5064C2068002804D14FF4927104A0AC
:10CF0000F8F78CFB2068BDE8104000476891FF1FD0
:10CF10002E2E5C2E2E5C2E2E5C2E2E5C2E2E5C6415
:10CF200072697665725C7372635C6863333266340F
:10CF300036305F6578696E745F6E6D695F737769AF
:10CF40002E6300002DE9FC41FA480178FA4D0629CC
:10CF500005D1002101700120687703F0CFF810207F
:10CF6000F6F722F900210846F6F718F9F348008889
:10CF7000F6F720F96868F24C00287CD0F1A0F5F7AC
:10CF8000F3F90C20F6F710F92088F6F713F91421BD
:10CF90000020F6F703F9EFA0F5F798FD08212868BF
:10CFA000F5F710FC20210020F6F7F8F8E9A0F5F7D6
:10CFB0008DFD08216868F5F705FC2C210020F6F7A7
:10CFC000EDF8E4A0F5F782FD0821A868F5F7FAFB73
:10CFD00038210020F6F7E2F8DEA0F5F777FD08210A
:10CFE000E868F5F7EFFB44210020F6F7D7F8D9A061
:10CFF000F5F76CFD08212869F5F7E4FBD64F388872
:10D00000F6F7D8F814215220F6F7C8F868680C240F
:10D01000C0F3C2604FF4784603286ED0042871D064
:10D02000CDE900640023CDA214215220F6F7C8F800
:10D0300014218120F6F7B2F895F8200038B1C8A085
:10D04000F5F744FD95F820000021F6F761F820215E
:10D050005220F6F7A3F82869410757D000F00700DF
:10D06000012857D0022859D003285BD00023202163
:10D07000BAA2522000E03CE1CDE90064F6F7A0F846
:10D080002C215220F6F78AF82869410A89074DD0E9
:10D09000C0F3412101294DD002294FD06FEA502021
:10D0A00080074FD0CDE900640023ACA22C21522090
:10D0B000F6F786F800210820F4F704FF287CC0F377
:10D0C0004110012842D0022844D0CDE90064002359
:10D0D000A2A22C217F20F6F773F838215220F6F710
:10D0E0005DF82869C0F34330092857D2DFE800F023
:10D0F00056363A3E42464A4E52009AA0F5F734F967
:10D1000096E7FFE799A0F5F72FF991E799A0F5F7D2
:10D11000DDFCB5E799A0F5F7D9FCB1E79AA0F5F7E2
:10D12000D5FCADE79BA0F5F7D1FCA9E79CA0F5F7EE
:10D13000CDFCBFE79BA0F5F7C9FCBBE79AA0F5F7CC
:10D14000C5FCB7E799A0F5F7C1FCB3E798A0F5F7E0
:10D15000BDFCC2E797A0F5F7B9FCBEE796A0F5F7CE
:10D16000B5FC23E095A0F5F7B1FC1FE094A0F5F71E
:10D17000ADFC1BE093A0F5F7A9FC17E092A0F5F732
:10D18000A5FC13E091A0F5F7A1FC0FE090A0F5F746
:10D190009DFC0BE08EA0F5F799FC07E0CDE900645B
:10D1A00000236EA238215320F6F70AF8286980037D
:10D1B00009D53888CDE90004002386A238217620DD
:10D1C000F5F7FEFF07E0CDE90064002381A23821D6
:10D1D0007620F5F7F5FF44215220F5F7DFFFA88808
:10D1E00042F6013280B2811A90425FD01DDC41F2DA
:10D1F000EF72A0EB020190424ED00BDCB0F57C7FC9
:10D2000045D0A0F5A060AC385FD0A0F550602538BF
:10D210001FD128E0E22935D0A1F52061EA392CD0D0
:10D22000A1F580613E3914D13BE0B1F5667F5BD05A
:10D2300009DC1C2953D0B1F5257F19D0A1F5407127
:10D24000863906D146E0A1F5C0611B3933D04029AB
:10D2500036D061A0F5F73AFCA888BDE8FC4180B261
:10D260000421F5F7AFBABDE8FC415DA0F5F72EBC8F
:10D27000BDE8FC415CA0F5F729BCBDE8FC415CA021
:10D28000F5F724BCBDE8FC415BA0F5F71FBCBDE889
:10D29000FC415BA0F5F71ABCBDE8FC4159A0F5F7CD
:10D2A00015BCBDE8FC4159A0F5F710BCBDE8FC4138
:10D2B00058A0F5F70BBCBDE8FC4157A0F5F706BC3C
:10D2C000BDE8FC4157A0F5F701BCBDE8FC4157A003
:10D2D000F5F7FCBBBDE8FC4156A0F5F7F7BBBDE890
:10D2E000FC4157A0F5F7F2BBBDE8FC4156A0F5F7AD
:10D2F000EDBB14A0F5F738F82088F5F75BFF687FE1
:10D3000078B128210020F5F749FF51A0F5F72CF856
:10D310003A210020F5F742FFBDE8FC4151A0F5F7A6
:10D3200023B832212320F5F739FFBDE8FC4152A094
:10D33000F5F71AB86083FF1F24CD0120AA83FF1FD1
:10D34000A883FF1F452D4D61726B6572B2E2CAD48E
:10D350000000000030780000AC83FF1F45525200EF
:10D360005442540050617373697665004163746977
:10D3700076650000555342322E300000555342333B
:10D380002E3247656E310000555342332E324765C9
:10D390006E3200005553423447656E330000000082
:10D3A0003230560033305600343056003530560097
:10D3B00033410000354100007E316D007E326D004A
:10D3C0007E336D007E346D007E356D007E366D00DF
:10D3D0007E376D0045505200556E6B6E6F770000C2
:10D3E00048756177656900005669766F0000000036
:10D3F0004F50504F00000000476F6F676C65000092
:10D40000485000004C656E6F766F00005869616F80
:10D410004D6900005A4D4900536F7574684368693F
:10D4200070000000596943686F6E67004170706C4E
:10D4300065000000496E6A6F696E69630000000054
:10D440004C696E746573000048796E6574656B0095
:10D45000CEB4B6C1C8A1B5BD456D61726B6572D061
:10D46000C5CFA200C7EBB0B427C8B7C8CF27BCFC54
:10D47000D6D8CAD400000000B0B427C8B7C8CF2798
:10D48000BCFCBDF8D0D0B2E2CAD400002DE9FC410A
:10D4900001F050FF1020F5F787FE42480088F5F7AD
:10D4A00089FE00210846F5F779FE3FA0F4F75CFFFE
:10D4B0000024DFF804813F4FA8F254453888F5F77F
:10D4C00079FE601C06460007010E0020F5F766FE97
:10D4D000687C844212D101210020F4F7F3FC0C2077
:10D4E000F5F762FE35480088F5F764FE34A0F5F7DD
:10D4F000EDFA4FF0FF310020F4F7E4FC1020F5F7CF
:10D5000053FE04EBC40058F83000F4F72DFF34B19B
:10D51000012C0ED0022C14D0032C23D11AE0A87CAD
:10D5200018B128A0F4F720FF1CE028A0F4F71CFF96
:10D5300018E00021E87CF5F7EBFD26A0F5F7C6FA28
:10D5400010E0022095ED120AF5F770FD21A0F5F725
:10D55000BDFA07E0022095ED130AF5F767FD1EA05E
:10D56000F5F7B4FAF4B2042CA8D3FF243888CDE937
:10D5700000049E224F2300211046F4F7BBFD38889B
:10D58000CDE90004687C9F2200EB800101EBC00024
:10D59000012101EB400300219D20F4F7ABFDBDE824
:10D5A000FC810000AC83FF1F5044D3D5C6ADC9E851
:10D5B000D6C30000AA83FF1F0488FF1FA883FF1F94
:10D5C0003E0000005050532F415653004649582FFB
:10D5D0004550520056000000410000002DE9F04780
:10D5E0000024FB4FDFF8EC83F888F978421802EB4F
:10D5F000420208EB82025288C2F30235DFF8D8A358
:10D600009AF800C0F54AA1461288561ED31FBCF1F5
:10D61000040F05D09AF800C0BCF1050F23D03BE001
:10D62000DFF8ACC3072A9CF803C00CF1010C0CF026
:10D63000FF0C07D2B14202DA87F803C010E087F886
:10D6400003900DE0062902D287F803C008E0984253
:10D6500004D187F80390A7F8069001E0401CF880F9
:10D660008AF8009018E0DFF868C3072A9CF803C026
:10D67000ACF1010C0CF0FF0C05D211B187F803C01E
:10D6800008E0FE7006E011B187F803C002E060B365
:10D69000401EF8808AF800900C20F5F785FD0021E7
:10D6A0000846F5F77BFDDFF83893B9F80000F5F789
:10D6B00081FDCCA0F5F70AFAF878F988084404212E
:10D6C000F5F726FD00210A20F4F7FCFBF888F9782D
:10D6D000084400EB400008EB80004088C00508D5F6
:10D6E000C1480088F5F766FD07E00620F870FB806A
:10D6F000D0E7BE480088F5F75DFDF888F978084462
:10D7000000EB400008EB80004088C10B71D000F0B6
:10D710001F001F285DD2DFE800F05C1014181C20E9
:10D7200024282C3034383C4044484C50545C5C5CD9
:10D730005C5C5C5C5C5C5C5C5800ADA0F5F7C6F9B9
:10D7400038E1AEA0F5F7C2F934E1AEA0F5F7BEF9C5
:10D7500030E1AFA0F5F7BAF92CE1ABA0F5F7B6F9D7
:10D7600028E1AEA0F5F7B2F924E1ADA0F5F7AEF9E6
:10D7700020E1AEA0F5F7AAF91CE1B0A0F5F7A6F9F3
:10D7800018E1B2A0F5F7A2F914E1B4A0F5F79EF9FB
:10D7900010E1B6A0F5F79AF90CE1B7A0F5F796F904
:10D7A00008E1B9A0F5F792F904E1BBA0F5F78EF90D
:10D7B00000E1BCA0F5F78AF9FCE0BDA0F5F786F919
:10D7C000F8E0BEA0F5F782F9F4E0C0A0F5F77EF925
:10D7D000F0E0C2A0F5F77AF9F888F978084400EB90
:10D7E000400008EB800004214088F4F7EBFFE1E003
:10D7F000FFE76DB100F01F00102870D2DFE800F0E5
:10D80000C08C9094989CA0A4A8ACB0B4B8C0C0BC84
:10D8100000F01F00192870D2DFE800F06F0D11151D
:10D82000191D2125292D3135393D4145494D515588
:10D83000595D62666A00AAA0F5F748F9AEE0AAA0B1
:10D84000F5F744F9AAE0AAA0F5F740F9A6E0AAA0E6
:10D85000F5F73CF9A2E0AAA0F5F738F99EE0AAA0F6
:10D86000F5F734F99AE0AAA0F5F730F996E0ABA005
:10D87000F5F72CF992E0ADA0F5F728F98EE0ADA010
:10D88000F5F724F98AE0ADA0F5F720F986E0AEA01F
:10D89000F5F71CF982E0AEA0F5F718F97EE0AFA02D
:10D8A000F5F714F97AE0B0A0F5F710F976E0B2A038
:10D8B000F5F70CF972E0B3A0F5F708F96EE0B5A042
:10D8C000F5F704F96AE0B6A0F5F700F966E0B6A04E
:10D8D000F5F7FCF862E0B8A0F5F7F8F85EE04FE085
:10D8E000BAA0F5F7F3F859E0BCA0F5F7EFF855E06A
:10D8F000BEA0F5F7EBF851E0FFE778A0F5F7E6F802
:10D90000F888F978084400EB400008EB8000042117
:10D910004088F4F757FF41E066A0F5F7D7F83DE0FF
:10D92000B6A0F5F7D3F839E0B6A0F5F7CFF835E0B3
:10D9300063A0F5F7CBF831E0B4A0F5F7C7F82DE018
:10D94000B6A0F5F7C3F829E0B6A0F5F7BFF825E0D3
:10D95000B9A0F5F7BBF821E0BAA0F5F7B7F81DE0DC
:10D96000BBA0F5F7B3F819E0BCA0F5F7AFF815E0E8
:10D970009FA0F5F7ABF811E0BBA0F5F7A7F80DE015
:10D9800056A0F5F7A3F8F888F978084400EB4000B2
:10D9900008EB800004214088F4F714FFF888F97838
:10D9A000084400EB400018F82000E02802D2B2A0A2
:10D9B000F5F78CF84DB1012D08D00021B04AFE7862
:10D9C000AE481388FA883244CDE15BE169E100009A
:10D9D0006C8DFF1FF0B9FF1F6083FF1F7083FF1F57
:10D9E000AA83FF1F4E3A0000AC83FF1FA883FF1FCE
:10D9F0005352435F4341505F455800005374617474
:10DA0000757300004765745F4261745F4341500065
:10DA10004765745F4261745F535441004765745FAA
:10DA20004D616E75665F496E666F00005365637584
:10DA3000726974795F526571000000005365637507
:10DA4000726974795F526573700000004669726D87
:10DA50005F5570645F526571000000004669726D29
:10DA60005F5570645F526573700000005050535FE3
:10DA70005374617475730000436F756E7472795FCF
:10DA8000496E666F00000000436F756E7472795FB7
:10DA9000436F64657300000053696E6B5F434150D0
:10DAA0005F45580045585F436F6E74726F6C00009D
:10DAB0004550525F5352435F434150004550525FBF
:10DAC00053696E6B5F4341500000000056656E6401
:10DAD0005F446566696E5F4558000000307800005D
:10DAE000476F6F6443524300476F746F4D696E0018
:10DAF000416363657074000052656A656374000079
:10DB000050696E670000000050535F524459000096
:10DB10004765745F5352435F436170004765745FAC
:10DB200053696E6B5F4361700000000044525F53A5
:10DB30007761700050525F537761700056434F4ECB
:10DB40004E5F5377617000005761697400000000F8
:10DB5000536F66745F5265736574000044415441AD
:10DB60005F52657365740000444154415F526573B0
:10DB700065745F4F4B0000004E6F745F537570709B
:10DB80006F7274004765745F5352435F4361705F07
:10DB9000455800004765745F5374617475730000E5
:10DBA00046525F53776170004765745F5050535F12
:10DBB00053746174757300004765745F436F756ECD
:10DBC0007472795F436F6465000000004765745F9D
:10DBD00053696E6B5F4361705F4558004765745FC2
:10DBE0005352435F494E464F000000004765745F43
:10DBF0005265766973696F6E000000005265717539
:10DC0000657374004249535400000000426174740B
:10DC10006572795F5374617475730000416C65724D
:10DC2000740000004765745F436F756E7472795FAE
:10DC3000496E666F00000000456E7465725F555353
:10DC4000420000004550525F526571756573740063
:10DC50004550525F4D6F6465000000005352435FB2
:10DC6000496E666F0000000056656E646F725F4417
:10DC70006566696E656400002A000000A48E0120BC
:10DC80007283FF1F0E215220F5F788FAA0A0F4F747
:10DC90001DFF00210420F4F715F99EA0F4F716FFEC
:10DCA00063E00A215220F5F779FAAFF2D010F4F7C9
:10DCB0000DFFF888F978084400EB400008EB80007D
:10DCC00008214068F4F77EFDF888F978084400EBF5
:10DCD000400008EB8000808884B246E01CD10A2115
:10DCE0005220F5F75BFAAFF20C20F4F7EFFEF8885C
:10DCF000F978084400EB400008EB800008214068F8
:10DD0000F4F760FDF888F978084400EB400008EB70
:10DD10008000808884B228E000EB4116B6F800C08D
:10DD200062451ED1002414E0601C824600EB800096
:10DD30004006010E5220F5F731FAAFF26020F4F7F9
:10DD4000C5FE06EB840008214068F4F73BFD0AF0AD
:10DD5000FF04AC42E8D36D1E06EB8500808884B2D8
:10DD600003E0491C89B29942B8D9B9F80000F5F727
:10DD700021FA0E210020F5F711FA68A0F4F7A6FEAB
:10DD8000AFF2A820F4F7A2FEF888F978084400EB77
:10DD9000400008EB800004214088F4F713FD1921AE
:10DDA0000020F5F7FBF95EA0F4F790FEF888F9780B
:10DDB000084400EB400008EB800001218078C0F3AC
:10DDC0008110401CF5F7A4F924210020F5F7E6F9AD
:10DDD00056A0F4F77BFEF888F978084400EB400081
:10DDE00008EB800001214088C0F34220F5F790F94C
:10DDF00000210820F4F766F8F888F978084400EB69
:10DE00004000022118F82000F4F7DCFC2F2100204C
:10DE1000F5F7C4F9F888F978084400EB400018F8E1
:10DE20002010E0290DD308EB80004088000AC007CD
:10DE300003D03FA0F4F74AFE10E03EA0F4F746FE00
:10DE40000CE008EB80004088000AC00703D03AA02D
:10DE5000F4F73CFE02E037A0F4F738FE002108207A
:10DE6000F4F730F8F888F978084400EB400008EB44
:10DE7000800080784009C00703D030A0F4F726FE68
:10DE800002E02FA0F4F722FEF888F978084400EBAE
:10DE9000400008EB80004088C00B36D03A210020BB
:10DEA000F5F77CF927A0F4F711FEAFF2D030F4F7C4
:10DEB0000DFE04212046F4F785FC45210020F5F7EE
:10DEC0006DF9E00B03D021A0F4F700FE02E020A0E2
:10DED000F4F7FCFD00210420F3F7F4FFAFF2FC405F
:10DEE000F4F7F4FD0021C4F3C320F5F711F9002184
:10DEF0000420F3F7E7FF17A0F4F7E8FDC4F30800E8
:10DF0000BDE8F0470021F5F703B9BDE8F087000050
:10DF10004E4F00004461746100000000483A000068
:10DF200056657273696F6E3A0000000049443A000A
:10DF300053524300534E4B0043616200444650002D
:10DF4000554650004558483A000000004300000084
:10DF500055430000533A00002DE9FC5FDFF8E493DD
:10DF600099F800B0F848F94D4FF0010C0088EA78B4
:10DF7000431EC41FE988DEB24FF0060AA7B24FF075
:10DF80000008BBF1040F11D099F800B0BBF10A0FE3
:10DF90000CD099F80040052C2FD099F800400B2C9C
:10DFA0002BD099F80010062943D04AE085F802806A
:10DFB00070B1DFF898C307289CF803C00CF1010C7E
:10DFC0000CF0FF0C0AD29A4205DA85F803C038E05B
:10DFD00085F802C035E085F8038032E0062A02D2D7
:10DFE00085F803C02DE0A14204D185F80380A5F88F
:10DFF000068026E0491CE98023E085F8028040B1D4
:10E00000D24CE478641EE4B2072807D222B1EC7047
:10E0100017E085F802C014E0EE7012E00AB1EC706F
:10E020000FE011B1491EE9800BE085F803A0EF80F5
:10E0300007E030B1C64A1221117085F8028089F8D4
:10E04000008099F80010042903D099F800100529E0
:10E0500001D189F80080A97841B1062B01D2EE7078
:10E0600004E0072802D3EF8085F803A00C20F5F721
:10E070009BF800210846F5F791F8DFF8D892B9F837
:10E080000000F5F797F8B4A0F4F720FD0021042074
:10E09000F3F718FFB1A0F4F719FDB24800210068AA
:10E0A000F5F736F8DFF8C0B20C240023BBF8000007
:10E0B000CDE90004ADA219466620F5F781F8DFF836
:10E0C000B0A20023ABA2BAF80000CDE900041946C3
:10E0D0008220F5F775F8FF24B9F80000CDE90004B7
:10E0E0009E224F2300211046F4F704F8964E308804
:10E0F000012820D9401E00EE100AB8EEC00A9FED9C
:10E100009E1AE878E988C1EE000A084400EE100A79
:10E110009F220021B8EE400A20EE800ABCEEC00A21
:10E1200010EE100A83B2B9F80000CDE900049D207A
:10E13000F3F7E0FF09E0B9F80000CDE900044F2350
:10E140009F2200219D20F3F7D5FF3088072802D2B7
:10E1500000F0FF0801E04FF007080024874E66E258
:10E16000B9F80000F5F726F8671C07EB8700FF21D8
:10E1700001EB4000C1B20020F5F710F8E888042157
:10E180002044F4F7C5FFE888204400EB400006EB8C
:10E1900080004088C00504D5BBF80000F5F70AF8F8
:10E1A00003E0BAF80000F5F705F800210220F3F7C4
:10E1B00089FEE878844203D171A0F4F787FC03E07C
:10E1C00000210C20F3F77EFEE888204400EB40009D
:10E1D00006EB8000007A012824D000210720F3F705
:10E1E00071FEE888204400EB400006EB8000408888
:10E1F000C0F30231C20B74D000F01F001F2861D29F
:10E20000DFE800F06014181C2024282C3034383C3F
:10E210004044484C5054586060606060606060608A
:10E2200060605C0057A0F4F751FCDAE756A0F4F701
:10E230004DFCF0E157A0F4F749FCECE157A0F4F7EE
:10E2400045FCE8E158A0F4F741FCE4E154A0F4F700
:10E250003DFCE0E157A0F4F739FCDCE156A0F4F70F
:10E2600035FCD8E157A0F4F731FCD4E159A0F4F71C
:10E270002DFCD0E15BA0F4F729FCCCE15DA0F4F724
:10E2800025FCC8E15FA0F4F721FCC4E160A0F4F72D
:10E290001DFCC0E162A0F4F719FCBCE164A0F4F736
:10E2A00015FCB8E165A0F4F711FCB4E166A0F4F741
:10E2B0000DFCB0E167A0F4F709FCACE169A0F4F74C
:10E2C00005FCA8E16BA0F4F701FCE88804212044D8
:10E2D00000EB400006EB80004088F4F773FA9AE107
:10E2E000FFE769B100F01F00102828D2DFE800F036
:10E2F00027EFEEEDECEBEAE9E8E7E6E5E42727298E
:10E3000000F01F0019281BD2DFE800F01A0D1115CC
:10E31000C2C6CACED2F2F6FAFEEDECEBEAE9E8E7C5
:10E32000E6E5E4E3E20054A0F4F7D0FB73E154A087
:10E33000F4F7CCFB6FE154A0F4F7C8FB6BE15CE1B0
:10E3400016E156E16083FF1F7083FF1F6C8DFF1F76
:10E35000B183FF1FAA83FF1F504400005061636B0D
:10E36000733A00007883FF1FAC83FF1F53524300B2
:10E37000A883FF1F534E4B0000009E42F0B9FF1FC1
:10E380003E000000A1CC00005352435F4341505F68
:10E390004558000053746174757300004765745FDD
:10E3A0004261745F434150004765745F4261745F2E
:10E3B000535441004765745F4D616E75665F496EE9
:10E3C000666F000053656375726974795F52657199
:10E3D0000000000053656375726974795F5265735C
:10E3E000700000004669726D5F5570645F52657120
:10E3F000000000004669726D5F5570645F5265737E
:10E40000700000005050535F5374617475730000C6
:10E41000436F756E7472795F496E666F000000001D
:10E42000436F756E7472795F436F646573000000AB
:10E4300053696E6B5F4341505F45580045585F43D9
:10E440006F6E74726F6C00004550525F5352435FA1
:10E45000434150004550525F53696E6B5F434150DA
:10E460000000000056656E645F446566696E5F4536
:10E470005800000030780000476F6F64435243003B
:10E48000476F746F4D696E0041636365707400007F
:10E4900069A0F4F71BFBBEE069A0F4F717FBBAE034
:10E4A00069A0F4F713FBB6E069A0F4F70FFBB2E044
:10E4B0006AA0F4F70BFBAEE097E092E08DE088E015
:10E4C00083E07EE079E074E06EE069E064E05EE0C5
:10E4D0004AE045E040E03BE036E031E02CE027E078
:10E4E00022E01DE018E013E00EE009E004E0FFE7A1
:10E4F0005EA0F4F7EBFA8EE05EA0F4F7E7FA8AE0AC
:10E500005EA0F4F7E3FA86E05FA0F4F7DFFA82E0BA
:10E510005FA0F4F7DBFA7EE060A0F4F7D7FA7AE0C8
:10E5200061A0F4F7D3FA76E063A0F4F7CFFA72E0D3
:10E5300064A0F4F7CBFA6EE066A0F4F7C7FA6AE0DD
:10E5400067A0F4F7C3FA66E067A0F4F7BFFA62E0E9
:10E5500069A0F4F7BBFA5EE06CA0F4F7B7FA5AE0F2
:10E560006EA0F4F7B3FA56E070A0F4F7AFFA52E0F9
:10E57000AFF20010F4F7AAFAE8880421204400EB77
:10E58000400006EB80004088F4F71CF943E0AFF24E
:10E590004410F4F79BFA3EE068A0F4F797FA3AE0EB
:10E5A00068A0F4F793FA36E0AFF25410F4F78EFA5D
:10E5B00031E066A0F4F78AFA2DE068A0F4F786FA55
:10E5C00029E068A0F4F782FA25E06BA0F4F77EFA60
:10E5D00021E06CA0F4F77AFA1DE06DA0F4F776FA6A
:10E5E00019E06EA0F4F772FA15E051A0F4F76EFA94
:10E5F00011E06DA0F4F76AFA0DE0AFF28810F4F7BD
:10E6000065FAE8880421204400EB400006EB800016
:10E610004088F4F7D7F8E888204400EB400016F86B
:10E620002000E02802D264A0F4F750FAFCB244457E
:10E63000FFF496ADBDE8FC9F52656A656374000007
:10E6400050696E670000000050535F52445900004B
:10E650004765745F5352435F436170004765745F61
:10E6600053696E6B5F4361700000000044525F535A
:10E670007761700050525F537761700056434F4E80
:10E680004E5F5377617000005761697400000000AD
:10E69000536F66745F526573657400004441544162
:10E6A0005F52657365740000444154415F52657365
:10E6B00065745F4F4B0000004E6F745F5375707050
:10E6C0006F7274004765745F5352435F4361705FBC
:10E6D000455800004765745F53746174757300009A
:10E6E00046525F53776170004765745F5050535FC7
:10E6F00053746174757300004765745F436F756E82
:10E700007472795F436F6465000000004765745F51
:10E7100053696E6B5F4361705F4558004765745F76
:10E720005352435F494E464F000000004765745FF7
:10E730005265766973696F6E0000000052657175ED
:10E7400065737400424953540000000042617474C0
:10E750006572795F5374617475730000416C657202
:10E76000740000004765745F436F756E7472795F63
:10E77000496E666F00000000456E7465725F555308
:10E78000420000004550525F526571756573740018
:10E790004550525F4D6F6465000000005352435F67
:10E7A000496E666F0000000056656E646F725F44CC
:10E7B0006566696E656400002A0000000349002058
:10E7C0000870034910200870704700006083FF1F25
:10E7D000B183FF1F2DE9F0472DED028B0C20F4F7DC
:10E7E000E3FCD7480088F4F7E5FC00210846F4F77D
:10E7F000D5FCDFF850A39AF8190001281BD09AF82D
:10E800001A00E0B1D0A0F4F761F9D14E96F82800D3
:10E8100096F8291008440021F4F77AFC00212B20F7
:10E82000F4F7BCFCDFF82C8398F8080001280AD024
:10E8300002282AD06DE0C8A0F4F748F9E5E7C7A0A0
:10E84000F4F744F9E1E7C7A0F4F740F998F80000BD
:10E850000221F4F75DFCC5A0F4F738F9C4A0F4F781
:10E8600035F900210820F3F72DFB98ED010A02216C
:10E87000BDEEC00A10EE100AF4F74AFCBBA0F4F794
:10E8800025F9BCA0F4F722F943E0BBA0F4F71EF988
:10E89000B8F80A009FEDBA8BB0F5FA7F12D2BAA091
:10E8A000F4F714F9B8F80A00F1F720FF53EC182B2D
:10E8B000F1F73BFEF1F784FF00EE100A0220F4F7B7
:10E8C000B5FB0CE0F1F712FF53EC182BF1F72DFE1E
:10E8D000F1F776FF00EE100A0220F4F7A7FBA4A0E0
:10E8E000F4F7F4F800210820F3F7ECFAA6A0F4F707
:10E8F000EDF898F80C0000EE100AB8EE400ADFEDD3
:10E90000A30A022020EE200AF4F790FB99A0F4F766
:10E91000DDF898F80800032820D19DA0F4F7D6F878
:10E9200098F800000221F4F7F3FB90A0F4F7CEF87A
:10E930008FA0F4F7CBF800210820F3F7C3FA98ED85
:10E94000010A0221BDEEC00A10EE100AF4F7E0FB46
:10E9500086A0F4F7BBF887A0F4F7B8F80A210020E6
:10E96000F4F71CFC0025DFF83092DCE006EB8504B0
:10E9700094ED0B0AD4ED150A20EE200AD6ED3D0ADF
:10E98000B4EEE00AF1EE10FA01DD86ED3D0A98F8EA
:10E990001900A84204D181480088F4F70BFC03E079
:10E9A0007F480088F4F706FC6F1C07EB87004006E1
:10E9B000010E0020F4F7F2FB354495F8F800012829
:10E9C00006D0022829D0032827D004287DD0A9E02A
:10E9D00094ED0B0A0220F4F729FB65A0F4F776F812
:10E9E00000210720F3F76EFA94ED150A0220F4F7E0
:10E9F0001DFB60A0F4F76AF800210720F3F762FA24
:10EA000094ED0B0AD4ED150A022020EE200AF4F74B
:10EA10000DFB64A0F4F75AF884E094ED330A022069
:10EA2000F4F704FB60A0F4F751F894ED290A0220F2
:10EA3000F4F7FCFA4EA0F4F749F800210720F3F7A9
:10EA400041FA94ED150A0220F4F7F0FA49A0F4F720
:10EA50003DF800210720F3F735FA95F8020120B3BD
:10EA600094ED290AD4ED150A60EE200A96ED3D0AD0
:10EA7000F4EEC00AF1EE10FA17D39AF81900012843
:10EA800013D010EE100A484502DA0120F4F7CEFA4E
:10EA900096ED3D0A10EE100A484502DB0020F4F71F
:10EAA000C5FA40A0F4F712F83CE094ED290AD4ED41
:10EAB000150A20EE200A10EE100A484502DA01205D
:10EAC000F4F7B4FA94ED290A00E00BE0D4ED150A4E
:10EAD00020EE200A10EE100A4845E2DB0020F4F791
:10EAE000A5FADEE794ED330A0220F4F79FFA2EA090
:10EAF000F3F7ECFF94ED290A0220F4F797FA1CA033
:10EB0000F3F7E4FF00210720F3F7DCF996ED3D0A67
:10EB10000021BDEEC00A10EE100AF4F7F9FA21A0A8
:10EB2000F3F7D4FFFDB296F8280096F829100844B0
:10EB3000A8423FF61BAFBDEC028BBDE8F08700009A
:10EB4000AC83FF1F24CD01204550523A0000000045
:10EB5000E4B8FF1F44B7FF1F4D493A0050444F3AF5
:10EB6000000000004649583A000000002E303000F6
:10EB700056000000410000005050533A00000000D1
:10EB80007B14AE47E17A943F30000000CDCC4C3D81
:10EB90005661723A000000000000C842A883FF1FBF
:10EBA000AA83FF1F570000007E0000002DE9FC5FD4
:10EBB00000F028FA0C20F4F7F7FAF94C2088F4F763
:10EBC000F9FA00210846F4F7E9FADFF8D8A39AF831
:10EBD0001900012820D09AF81A0008B3F2A0F3F720
:10EBE00075FFF34F97F8280097F829100844002183
:10EBF000F4F78EFA00212D20F4F7D0FAED49EE4D0E
:10EC000091ED000A10EE100AA8420DDA032091EDF2
:10EC1000000AF4F70BFA0CE0E8A0F3F757FFE0E77F
:10EC2000E7A0F3F753FFDCE7022091ED000AF4F7C9
:10EC3000FDF9E5A0F3F74AFF00210820F3F742F9B8
:10EC4000E24991ED000A10EE100AA84205DA03200D
:10EC500091ED000AF4F7EAF904E0022091ED000AD0
:10EC6000F4F7E4F9DAA0F3F731FFDFF8688398F8F6
:10EC70000000D94E4FF00C053178084208D02088AA
:10EC8000CDE900050023D5A219468A20F4F798FAA9
:10EC900098F800003178884308D02088CDE9000535
:10ECA0000023CFA219468A20F4F78AFA307898F820
:10ECB0000010884308D02088CDE900050023C8A2B1
:10ECC00019468A20F4F77CFA98F8000050B9307899
:10ECD00040B92088CDE900050023C0A219468A204A
:10ECE000F4F76EFA0A210020F4F758FA97F8280092
:10ECF00097F829100844072801D9072600E0C6B272
:10ED00000024DFF8E0B2DFF8E092DFF8E08211E102
:10ED100098F80100204407EB800090ED0B0AD0ED3D
:10ED2000150A20EE200AD7ED3D0AB4EEE00AF1EE16
:10ED300010FA01DD87ED3D0A651C05EB85004006F4
:10ED4000010E0020F4F72AFAA948007EA04207D15C
:10ED5000A8480088F4F72EFAA0A0F3F7B7FE03E066
:10ED6000BBF80000F4F726FA98F801002044C11916
:10ED700091F8F810012906D0022935D0032933D0A3
:10ED800004297DD0D5E007EB800090ED0B0A02202E
:10ED9000F4F74CF98CA0F3F799FE00210720F3F764
:10EDA00091F898F80100204407EB800090ED150AD7
:10EDB0000220F4F73BF986A0F3F788FE0021072034
:10EDC000F3F780F898F80100204407EB800090EDFD
:10EDD0000B0AD0ED150A022020EE200AF4F726F9DE
:10EDE00085A0F3F773FEA4E007EB800090ED330AF3
:10EDF0000120F4F71BF981A0F3F768FE98F80100F1
:10EE0000204407EB800090ED290A0120F4F70EF969
:10EE10006DA0F3F75BFE00210720F3F753F898F895
:10EE20000100204407EB800090ED150A0220F4F762
:10EE3000FDF867A0F3F74AFE00210720F3F742F838
:10EE400098F801002044C11991F8021141B307EB71
:10EE5000800191ED290AD1ED150A60EE200A97EDA7
:10EE60003D0AF4EEC00AF1EE10FA19D39AF819101F
:10EE7000012915D010EE100A484504DA012000E0FF
:10EE800030E0F4F7D3F897ED3D0A10EE100A48454C
:10EE900002DB0020F4F7CAF857A0F3F717FE48E0AA
:10EEA00007EB800090ED290AD0ED150A20EE200A2C
:10EEB00010EE100A484502DA0120F4F7B7F898F886
:10EEC0000100204407EB800090ED290AD0ED150ADF
:10EED00020EE200A10EE100A4845DDDB0020F4F792
:10EEE000A5F8D9E707EB800090ED330A0220F4F78C
:10EEF0009DF842A0F3F7EAFD98F80100204407EBE3
:10EF0000800090ED290A0220F4F790F82EA0F3F784
:10EF1000DDFD00210720F2F7D5FF97ED3D0A002126
:10EF2000BDEEC00A10EE100AF4F7F2F832A0F3F7C3
:10EF3000CDFDECB2B442FFF4EBAEFF24BBF8000011
:10EF4000CDE900049E224F2300211046F3F7D2F8AA
:10EF500017F8280F9FED2A1A79789F220844401E3F
:10EF600000EE100A224898F80110B8EEC00A007EA0
:10EF70000844C1EE000A00EE100A0021B8EE400A73
:10EF800020EE800ABCEEC00A10EE100A83B2BBF875
:10EF90000000CDE900049D20F3F7ACF8BDE8FC9F2C
:10EFA000AC83FF1F24CD01204550523A00000000E1
:10EFB000E4B8FF1F3483FF1F000020414D493A0091
:10EFC00050444F3A00000000560000003C83FF1FF1
:10EFD000410000003083FF1FA683FF1F3E0000009A
:10EFE0003C000000AA83FF1F0000C8426C8DFF1F79
:10EFF00044B7FF1FA883FF1F570000007E000000DA
:10F0000000009E422DE9F0412A4CA07B032801D14B
:10F010000120A073284E96F800802848DFF8A0C091
:10F0200000274178007845182248EB1F6A1E007EB1
:10F030009CF80110B8F1040F15D096F80080B8F1D3
:10F04000050F24D03278062A0BD10844C0B260766E
:10F05000F7F7CAFF94F8340010B11A490920087074
:10F060003770BDE8F081824204DD062802D2401CE0
:10F0700020760AE08B4201D0824203D127768CF8B9
:10F08000017002E0491C8CF801103770E9E710B1FB
:10F09000401E207603E021B1491E8CF80110377024
:10F0A000DFE7072D04D9062020768CF80130F6E73B
:10F0B0002276F4E744B7FF1F6083FF1F0CB9FF1FE0
:10F0C0006C8DFF1FB183FF1F0349002008700349A7
:10F0D00008200870704700006083FF1FB183FF1F86
:10F0E0002DE9FC477D4D2B787E4C7D4F002694F812
:10F0F00039003A7994F83810042B09D02B78052B75
:10F100001AD0287806282BD028780C282DD039E062
:10F110002E7042B1092803D2401C84F8390031E036
:10F1200084F839602EE0032903D2491C84F8381092
:10F1300028E084F8386025E02E7042B118B1401EF6
:10F1400084F839001EE0092084F839001AE019B16A
:10F15000491E84F8381015E0032084F8380011E0C7
:10F1600082F0010038712E700CE02E70F8F744FE2A
:10F1700000210220F8F770FD46210920F8F76CFD08
:10F18000594806701020F4F70FF800210846F4F7EC
:10F1900005F8564E3088F4F70DF83879DFF85081CD
:10F1A0006FF00109A0B902210020F2F78BFE0C20BC
:10F1B000F3F7FAFFB8F80000F3F7FCFF4DA0F3F700
:10F1C00085FC49460020F2F77DFE1020F3F7ECFFA6
:10F1D00049A0F3F7C9F894F83800414900EB8000E2
:10F1E000083151F83000F3F771FC10210020F3F7DB
:10F1F000D5FF3088F3F7DEFF3879A0B10221002077
:10F20000F2F760FE0C20F3F7CFFFB8F80000F3F739
:10F21000D1FF38A0F3F75AFC49460020F2F752FE1E
:10F220001020F3F7C1FF37A0F3F79EF8012100206B
:10F23000F2F748FE35A0F3F749FC94F83900284965
:10F2400000EB8000A83151F83000F3F73FFC352186
:10F250000E20F3F7A3FF3088F3F7ACFF47F6EF3645
:10F26000002231461E2007F093FE0224CDE9004023
:10F270001523892232210B20F2F77EFF28780328FC
:10F280001ED1234D2868234F3968401AFA2817D910
:10F2900000223146DC2007F07BFE29683A68CDE980
:10F2A00000408A1A02EBC20101EBC2114FF47A72DC
:10F2B000B1FBF2F1CAB2152332210B20F2F75CFF49
:10F2C000CDE900461523892232210B20F2F70CFEEE
:10F2D000BDE8FC4710A0F3F747B800006083FF1FAC
:10F2E0006C8DFF1F74610220B183FF1FAA83FF1F73
:10F2F000A883FF1F3E000000312ED3D5C6ADC4A3A6
:10F30000CABD3A00322EC4A3C4E20000456D3A00E3
:10F310007C83FF1F6C83FF1FB0B4D7A1C8B7C8CFD1
:10F32000BCFCB1A3B4E6B2A2D6D8D0C2D3D5C6AD88
:10F33000000000002DE9F041574D2A780127DFED4C
:10F34000571A9FED571A9FED572A574C0026042A4B
:10F35000E07C94ED120AD4ED130A617C0FD02A7878
:10F360000A2A0CD02A78052A34D02A780B2A31D0E0
:10F370002A78062A59D0287809287AD080E031B135
:10F38000012906D0022909D0032979D118E0A774F0
:10F3900076E0242874D2401CE07471E010EE100A6C
:10F3A000424988426CDA28780A2804D030EE010AF3
:10F3B00084ED120A64E030EE210A84ED120A5FE067
:10F3C00010EE900AB0F1824F5ADA30EE820A84EDE4
:10F3D000130A55E031B1012906D0022909D00329C9
:10F3E0004ED118E0A6744BE0052849D9401EE074C0
:10F3F00046E010EE100A2E49884241DD28780B289D
:10F4000004D030EE410A84ED120A39E030EE610A90
:10F4100084ED120A34E010EE900A264988422FDD6E
:10F4200030EEC20A84ED130A2AE022780AB9491C98
:10F430006174617C042923D112BB032161741E49CC
:10F44000A27CCA7108720920F8F720FD94ED130A16
:10F450000D20F8F71BFDF8F7CFFC18480168226B68
:10F46000891AB1F5487F0BD927700068206307E03F
:10F47000FFE711B1491E617401E0112060702E7028
:10F480002878062805D02878052802D0287804286E
:10F4900000D12E70BDE8F0816083FF1FCDCCCC3D44
:10F4A0000AD7A33CCDCC4C3DB083FF1F00001042D7
:10F4B000333353408FC2753D746102207C83FF1F3C
:10F4C0002DE9F04F2DED048B85B0DFF8F8A3FE4C4D
:10F4D000BAF8040000EBC00C04EB8C0090F821108B
:10F4E00001297DD1DAF80810491CCAF8081090F8F3
:10F4F00020805246F54D1788012607EB470305EBA0
:10F500008302B8F1010F03D11672491CCAF8081022
:10F51000ED4911F82C40ED4901F823404188518014
:10F520004188C1F302334188E64C5FEAD13BDFF802
:10F53000A48361888E4601F1010189B2049121887A
:10F54000E34C01F1010189B204EB4E149FEDE29A04
:10F55000DFEDE28A9FEDE28ADFEDE29A0391E24974
:10F56000E24DDFF88C9391F828100291A97B79D0B5
:10F57000012B04D0BEF5FA7F14D200220CE04468BF
:10F5800054600FE000EB820CDCF804C004EB820B4B
:10F59000CBF804C0521CD2B29A42F3D32780049A0B
:10F5A000AAF8022042F20F72974202D2039AAAF8F6
:10F5B00000205B1E00EB830252681FFA82FB428828
:10F5C00002F01F02102A7DD0112A7CD14088C0058C
:10F5D0007AD51BF4F04F77D0C34880F8293000E08B
:10F5E000F0E3029CFDE0BAF80420201A02EBC2030B
:10F5F000B54A02EB830202EB8000406841F8240028
:10F60000820F03D0C243920F2DD0E8E0081980F892
:10F61000F86051F8240001EB8401C0F3892200EE68
:10F62000102AB8EE400A20EE280A81ED0B0AC0F33A
:10F63000090000EE900AF8EE600A60EE880AC1ED5B
:10F64000150A98F8070000280BD198F8080000EE7A
:10F65000900AF8EE600AB4EEE00AF1EE10FA00D873
:10F66000AC76BCE0EEE0C00052D504200A1902F8E6
:10F67000F80F51F8240001EB8407C0F3484300EE73
:10F68000103AB8EE400A20EE090A87ED290AC0F3C5
:10F69000072100EE101AB8EE400A20EE090A87EDA5
:10F6A000330A907298F80700012830D10920F8F742
:10F6B0008DFBD7ED330AB4EEE00AF1EE10FA26DB4B
:10F6C000092002E0B9E0AAE094E0F8F77FFBD7ED6B
:10F6D000290AB4EEE00AF1EE10FA18D8AC76092047
:10F6E000F8F774FB30EE080ADFED820A80EE201A8C
:10F6F000BCEEC10A10EE100A68810D20F8F766FB17
:10F70000C0EE280ABCEEE00A10EE100A287366E08C
:10F710000322081900F8F82F51F82420C2F3C06220
:10F72000827251F8240001EB8407C0F3474200EED7
:10F73000102AB8EE400A20EE090A87ED290AC0F324
:10F74000072100EE101AB8EE400A20EE090A87EDF4
:10F75000330AC0B200EE100AB8EE400A20EE280AC2
:10F7600087ED150A98F80700012838D10920F8F725
:10F770002DFBD7ED330AB4EEE00AF1EE10FA2EDBE2
:10F780000920F8F723FBD7ED290AB4EEE00AF1EEE1
:10F7900010FA24D8287B58B10D20F8F717FBD7EDC5
:10F7A000150A70EE880AB4EEE00AF1EE10FA16D8E7
:10F7B000AC760920F8F70AFB30EE080AC0EE290AF9
:10F7C000BCEEE00A10EE100A68810D20F8F7FEFA90
:10F7D000C0EE280ABCEEE00A10EE100A2873641C82
:10F7E000E4B2414991F8280091F829200244A2424C
:10F7F0003FF6F9AE99F81A00012810D1A87B01282C
:10F80000FBD199F81F0058B9CBF30801182907D983
:10F81000F7F794FB99F81F00401C89F81F0050E08F
:10F820000128FCD1A87EF7F7DFFBA87E2876687652
:10F830002E7431480068686243E00129EFD100204E
:10F84000A8743EE0DFF8A8B09BF817B0CDF804B07C
:10F8500033B1012B70D0BEF5FA7F6ED2002230E1B9
:10F8600042F20F72974202D2039AAAF8002040880F
:10F870001F4A00F01F0B1C48137D927D04681B4833
:10F88000BBF1110F477C807EC9D2DFE80BF01A096B
:10F890001A37701A801AAC1A1AB11AE41A1AFC0034
:10F8A000BAF800000128BAD9811E01EB41020749CC
:10F8B00001EB82010A7A002AB1D10E72401EAAF829
:10F8C0000000E3E37083FF1F7CB7FF1FF0B9FF1F49
:10F8D000A48E012074610220CDCCCC3DCDCC4C3D1A
:10F8E0000AD7233C0AD7A33CE4B8FF1F44B7FF1F45
:10F8F00024CD0120CDCCCC3C7C83FF1F01298ED1AF
:10F9000099F81500012800D113B1012A05D006E0AD
:10F9100089F81460F8F716F8B8E3019810B1012AD5
:10F920000CD0B3E3002089F8160089F8176089F835
:10F930002160F7F755F8A9E3B6E0C8E0019801287F
:10F94000BFD1002089F8160089F8170099F819002E
:10F95000012806D02002B4D5F6F73AFD89F81E60DA
:10F9600094E3F7F7A9FF0C2089F821008EE3012921
:10F97000A7D1012AA5D1002189F81610002FA0D106
:10F98000F7F732FBA87E287668766E747EE301294D
:10F9900097D11FB199F8180038B116E0F7F724FB9A
:10F9A000A87E287668766E740FE0FD4800780128FE
:10F9B0000BD998F8380002280AD0012805D089F818
:10F9C0001860F6F75BFC89F816600020A8745DE308
:10F9D0002002FAD599F81E000028F6D1F6F7F8FCB7
:10F9E00089F81E60F1E7012996D1F8F763F84DE335
:10F9F0004BB10020F6F776FBEA48007801281DD0CD
:10FA0000022820D023E00020F6F76CFBE5480078C0
:10FA1000012802D0022805D008E025210220F8F7AD
:10FA20001BF903E01A210220F8F716F9F7F78AFF0D
:10FA300089F81460DC480068A86227E305210220E9
:10FA4000F8F70AF903E00A210220F8F705F9002087
:10FA500089F814001AE3D54810F82C00DF2813D8D1
:10FA60004FF40051022000F047FC01288ED1D04C09
:10FA7000207800288AD0CF49002008700120F6F7AE
:10FA800031FB267002E307E00129A0D1CA4900201A
:10FA90000870F6F727FBF9E2012998D1012A96D1DF
:10FAA000002089F81600F1E2446854600FE000EB92
:10FAB000820BDBF804B004EB820ECEF804B0521CCB
:10FAC000D2B29A42F3D32780049AAAF8022042F2D3
:10FAD0000F72974202D2039AAAF80020DFF8CCB244
:10FAE0004288022402F01F02B44F102AA5D2DFE898
:10FAF00002F0FC08FBFCFCFCFCFCFCFAF9FCFCFC46
:10FB0000FCF8AF4F87F82830002106E000EB8102B7
:10FB1000526847F82120491CC9B297F828208A4228
:10FB2000F4D84FF00009CCE057F82900810F29D014
:10FB3000B4EB907F53D107EB090080F8F84057F8F9
:10FB40002900C0F3095100EE101A07EB8901B8EE45
:10FB5000400A20EE280A81ED290AC0F3892200EE2E
:10FB6000102AB8EE400A20EE280A81ED330AC0F3CD
:10FB7000090000EE100AB8EE400A20EE080A81EDF6
:10FB8000150A9AE007EB090080F8F86057F8290099
:10FB9000C0F3892100EE101A07EB8901B8EE400A84
:10FBA00020EE280A81ED0B0AC0F3090000EE900A4E
:10FBB000F8EE600A60EE880AC1ED150A98F80700B1
:10FBC000F0BB98F8080000EE900AF8EE600AB4EE78
:10FBD000E00AF1EE10FA70D885F81A906DE0C04393
:10FBE000800F6AD107EB0900032100F8F81F57F8CE
:10FBF0002910C1F3C061817257F8290007EB890B06
:10FC0000C0F3474100EE101AB8EE400A20EE090A90
:10FC10008BED290AC0F3072100EE101AB8EE400A56
:10FC200020EE090A8BED330AC0B200EE100AB8EEDE
:10FC3000400A20EE280A8BED150A98F8070000E02C
:10FC40003BE0012839D10920F8F7C0F8DBED330A91
:10FC5000B4EEE00AF1EE10FA2FDB0920F8F7B6F85F
:10FC6000DBED290AB4EEE00AF1EE10FA25D8287B84
:10FC700058B10D20F8F7AAF8DBED150A70EE880AE6
:10FC8000B4EEE00AF1EE10FA17D885F81A900920C0
:10FC9000F8F79CF870EE080A80EEA90ABCEEC00ADC
:10FCA00010EE100A68810D20F8F790F8C0EE280ACF
:10FCB000BCEEE00A10EE100A287309F1010909F000
:10FCC000FF0997F8280048453FF62EAFA87B01288A
:10FCD0000BD1BAF8040000EBC001344800EB8100FE
:10FCE00004E0DEE0B2E06EE011E086E090F8200093
:10FCF0000128EDD1687C30B1A87EF7F775F9A87EB0
:10FD000028766876C2E10020F7F76EF9BEE1416817
:10FD1000C1F30271397009B14A1E6A76284B5A182C
:10FD200092F8F720012A04D0032A19D0022A1FD002
:10FD3000ACE12E72491E03EB810191ED0B0ABCEE82
:10FD4000C00A10EE101A29704068C0F3892000EE36
:10FD5000100AB8EE400A20EE080A85ED010A95E186
:10FD60002C724168C1F34A216981406828738DE192
:10FD700003222A72491E03EB810191ED290ABCEE90
:10FD8000C00A10EE101A29704068C0F3892000EEF6
:10FD9000100AB8EE400A20EE080A85ED010A75E166
:10FDA0002283FF1F2083FF1F7C83FF1F7CB7FF1F61
:10FDB0002183FF1F2483FF1F2383FF1F2583FF1F32
:10FDC000E4B8FF1F74E10299BC4B002915D04168CB
:10FDD000090F3970072903D9029AC91F11443970D4
:10FDE000397809B14A1E6A765A1892F8F720012A22
:10FDF00004D0032A19D0042A1FD047E12E72491ECD
:10FE000003EB810191ED0B0ABCEEC00A10EE101A53
:10FE100029704068C0F3892000EE100AB8EE400A4D
:10FE200020EE080A85ED010A30E12C724168C1F329
:10FE30004A2169814068287328E1042129724168B8
:10FE4000C1F34A216981406828731FE14268B4EB1D
:10FE5000126F01D1012907D042680321B1EB126F63
:10FE600016D189F81A6011E195480078012802D06E
:10FE7000022805D008E001210320F7F7EDFE03E09A
:10FE800002210320F7F7E8FE8E4804210170FDE00F
:10FE900040680521B1EB106F02D1002089F81A00EB
:10FEA000F4E01BF82C20A02A6FD31BF82C20DF2AAB
:10FEB0006BD84FF40051022000F01EFA012836D111
:10FEC00098F8390078B3BAF8040000EBC0000BEBE7
:10FED000800041684AF2010289B2914202D1F7F7EB
:10FEE00089FAD3E0416889B2A1F50042023A11D003
:10FEF000416889B2A1F50042033A0ED0416889B247
:10FF0000B1F5827F10D0406880B2A0F521411F3941
:10FF100006D0BBE0F7F72CFBB8E0F7F78BFBB5E0BA
:10FF2000F7F764FCB2E002E0F7F7FAFBAEE099F80D
:10FF30001B0030B999F81C1019B999F81D10012946
:10FF400006D0012822D099F81C00012827D09DE076
:10FF5000BAF8040000EBC0000BEB80004168C9F860
:10FF600000108168C9F80410C268C9F80820026945
:10FF7000C9F80C204069C9F81000480104D50120D7
:10FF8000F7F726FD89F81B6080E024E00220F7F7F0
:10FF90001FFD002089F81B0089F81C6076E0BAF884
:10FFA000040000EBC0000BEB80008168C1F303414B
:10FFB000032905D08068C0F303400B2804D006E075
:10FFC000032089F8200002E0042089F820000020A6
:10FFD00089F81C005AE0012902D1019A012A02D0B5
:10FFE00001294BD052E099F82110022905D18268ED
:10FFF000A9F824200069A9F82600B9F82400A0F582
:020000040002F8
:100000001C52173A03D042F60132904231D1B9F86E
:100010002600A0F52440753816D0112806D00729EF
:1000200020D0052932D8F6F7DBFC2FE00B2904D0CD
:100030000A292BD8F6F722FA28E0F6F71FF989F8F3
:10004000196089F8166021E00B2904D00A291DD80F
:10005000F6F714FA1AE0F6F711F989F8196089F839
:10006000166013E0F6F70AF989F8196089F8166046
:100070000CE0F6F703F989F8166007E0406880B2F3
:10008000A0F52041023901D1F6F7DCFEBAF80400F0
:100090000D4A00EBC00302EB8302002182F821101D
:1000A000401C80B2AAF804000A2801D1AAF8041062
:1000B00005B0BDEC048BBDE8F08F0000E4B8FF1F75
:1000C0002083FF1F2183FF1F7CB7FF1F0449C878CF
:1000D000401CC0B2C870072801D90020C870704702
:1000E0002083FF1F04490879401CC0B2087107280B
:1000F00001D90020087170472083FF1F2DE9F041CE
:10010000254E264C2648B27B012500786168012ADD
:1001100014D000291DD16575224C01282FD002284A
:1001200017D11821F7F798FD2078BDE8F04102219A
:1001300001EB4010C1B20320F7F78EBD627D002AAB
:1001400007D1002905D1217D174F21B16575386888
:10015000B062BDE8F081012802D0022805D008E095
:1001600025210220F7F778FD03E01A210220F7F796
:1001700073FDF7F715FD65753868B062E9E724216E
:100180000220F7F769FD207805EB4010BDE8F0414B
:10019000C1B20320F7F760BD44B7FF1F24CD012093
:1001A0002083FF1F2283FF1F7C83FF1F2DE9F04167
:1001B000304F314C314D97F82100062807D1E86ABD
:1001C00028B12168081A2D2801D9F6F709FC95F8FD
:1001D000340001280DD1287C58B9286A2168081AF2
:1001E00042F22831884204D9687EF6F7FDFE206885
:1001F0002862287C01280ED1686A2168091A40F219
:10020000EE20814207D9F6F78BF82068686201205A
:10021000A87420682863787D002601280FD1A86A79
:100220002168081A96280AD97E750020F7F7D0FBB6
:1002300097F82200012802D1022087F82200A87B2B
:10024000012808D1A87C30B9E87C012803D1687E58
:10025000F6F7CAFEEE74A87B012809D1A87C012814
:1002600006D1286B2168081AB0F5FA7F00D9AE7460
:10027000BDE8F08124CD01207C83FF1F44B7FF1F20
:1002800070B505460C461F2D04D940F223110EA06F
:10029000F5F7C4F934B1012C04D04FF492710AA0DF
:1002A000F5F7BCF900F036FA124905F01F00012CF1
:1002B00006D00A8882430A8000F050F9002070BD01
:1002C0000A8802430A80F7E72E2E5C2E2E5C2E2E23
:1002D0005C2E2E5C2E2E5C6472697665725C737285
:1002E000635C68633332663436305F6770696F2EE3
:1002F00063000000F43B054070B505460C46002D38
:100300000ED0012D0CD0022D0AD0032D08D0042DC3
:1003100006D0052D04D04FF4C8711CA0F5F77EF966
:10032000012C2AD0022C28D0042C26D0082C24D032
:10033000102C22D0202C20D0402C1ED0802C1CD061
:10034000B4F5807F19D0B4F5007F16D0B4F5806F76
:1003500013D0B4F5006F10D0B4F5805F0DD0B4F5B4
:10036000005F0AD0B4F5804F07D0B4F5004F04D039
:1003700040F2911105A0F5F751F90F4800EB051077
:100380000068204000D0012070BD00002E2E5C2EA1
:100390002E5C2E2E5C2E2E5C2E2E5C647269766591
:1003A000725C7372635C68633332663436305F67E5
:1003B00070696F2E63000000003805402DE9F041A0
:1003C00006460F4614460025002E0DD0012E0BD0F8
:1003D000022E09D0032E07D0042E05D0052E03D0FF
:1003E000AC2152A0F5F71AF9207838B1012805D0D0
:1003F000022803D0AE214DA0F5F710F9607938B18D
:10040000012805D0022803D0AF2148A0F5F706F94E
:10041000A07928B1012803D0B02144A0F5F7FEF857
:10042000607828B1012803D0B12140A0F5F7F6F893
:10043000A07828B1012803D0B2213CA0F5F7EEF84E
:10044000E07828B1012803D0B32138A0F5F7E6F809
:10045000207928B1012803D0B42134A0F5F7DEF8C3
:10046000E07928B1012803D0B52130A0F5F7D6F8FE
:1004700000F050F9012101FA05F038424CD0B001EA
:10048000354A00EB85008318921C024494F801C0A1
:1004900018886CF38E30188094F802C018886CF3BA
:1004A0000C30188094F803C018886CF34920188029
:1004B00094F804C018886CF38610188094F806C06D
:1004C00018886CF38200188094F805C018886CF3C3
:1004D00005101880207820B101280BD0022816D1F1
:1004E00011E0188820F400401880188820F00200DD
:1004F00018800CE0188820F400401880188840F01C
:100500000200188003E0188840F400401880E37966
:10051000108863F3082010806D1CEDB2102DAAD353
:1005200000F01CF80020BDE8F08100002E2E5C2EAB
:100530002E5C2E2E5C2E2E5C2E2E5C6472697665EF
:10054000725C7372635C68633332663436305F6743
:1005500070696F2E63000000003C054002494FF4B3
:100560002540088070470000FC3B054070B50446FC
:100570000D46002C0ED0012C0CD0022C0AD0032CDE
:1005800008D0042C06D0052C04D040F20F2105A081
:10059000F5F744F80E4800EB041002882A43028065
:1005A000002070BD2E2E5C2E2E5C2E2E5C2E2E5C1E
:1005B0002E2E5C6472697665725C7372635C68632C
:1005C0003332663436305F6770696F2E6300000027
:1005D0000A38054070B504460D46002C0ED0012C9B
:1005E0000CD0022C0AD0032C08D0042C06D0052CE9
:1005F00004D040F2F71105A0F5F710F80E4800EB13
:10060000041002882A430280002070BD2E2E5C2E2A
:100610002E5C2E2E5C2E2E5C2E2E5C64726976650E
:10062000725C7372635C68633332663436305F6762
:1006300070696F2E63000000083805402DE9F04115
:100640000646884615461F460024002E0ED0012E71
:100650000CD0022E0AD0032E08D0042E06D0052E70
:1006600004D04FF41A711FA0F4F7D8FF75B1681EBB
:1006700009280BD90E2D09D00F2D07D01F381B28A4
:1006800004D940F2692117A0F4F7C8FF37B1012F50
:1006900004D040F26A2113A0F4F7C0FF00F03AF84A
:1006A0000123B1011A4E03FA04F010EA080F0CD02E
:1006B00001EB84003044028865F305020280012FBB
:1006C0000CD0028822F480720280641CE4B2102CE8
:1006D000E9D3FFF743FF0020BDE8F081028842F430
:1006E0008072F1E72E2E5C2E2E5C2E2E5C2E2E5C60
:1006F0002E2E5C6472697665725C7372635C6863EB
:100700003332663436305F6770696F2E63000000E5
:10071000023C054002494AF201500880704700003F
:10072000FC3B05402DE9F0412DED028B82B000F03D
:10073000C3F9C748C74F1C2490ED000AC64D10EE00
:10074000101AB9420BDA2988CDE90014002390ED84
:10075000000A042219461846F2F79CFF0AE029888D
:10076000CDE90014002390ED000A03221946184633
:10077000F2F790FF2888CDE900040023B7A21946BC
:100780005320F2F71DFDB648DFF8D88290ED000A3D
:1007900010EE101AB9420CDAB8F80010CDE90014C6
:1007A000002390ED000A04221B211846F2F772FF85
:1007B0000BE0B8F80010CDE90014002390ED000A1A
:1007C00003221B211846F2F765FFB8F80000CDE9B7
:1007D00000040023A4A21B215320F2F7F1FCA3483C
:1007E000A34E90ED000A10EE101AB9420BDA3188D0
:1007F000CDE90014002390ED000A042237211846A9
:10080000F2F748FF23E090ED000A10EE101AB9420B
:1008100012DB90ED000A974A10EE101A91420BDAA3
:100820003188CDE90014002390ED000A032237211E
:100830001846F2F72FFF0AE03188CDE900140023B3
:1008400090ED000A022237211846F2F723FF308884
:10085000CDE90004002388A237215320F2F7B0FC31
:10086000FF20B8F80010CDE900104F2368220021C6
:100870006720F1F73FFC3088F2F79CFC02217720DB
:10088000F2F78CFC1020F2F78FFC7C4C207A0428C5
:100890000CD07BA0F2F71AF97A480078072838D2F2
:1008A000DFE800F0370810182028300076A0F2F7B3
:1008B0000DF9F1E72888F2F77DFC19217520F2F790
:1008C0006DFC26E02888F2F775FC19218320F2F7E9
:1008D00065FC1EE02888F2F76DFC19218C20F2F7E8
:1008E0005DFC16E03088F2F765FC2D217520F2F7EB
:1008F00055FC0EE03088F2F75DFC2D218320F2F7E5
:100900004DFC06E03088F2F755FC2D218C20F2F7E3
:1009100045FC5EA0F2F7DAF82888F2F74BFC1721C5
:100920006C20F2F73BFC608900EE100AB8EE400A3A
:10093000DFED570A20EE208A217A042907D100EE44
:10094000100AB8EE400ADFED530A20EE208A18EEB6
:10095000100AB8420BDA50A0F2F7B8F80220B0EE55
:10096000480AF2F763FB3DA0F2F7B0F807E0022077
:10097000B0EE480AF2F75AFB38A0F2F7A7F8B8F839
:100980000000F2F717FC2B216C20F2F707FC207B0C
:1009900000EE100AB8EE400ADFED400A20EE208A91
:1009A0003DA0F2F793F80220B0EE480AF2F73EFBC2
:1009B0002DA0F2F78BF83088F2F7FCFB384F38782F
:1009C000384D4FF010042978084208D03088CDE91E
:1009D0000004002334A23F216A20F2F7F1FB3878AB
:1009E0002978884308D03088CDE9000400232FA25D
:1009F0003F216A20F2F7E4FB28783978884308D051
:100A00003088CDE90004002328A23F216A20F2F7B4
:100A1000D7FB387850B9287840B93088CDE9000440
:100A2000002321A23F216A20F2F7CAFB40217C204B
:100A3000F2F7B4FB1E49002091ED000AF2F7F6FA36
:100A400002B01CA0BDEC028BBDE8F041F2F73EB84D
:100A50003483FF1F00002041A883FF1F56000000C1
:100A60003C83FF1FAA83FF1F410000004083FF1F3C
:100A7000AC83FF1F0000C8425700000044B7FF1FAF
:100A8000505053006C8DFF1F415653005F00000013
:100A90000AD7A33CCDCCCC3C30000000CDCC4C3DA3
:100AA0003083FF1FA683FF1F3E0000003C000000B4
:100AB0008483FF1FA1E600002DE9F0410021484C8E
:100AC000DFF820C1207A9CF80020042807D0072AEC
:100AD00022D2DFE802F02116181A1C1E2000072A75
:100AE0001AD2DFE802F019040619080A0C002821BE
:100AF00012E0042110E014210EE002210CE001219B
:100B00000AE0322108E0052106E0012104E0142179
:100B100002E0022100E00121334E96F800803048C7
:100B2000304FB8F1040F037E7F7845891F44037B63
:100B3000F8B211D037780A2F0ED096F8008001272E
:100B4000B8F1050F20D096F80080B8F10B0F1BD03C
:100B5000307806282FD036E0032A0AD8294489B2F3
:100B60006181A28A914200D962816076F6F73CFAEF
:100B700029E01944C9B22173627B914200D92273E2
:100B80006076F6F731FA1EE0042A0AD2691A89B2B1
:100B90006181E28A914200D262816076F6F724FA9E
:100BA00011E08B4202D9591A217300E02773607655
:100BB000F6F71AFA07E0521CD0B28CF800000628AB
:100BC00001D98CF800703078062805D030780528D7
:100BD00002D03078042801D100203070BDE8F081C7
:100BE00044B7FF1F6C8DFF1F6083FF1F70B5044665
:100BF0000D461048044200D124B940F286210EA0CF
:100C0000F4F70CFD35B1012D04D040F287210AA084
:100C1000F4F704FD144813490161012D06D0016861
:100C2000214301600F49491E016170BD0168A14364
:100C30000160F7E7EE3A0C702E2E5C2E2E5C2E2E05
:100C40005C2E2E5C2E2E5C6472697665725C73720B
:100C5000635C68633332663436305F7077632E636B
:100C6000000000000100A5A50080044070B5044606
:100C70000D460E48044200D124B940F2BF210CA019
:100C8000F4F7CCFC35B1012D04D04FF4307108A03D
:100C9000F4F7C4FC1148012D03D0416821434160A1
:100CA00070BD4168A143416070BD00008602F0F054
:100CB0002E2E5C2E2E5C2E2E5C2E2E5C2E2E5C6438
:100CC00072697665725C7372635C68633332663432
:100CD00036305F7077632E630000000000800440B0
:100CE00070B504460D460E48044200D124B94FF4B5
:100CF0003C710CA0F4F792FC35B1012D04D040F208
:100D0000F12108A0F4F78AFC1148012D03D0816875
:100D10002143816070BD8168A143816070BD000086
:100D20000078F8FF2E2E5C2E2E5C2E2E5C2E2E5C74
:100D30002E2E5C6472697665725C7372635C6863A4
:100D40003332663436305F7077632E630000000004
:100D50000080044070B504460D4641F2131034EA99
:100D6000000000D124B940F215310BA0F4F756FC75
:100D700035B1012D04D040F2163107A0F4F74EFC36
:100D80001048012D03D0C1682143C16070BDC16806
:100D9000A143C16070BD00002E2E5C2E2E5C2E2E55
:100DA0005C2E2E5C2E2E5C6472697665725C7372AA
:100DB000635C68633332663436305F7077632E630A
:100DC000000000000080044010B50446002C06D04E
:100DD000012C04D04FF416710FA0F4F71FFC194A30
:100DE000B2F8FE034AF202510843A2F8FE03164984
:100DF000012C0CD0087820F080000870B2F8FE03B7
:100E000020F0020040F42540A2F8FE0310BD08784F
:100E100040F08000F1E700002E2E5C2E2E5C2E2E7E
:100E20005C2E2E5C2E2E5C6472697665725C737229
:100E3000635C68633332663436305F7077632E6389
:100E400000000000004005400A44054010B5AFF323
:100E5000008010BD1CB500200090019001208DF88D
:100E6000000002208DF8050001026A460120FFF70C
:100E7000A5FA6A4610210120FFF7A0FAF4F788FBD3
:100E8000F4F762FB1CBD1CB500200090019001200E
:100E90008DF8000002208DF8050001026A4601204D
:100EA000FFF78CFA6A4610210120FFF787FAF4F762
:100EB0007BFBF4F755FB1CBD2DE9FC4799490A78EB
:100EC000DFF864820024042A98F8030006D00A7828
:100ED000052A0DD00978062914D03CE0042803D255
:100EE000401C88F8030001E088F803400C7032E0F1
:100EF00018B1401E88F8030002E0042088F80300BF
:100F00000C7028E098F8041041B1042806D000F0D5
:100F1000E9FAC820F4F7A2FB88F8044098F8030027
:100F2000052818D2DFE800F00306090C0F0000F0D6
:100F3000D9FA10E000F0EFFA0DE0FFF78BFF0AE0BE
:100F4000FFF7A1FF07E000F01DF90C2088F8010071
:100F5000012088F804001020F2F726F9734D288844
:100F6000F2F728F900210846F2F718F970A0F1F716
:100F7000ADFD00215820F2F711F96F49012091EDE4
:100F8000000AF2F753F86DA0F1F7A0FD6C4E30782F
:100F90006C4F4FF010043978084208D02888CDE90A
:100FA0000004002368A219469020F2F709F930786E
:100FB0003978884308D02888CDE90004002363A24B
:100FC00019469020F2F7FCF838783178884308D039
:100FD0002888CDE9000400235CA219469020F2F78E
:100FE000EFF8307850B9387840B92888CDE9000456
:100FF000002355A219469020F2F7E2F815210020AF
:10100000F2F7CCF80024DFF82091514F514E09F14E
:10101000D0093088F2F7CEF898F80300844202D164
:101020003888F2F7C7F804EB840059F82000F1F78C
:101030004DFD00210920F0F745FF641CE4B2062CA9
:10104000E7D328210520F2F7A9F82888F2F7B2F8AB
:1010500041A0F1F73BFD4149022091ED000AF1F773
:10106000E5FF3FA0F1F732FD00211120F0F72AFF44
:101070003CA0F1F72BFD3C49022091ED000AF1F76D
:10108000D5FF37A0F1F722FD3888F2F793F83C211D
:101090000020F2F783F8354C354D94ED000A10EE40
:1010A000100AA8420BDA33A0F1F710FD032094EDEB
:1010B000000AF1F7BBFF2AA0F1F708FD0AE02DA016
:1010C000F1F704FD022094ED000AF1F7AFFF24A030
:1010D000F1F7FCFC00210F20F0F7F4FE3088F2F766
:1010E00069F8264991ED000A10EE100AA84205DAC7
:1010F000032091ED000AF1F799FF04E0022091ED41
:10110000000AF1F793FF1EA0F1F7E0FCFF20318801
:10111000CDE9001010239F2219460020F0F7EAFFC6
:10112000BDE8FC876083FF1FB083FF1FAC83FF1FF8
:101130005143322E300000008483FF1FA1E60000DF
:101140003083FF1FA683FF1F3E0000003C0000000D
:10115000A883FF1FAA83FF1F442B3A008883FF1F29
:1011600056000000442D3A008C83FF1F3483FF1F7C
:10117000000020414E4F573A000000003C83FF1F03
:10118000410000001CB500200090019001208DF866
:10119000000002208DF8050001026A460120FFF7D9
:1011A0000DF96A4610210120FFF708F9F4F7F0F96C
:1011B000F4F7D6F91CBD00002DE9FC47A44E3078A9
:1011C000042809D030780A2806D03078052806D0BF
:1011D00030780B2803D004E000F076F901E000F04D
:1011E00065F93078042802D03078052801D1002034
:1011F00030709848DFF860921C2490ED000ADFF808
:101200005C8210EE101A49450CDAB8F80010CDE9EE
:101210000014002390ED000A042219461846F2F744
:1012200039FA0BE0B8F80010CDE90014002390ED76
:10123000000A032219461846F2F72CFAB8F8000003
:10124000CDE90004002386A219465320F1F7B8FF28
:101250008448854F90ED000A10EE101A49450BDACC
:101260003988CDE90014002390ED000A04221B21E7
:101270001846F2F70FFA0AE03988CDE90014002386
:1012800090ED000A03221B211846F2F703FA388872
:10129000CDE90004002375A21B215320F1F790FF34
:1012A0007348744D90ED000A10EE101A49450BDAA0
:1012B0002988CDE90014002390ED000A042237218B
:1012C0001846F2F7E7F923E090ED000A10EE101A45
:1012D000494512DB90ED000A674A10EE101A914260
:1012E0000BDA2988CDE90014002390ED000A0322CF
:1012F00037211846F2F7CEF90AE02988CDE9001423
:10130000002390ED000A022237211846F2F7C2F9B5
:101310002888CDE90004002358A237215320F1F793
:101320004FFFFF203988CDE900104F2368220021AC
:101330006720F0F7DFFE10242888CDE900040023A1
:101340004FA203217720F1F73BFF3078012846D0E8
:1013500030780A2843D03888CDE90004002349A218
:1013600017216F20F1F72CFF3078022842D0307817
:101370000B283FD03888CDE90004002343A22B215D
:101380007020F1F71DFF434F3878434E3178084203
:1013900008D02888CDE90004002340A23F216A201C
:1013A000F1F70EFF38783178884308D02888CDE9E6
:1013B000000400233AA23F216A20F1F701FF3078B0
:1013C0003978884308D02888CDE90004002334A266
:1013D0003F216A20F1F7F4FE3878B0B120E0B8F888
:1013E0000000CDE90004002326A217216F20F1F7A9
:1013F000E7FEB9E7B8F80000CDE90004002323A216
:101400002B217020F1F7DCFEBDE7307840B9288849
:10141000CDE90004002321A23F216A20F1F7D0FE8C
:101420002888CDE900041F4800231A4690ED000AE1
:101430003F217C20F2F72EF92888CDE90004002313
:1014400019A23F218E20F1F7BBFEBDE8FC8700000A
:101450006083FF1F3483FF1F00002041A883FF1F0C
:10146000560000003C83FF1FAA83FF1F41000000BD
:101470004083FF1FAC83FF1F0000C84257000000DD
:10148000514333002B302E32560000002D302E32C7
:10149000560000003083FF1FA683FF1F3E000000A0
:1014A0003C0000008483FF1FA1E6000010B5F4F7A4
:1014B0006FF8F4F749F80A20F4F7D0F8F4F768F871
:1014C000BDE81040F4F74CB810B5F4F76DF8F4F738
:1014D00047F80A20F4F7C2F8F4F75AF8BDE81040CC
:1014E000F4F73EB81CB500200090019001208DF863
:1014F000000002208DF8050001026A460120FEF777
:101500005DFF6A4610210120FEF758FFF4F740F80E
:10151000F4F70EF81CBD1CB50020009001900120CE
:101520008DF8000002208DF8050001026A460120B6
:10153000FEF744FF6A4610210120FEF73FFFF4F753
:1015400033F8F4F701F81CBD1CB5002000900190A1
:1015500001208DF8000002208DF80500C1016A46C7
:101560000120FEF72BFF6A4608210120FEF726FF27
:10157000F4F70EF81CBD1CB5002400940194F3F799
:10158000FBFFF3F7D5FF0A20F4F768F88DF8004069
:101590006A464FF480710120FEF710FF6A46082169
:1015A0000120FEF70BFF6A464FF400710120FEF7A1
:1015B00005FF6A4610210120FEF700FF1CBD000058
:1015C0002DE9F05FFE480178FE4EFF4FFF4D4FF0D2
:1015D000000A002913D00178052905D001780429D3
:1015E00002D00178062908D1297931B180F800A00C
:1015F00085F804A03079F9F7FFFB38686862F07865
:101600000124072855D054D2DFE800F004101C282C
:10161000333E49003868696A401A43F69821884287
:1016200047D92C717079F9F7E7FB42E03868696AAD
:10163000401A47F2305188423BD92C717079F9F742
:10164000DBFB36E03868696A401A4EF66021884252
:101650002FD92C717079F9F7CFFB2AE03868696AC5
:10166000401ADB49884224D92C717079F9F7C4FB00
:101670001FE03868696A401AD649884219D92C7126
:101680007079F9F7B9FB14E03868696A401AD249F1
:1016900088420ED92C717079F9F7AEFB09E03868F1
:1016A000696A401ACD49884203D92C717079F9F7DB
:1016B000A3FBDFF82C83CB4EDFF82C9398ED000AC8
:1016C00010EE100AB0F1804F32DA3868B0F57A7F48
:1016D0002ED9B07B20B172B6F4F792FA62B61FE051
:1016E00099F80000152804D099F800000D280CD0B6
:1016F00016E072B6F4F7FCFA62B6B07B03280FD19D
:10170000B473152089F800000AE072B6F4F7F0FA15
:10171000B07B032803D1B4730D2089F8000062B6B2
:10172000B24E307888B1FFF726FF86F800A00CE0B3
:1017300098ED000AAE4910EE100A884205DBB07B36
:1017400018B972B6F4F7A2FA62B63868E96E401AB0
:10175000C8287DD3EFF7FCFC08F0B2FC06F004FBD0
:1017600099F80000DFEDA31AA34E032804D099F8DE
:1017700000000F2855D0CEE0002200219F480078BD
:1017800020B11E230020DFF878B20CE09D480078DD
:10179000401CC3B2F6E73BF810C08C4500D9614647
:1017A0006244401CC0B29842F5D39748DFF85CC24F
:1017B00000880A2818D2B2FBF3F000EE100AB8EE47
:1017C000400ADFED930A60EE200A00EE101AB8EE30
:1017D000400A9FED901A40EE010ABCEEE00A10EEBE
:1017E000100AACF8000017E0B2FBF3F000EE100AAC
:1017F000F6EE080AB5EE001AB8EE400A60EE200ACE
:1018000000EE101AB8EE400A40EE010ABCEEE00A03
:1018100010EE100AACF800007F488049008808806C
:1018200079E07F48D0ED000A7E4890ED001ADFEDA8
:101830007E2A7E489FED7E0AF4EEC10AB1EE0C2AA4
:10184000F1EE10FA7B4A7C4931DD96ED003A00E07A
:10185000D5E113EE103A934229DD70EEC10A80EE15
:10186000A21AD0ED000AD6ED002AA87901EB800279
:1018700021EE201AC1EE220A60EEA10AC2ED000A92
:10188000062802D2401CA87145E0002001EB80022E
:10189000D2ED000A30EE800A401CC0B20728F5D312
:1018A000C0EE020AC5ED190A85F806A033E096EDF0
:1018B000003A13EE103A934229DD31EE601AC1EE80
:1018C000220A90ED001AD6ED002AA87901EB8002D9
:1018D00020EE811AC1EE220A60EEA10AC2ED000AD2
:1018E000062802D2401CA87115E0002001EB8002FE
:1018F000D2ED000A30EE800A401CC0B20728F5D3B2
:10190000C0EE020AC5ED190A85F806A003E085F8C5
:1019100006A085ED190A98ED000A688960EE210A93
:1019200000EE100AB8EE400AF4EEC00AF1EE10FA2A
:1019300008DD98ED000A20EE210ABCEEC00A10EE88
:10194000100A688196ED000AA88960EE210A00EE6F
:10195000100AB8EE400AF4EEC00AF1EE10FA08DD03
:1019600096ED000A20EE210ABCEEC00A10EE100A25
:10197000A881E889401C80B2E8812F492B8A1C315C
:1019800001F5A072984218D198ED000AE87920EE8E
:10199000210ABCEEC00A10EE10CA21F810C096ED64
:1019A000000A20EE210ABCEEC00A10EE10CA22F88E
:1019B00010C0401CE871A5F80EA0E879A0283DE011
:1019C0006083FF1F746102207C83FF1FF48CFF1F64
:1019D000C0D40100E0930400C027090040771B0039
:1019E0003483FF1F44B7FF1FB183FF1FB283FF1F64
:1019F0000000404000007A443C83FF1FB883FF1F73
:101A00004C390220B783FF1FD083FF1FD483FF1FF1
:101A10006666263F3333B33ED683FF1FD883FF1F4E
:101A20009083FF1F9483FF1F00F07F458083FF1F7B
:101A300000000000CDCCCC3ED85E022013D1502057
:101A4000E8714FF6FF7000EA43002882002031F869
:101A5000203021F8103032F8203022F81030401CAD
:101A6000C0B25028F3D3DFF89CB1DFF89CA106E0A8
:101A70001E2089F80000F8F7FBFE01F055FB9BF8EB
:101A800000009AF800100843F2D09BF8000060B9FB
:101A90003868296B401A5D49884206D99AF80000D7
:101AA00018B100F0B7F8386828639BF8000058B9FF
:101AB0003868B0F57A7F07D99AF8000020B16879C4
:101AC00010B900F0A7F86C71E869B0F5FA6F7DD92C
:101AD00098ED000AD5ED0D0AB4EEE00AF1EE10FA29
:101AE00004DD98ED000A85ED0D0A0CE098ED000A82
:101AF000D5ED130AB4EEE00AF1EE10FA03D298ED38
:101B0000000A85ED130A96ED000AD5ED0E0AB4EE33
:101B1000E00AF1EE10FA04DD96ED000A85ED0E0AFA
:101B20000CE096ED000AD5ED140AB4EEE00AF1EEF1
:101B300010FA03D296ED000A85ED140A344AD5ED69
:101B40000F0A92ED000AB4EEE00AF1EE10FA04DD9D
:101B500092ED000A85ED0F0A0CE092ED000AD5ED3A
:101B6000150AB4EEE00AF1EE10FA03D292ED000A83
:101B700085ED150AA96ED5ED160A411A00EE101A68
:101B800098ED001AB8EE400A41EE000AC5ED160ABB
:101B900000EE101AD6ED001AB8EE401A95ED170AAD
:101BA00001EE810A85ED170A01EE101A92ED002A66
:101BB000F8EE411A95ED181A02EE211A85ED181A61
:101BC000A866A0F5FA6001EE900A00E015E0F8EED4
:101BD000611A80EEA12A85ED102A00EE900AF8EE37
:101BE000600AC0EE201AC5ED111A00EE100AB8EE18
:101BF000400AC1EE000AC5ED120A3868E866BDE881
